 usersEditor

 Timestamp is 614c802e (Thu Sep 23 13:25:02 2021)

 Preferred load address is 10000000

 Start         Length     Name                   Class
 0001:00000000 000000c6H .text$di                CODE
 0001:000000d0 000055ccH .text$mn                CODE
 0001:0000569c 00000e26H .text$x                 CODE
 0001:000064c2 00000042H .text$yd                CODE
 0002:00000000 00000a28H .idata$5                DATA
 0002:00000a28 00000004H .CRT$XCA                DATA
 0002:00000a2c 00000018H .CRT$XCU                DATA
 0002:00000a44 00000004H .CRT$XCZ                DATA
 0002:00000a48 00000004H .CRT$XIA                DATA
 0002:00000a4c 00000004H .CRT$XIAA               DATA
 0002:00000a50 00000004H .CRT$XIC                DATA
 0002:00000a54 00000004H .CRT$XIZ                DATA
 0002:00000a58 000024c0H .rdata                  DATA
 0002:00002f18 00000d44H .rdata$r                DATA
 0002:00003c5c 00000004H .rtc$IAA                DATA
 0002:00003c60 00000004H .rtc$IZZ                DATA
 0002:00003c64 00000004H .rtc$TAA                DATA
 0002:00003c68 00000004H .rtc$TZZ                DATA
 0002:00003c70 00000ddcH .xdata$x                DATA
 0002:00004a50 0000005fH .edata                  DATA
 0002:00004ab0 00000050H .idata$2                DATA
 0002:00004b00 00000014H .idata$3                DATA
 0002:00004b14 00000a28H .idata$4                DATA
 0002:0000553c 00006632H .idata$6                DATA
 0003:00000000 00000084H .data                   DATA
 0003:00000084 000004a0H .data$r                 DATA
 0003:00000528 000003dcH .bss                    DATA
 0004:00000000 000000a0H .rsrc$01                DATA
 0004:000000a0 00000608H .rsrc$02                DATA

  Address         Publics by Value              Rva+Base       Lib:Object

 0000:00000000       ___guard_flags             00000000     <absolute>
 0000:00000000       ___safe_se_handler_count   00000000     <absolute>
 0000:00000000       ___guard_fids_table        00000000     <absolute>
 0000:00000000       ___safe_se_handler_table   00000000     <absolute>
 0000:00000000       ___guard_fids_count        00000000     <absolute>
 0000:00000000       ___ImageBase               10000000     <linker-defined>
 0001:000000d0       ??0bncsTable@@QAE@PAVQWidget@@PBD@Z 100010d0 f   bncsTable.obj
 0001:000000f6       ??1bncsTable@@UAE@XZ       100010f6 f   bncsTable.obj
 0001:00000109       ??_EbncsTable@@WCI@AEPAXI@Z 10001109 f i bncsTable.obj
 0001:00000111       ??_EbncsTable@@UAEPAXI@Z   10001111 f i bncsTable.obj
 0001:00000111       ??_GbncsTable@@UAEPAXI@Z   10001111 f i bncsTable.obj
 0001:00000130       ?doCopy@bncsTable@@QAEXXZ  10001130 f   bncsTable.obj
 0001:000002c2       ?doUndo@bncsTable@@QAEXXZ  100012c2 f   bncsTable.obj
 0001:000002c2       ?doPaste@bncsTable@@QAEXXZ 100012c2 f   bncsTable.obj
 0001:000002c2       ?apply@config_plugin_base@@UAEXXZ 100012c2 f   usersEditor.obj
 0001:000002c2       ?doDelete@bncsTable@@QAEXXZ 100012c2 f   bncsTable.obj
 0001:000002c3       ?keyPressEvent@bncsTable@@UAEXPAVQKeyEvent@@@Z 100012c3 f   bncsTable.obj
 0001:0000030c       ?metaObject@bncsTable@@UBEPAVQMetaObject@@XZ 1000130c f i bncsTable.obj
 0001:00000311       ?validateRow@bncsTable@@MAE_NH@Z 10001311 f   bncsTable.obj
 0001:00000316       ??0panelsetsTableItem@@QAE@ABVQString@@PAVQTable@@W4EditType@QTableItem@@0@Z 10001316 f   panelsetsTableItem.obj
 0001:00000363       ??1panelsetsTableItem@@UAE@XZ 10001363 f   panelsetsTableItem.obj
 0001:00000399       ??_EQComboBox@@WCI@AEPAXI@Z 10001399 f i panelsetsTableItem.obj
 0001:000003a1       ??_GQComboBox@@UAEPAXI@Z   100013a1 f i panelsetsTableItem.obj
 0001:000003a1       ??_EQComboBox@@UAEPAXI@Z   100013a1 f i panelsetsTableItem.obj
 0001:000003c1       ??_GpanelsetsTableItem@@UAEPAXI@Z 100013c1 f i panelsetsTableItem.obj
 0001:000003c1       ??_EpanelsetsTableItem@@UAEPAXI@Z 100013c1 f i panelsetsTableItem.obj
 0001:000003e0       ?createEditor@panelsetsTableItem@@UBEPAVQWidget@@XZ 100013e0 f   panelsetsTableItem.obj
 0001:0000066a       ?setContentFromEditor@panelsetsTableItem@@UAEXPAVQWidget@@@Z 1000166a f   panelsetsTableItem.obj
 0001:0000066a       ?setContentFromEditor@userLevelTableItem@@UAEXPAVQWidget@@@Z 1000166a f   userLevelTableItem.obj
 0001:00000708       ??_Econfig_plugin_desc_base@@UAEPAXI@Z 10001708 f i plugindesc.obj
 0001:00000708       ??_Gplugindesc@@UAEPAXI@Z  10001708 f i plugindesc.obj
 0001:00000708       ??_Eplugindesc@@UAEPAXI@Z  10001708 f i plugindesc.obj
 0001:00000708       ??_Gconfig_plugin_desc_base@@UAEPAXI@Z 10001708 f i plugindesc.obj
 0001:00000728       ?create@plugindesc@@UAEPAVconfig_plugin_base@@ABVQString@@00@Z 10001728 f   plugindesc.obj
 0001:00000763       ?keys@plugindesc@@UAE?AVQStringList@@ABVQString@@0@Z 10001763 f   plugindesc.obj
 0001:000007be       ?pixmap@plugindesc@@UAE?AVQPixmap@@ABVQString@@@Z 100017be f   plugindesc.obj
 0001:000007dd       _load_bncs_config_plugin_desc 100017dd f   plugindesc.obj
 0001:000007f3       ??0userLevelTableItem@@QAE@ABVQString@@PAVQTable@@W4EditType@QTableItem@@0@Z 100017f3 f   userLevelTableItem.obj
 0001:00000840       ??1userLevelTableItem@@UAE@XZ 10001840 f   userLevelTableItem.obj
 0001:00000876       ??_EuserLevelTableItem@@UAEPAXI@Z 10001876 f i userLevelTableItem.obj
 0001:00000876       ??_GuserLevelTableItem@@UAEPAXI@Z 10001876 f i userLevelTableItem.obj
 0001:00000895       ?createEditor@userLevelTableItem@@UBEPAVQWidget@@XZ 10001895 f   userLevelTableItem.obj
 0001:00000a3c       ??0?$QGuardedPtr@VQPopupMenu@@@@QAE@XZ 10001a3c f i usersEditor.obj
 0001:00000a3c       ??0?$QGuardedPtr@VQDockWindow@@@@QAE@XZ 10001a3c f i usersEditor.obj
 0001:00000a7d       ??0config_plugin_base@@QAE@ABVQString@@00@Z 10001a7d f i usersEditor.obj
 0001:00000b0a       ??0usersEditor@@QAE@ABVQString@@00@Z 10001b0a f   usersEditor.obj
 0001:00001130       ??1?$QDict@VQAction@@@@UAE@XZ 10002130 f i usersEditor.obj
 0001:00001163       ??1?$QGuardedPtr@VQDockWindow@@@@QAE@XZ 10002163 f i usersEditor.obj
 0001:00001163       ??1?$QGuardedPtr@VQPopupMenu@@@@QAE@XZ 10002163 f i usersEditor.obj
 0001:00001168       ??1?$QPtrList@VQPopupMenu@@@@UAE@XZ 10002168 f i usersEditor.obj
 0001:0000119b       ??1QDockWindowList@@UAE@XZ 1000219b f i usersEditor.obj
 0001:000011e4       ??1QPopupMenuList@@UAE@XZ  100021e4 f i usersEditor.obj
 0001:00001216       ??1config_plugin_base@@UAE@XZ 10002216 f i usersEditor.obj
 0001:00001270       ??1usersEditor@@UAE@XZ     10002270 f   usersEditor.obj
 0001:00001320       ??4?$QGuardedPtr@VQDockWindow@@@@QAEAAV0@PAVQDockWindow@@@Z 10002320 f i usersEditor.obj
 0001:00001320       ??4?$QGuardedPtr@VQPopupMenu@@@@QAEAAV0@PAVQPopupMenu@@@Z 10002320 f i usersEditor.obj
 0001:0000137e       ??_EQPopupMenu@@WCI@AEPAXI@Z 1000237e f i usersEditor.obj
 0001:00001386       ??_EQPopupMenu@@WIM@AEPAXI@Z 10002386 f i usersEditor.obj
 0001:00001391       ??_EQToolBar@@WCI@AEPAXI@Z 10002391 f i usersEditor.obj
 0001:00001399       ??_Econfig_plugin_base@@WCI@AEPAXI@Z 10002399 f i usersEditor.obj
 0001:000013a1       ??_EusersEditor@@WCI@AEPAXI@Z 100023a1 f i usersEditor.obj
 0001:000013a9       ??_E?$QDict@VQAction@@@@UAEPAXI@Z 100023a9 f i usersEditor.obj
 0001:000013a9       ??_G?$QDict@VQAction@@@@UAEPAXI@Z 100023a9 f i usersEditor.obj
 0001:000013c8       ??_E?$QPtrList@VQPopupMenu@@@@UAEPAXI@Z 100023c8 f i usersEditor.obj
 0001:000013c8       ??_G?$QPtrList@VQPopupMenu@@@@UAEPAXI@Z 100023c8 f i usersEditor.obj
 0001:000013e7       ??_EQAction@@UAEPAXI@Z     100023e7 f i usersEditor.obj
 0001:000013e7       ??_GQAction@@UAEPAXI@Z     100023e7 f i usersEditor.obj
 0001:00001407       ??_EQDockWindowList@@UAEPAXI@Z 10002407 f i usersEditor.obj
 0001:00001407       ??_GQDockWindowList@@UAEPAXI@Z 10002407 f i usersEditor.obj
 0001:00001426       ??_GQGuardedPtrPrivate@@UAEPAXI@Z 10002426 f i usersEditor.obj
 0001:00001426       ??_EQGuardedPtrPrivate@@UAEPAXI@Z 10002426 f i usersEditor.obj
 0001:00001446       ??_GQPopupMenu@@UAEPAXI@Z  10002446 f i usersEditor.obj
 0001:00001446       ??_EQPopupMenu@@UAEPAXI@Z  10002446 f i usersEditor.obj
 0001:00001466       ??_GQPopupMenuList@@UAEPAXI@Z 10002466 f i usersEditor.obj
 0001:00001466       ??_EQPopupMenuList@@UAEPAXI@Z 10002466 f i usersEditor.obj
 0001:00001485       ??_GQToolBar@@UAEPAXI@Z    10002485 f i usersEditor.obj
 0001:00001485       ??_EQToolBar@@UAEPAXI@Z    10002485 f i usersEditor.obj
 0001:000014a5       ??_Gconfig_plugin_base@@UAEPAXI@Z 100024a5 f i usersEditor.obj
 0001:000014a5       ??_Econfig_plugin_base@@UAEPAXI@Z 100024a5 f i usersEditor.obj
 0001:000014c4       ??_GusersEditor@@UAEPAXI@Z 100024c4 f i usersEditor.obj
 0001:000014c4       ??_EusersEditor@@UAEPAXI@Z 100024c4 f i usersEditor.obj
 0001:000014e3       ?about@config_plugin_base@@UAE?AVQString@@XZ 100024e3 f i usersEditor.obj
 0001:00001539       ?about@usersEditor@@UAE?AVQString@@XZ 10002539 f   usersEditor.obj
 0001:000015e1       ?activate@usersEditor@@UAEX_N@Z 100025e1 f   usersEditor.obj
 0001:000018a8       ?apply@usersEditor@@UAEXXZ 100028a8 f   usersEditor.obj
 0001:0000193f       ?clear@?$QDict@VQAction@@@@UAEXXZ 1000293f f i usersEditor.obj
 0001:00001945       ?clear@?$QPtrList@VQPopupMenu@@@@UAEXXZ 10002945 f i usersEditor.obj
 0001:00001945       ?clear@?$QPtrList@H@@UAEXXZ 10002945 f i usersEditordlgimpl.obj
 0001:0000194b       ?closeEvent@config_plugin_base@@UAEXPAVQCloseEvent@@@Z 1000294b f i usersEditor.obj
 0001:00001959       ?closeEvent@usersEditor@@UAEXPAVQCloseEvent@@@Z 10002959 f   usersEditor.obj
 0001:000019b5       ?count@?$QDict@VQAction@@@@UBEIXZ 100029b5 f i usersEditor.obj
 0001:000019b9       ?db@@YAXABVQString@@@Z     100029b9 f   usersEditor.obj
 0001:00001a01       ?deleteItem@?$QDict@VQAction@@@@EAEXPAX@Z 10002a01 f i usersEditor.obj
 0001:00001a01       ?deleteItem@?$QPtrList@VQPopupMenu@@@@EAEXPAX@Z 10002a01 f i usersEditor.obj
 0001:00001a1c       ?deref@?$QGuardedPtr@VQPopupMenu@@@@AAEXXZ 10002a1c f i usersEditor.obj
 0001:00001a1c       ?deref@?$QGuardedPtr@VQDockWindow@@@@AAEXXZ 10002a1c f i usersEditor.obj
 0001:00001a31       ?fileSelected@usersEditor@@AAEXABVQString@@@Z 10002a31 f   usersEditor.obj
 0001:00001aa9       ?validate@config_plugin_base@@UAE_NXZ 10002aa9 f i usersEditor.obj
 0001:00001aa9       ?isDirty@config_plugin_base@@UAE_NXZ 10002aa9 f i usersEditor.obj
 0001:00001aac       ?isDirty@usersEditor@@UAE_NXZ 10002aac f   usersEditor.obj
 0001:00001ab6       ?menus@config_plugin_base@@UAE?AVQPopupMenuList@@XZ 10002ab6 f i usersEditor.obj
 0001:00001ad9       ?menus@usersEditor@@UAE?AVQPopupMenuList@@XZ 10002ad9 f   usersEditor.obj
 0001:00001b23       ?metaObject@usersEditor@@UBEPAVQMetaObject@@XZ 10002b23 f i usersEditor.obj
 0001:00001b28       ?navigate@config_plugin_base@@UAEXABVQString@@0@Z 10002b28 f i usersEditor.obj
 0001:00001b2b       ?navigate@usersEditor@@UAEXABVQString@@0@Z 10002b2b f   usersEditor.obj
 0001:00001ba7       ?reply@config_plugin_base@@UAEXPAVresponse@@@Z 10002ba7 f i usersEditor.obj
 0001:00001ba7       ?activate@config_plugin_base@@UAEX_N@Z 10002ba7 f i usersEditor.obj
 0001:00001baa       ?reply@usersEditor@@UAEXPAVresponse@@@Z 10002baa f   usersEditor.obj
 0001:00001ed3       ?resizeEvent@usersEditor@@UAEXPAVQResizeEvent@@@Z 10002ed3 f   usersEditor.obj
 0001:00001f08       ?textStatus@response@@QAE?AVQString@@W4status@1@@Z 10002f08 f i usersEditor.obj
 0001:00001f57       ?toolbars@config_plugin_base@@UAE?AVQDockWindowList@@XZ 10002f57 f i usersEditor.obj
 0001:00001f7a       ?toolbars@usersEditor@@UAE?AVQDockWindowList@@XZ 10002f7a f   usersEditor.obj
 0001:00001fd2       ??0usersEditorDlg@@QAE@ABVQString@@PAVQWidget@@PBDI@Z 10002fd2 f   usersEditordlgimpl.obj
 0001:000023df       ??1?$QPtrList@H@@UAE@XZ    100033df f i usersEditordlgimpl.obj
 0001:00002412       ??1usersEditorDlg@@UAE@XZ  10003412 f   usersEditordlgimpl.obj
 0001:0000245e       ??_EusersEditorDlg@@WCI@AEPAXI@Z 1000345e f i usersEditordlgimpl.obj
 0001:00002466       ??_G?$QPtrList@H@@UAEPAXI@Z 10003466 f i usersEditordlgimpl.obj
 0001:00002466       ??_E?$QPtrList@H@@UAEPAXI@Z 10003466 f i usersEditordlgimpl.obj
 0001:00002485       ??_EQCheckTableItem@@UAEPAXI@Z 10003485 f i usersEditordlgimpl.obj
 0001:00002485       ??_GQCheckTableItem@@UAEPAXI@Z 10003485 f i usersEditordlgimpl.obj
 0001:000024a5       ??_EusersEditorDlg@@UAEPAXI@Z 100034a5 f i usersEditordlgimpl.obj
 0001:000024a5       ??_GusersEditorDlg@@UAEPAXI@Z 100034a5 f i usersEditordlgimpl.obj
 0001:000024c4       ?addUser@usersEditorDlg@@QAEXXZ 100034c4 f   usersEditordlgimpl.obj
 0001:00002791       ?count@?$QPtrList@VQPopupMenu@@@@UBEIXZ 10003791 f i usersEditor.obj
 0001:00002791       ?count@?$QPtrList@H@@UBEIXZ 10003791 f i usersEditordlgimpl.obj
 0001:00002795       ?deleteItem@?$QPtrList@H@@EAEXPAX@Z 10003795 f i usersEditordlgimpl.obj
 0001:000027ab       ?deleteUser@usersEditorDlg@@QAEXXZ 100037ab f   usersEditordlgimpl.obj
 0001:00002854       ?load@usersEditorDlg@@QAE_NABVQString@@@Z 10003854 f   usersEditordlgimpl.obj
 0001:00002ee7       ?metaObject@usersEditorDlg@@UBEPAVQMetaObject@@XZ 10003ee7 f i usersEditordlgimpl.obj
 0001:00002eec       ?save@usersEditorDlg@@QAEXABVQString@@@Z 10003eec f   usersEditordlgimpl.obj
 0001:0000330b       ?setClean@usersEditorDlg@@QAEXXZ 1000430b f   usersEditordlgimpl.obj
 0001:00003351       ?setDirty@usersEditorDlg@@QAEXXZ 10004351 f   usersEditordlgimpl.obj
 0001:00003397       ?setReadOnly@usersEditorDlg@@QAEX_N@Z 10004397 f   usersEditordlgimpl.obj
 0001:000033d2       ?textChanged@usersEditorDlg@@QAEXHH@Z 100043d2 f   usersEditordlgimpl.obj
 0001:0000342b       ?toXML@usersEditorDlg@@AAE?AVQString@@ABV2@@Z 1000442b f   usersEditordlgimpl.obj
 0001:000035c7       ?className@bncsTable@@UBEPBDXZ 100045c7 f   moc_bncsTable.obj
 0001:000035cd       ?qt_cast@bncsTable@@UAEPAXPBD@Z 100045cd f   moc_bncsTable.obj
 0001:000035fb       ?qt_emit@bncsTable@@UAE_NHPAUQUObject@@@Z 100045fb f   moc_bncsTable.obj
 0001:00003605       ?qt_invoke@bncsTable@@UAE_NHPAUQUObject@@@Z 10004605 f   moc_bncsTable.obj
 0001:00003655       ?qt_property@bncsTable@@UAE_NHHPAVQVariant@@@Z 10004655 f   moc_bncsTable.obj
 0001:0000365f       ?staticMetaObject@bncsTable@@SAPAVQMetaObject@@XZ 1000465f f   moc_bncsTable.obj
 0001:000036a9       ?staticMetaObject@toolWindowBase@@SAPAVQMetaObject@@XZ 100046a9 f   moc_toolwindow.obj
 0001:000036f3       ?staticMetaObject@toolWindow@@SAPAVQMetaObject@@XZ 100046f3 f   moc_toolwindowimpl.obj
 0001:0000379f       ?className@usersEditor@@UBEPBDXZ 1000479f f   moc_usersEditor.obj
 0001:000037a5       ?command@usersEditor@@IAEXVQString@@0@Z 100047a5 f   moc_usersEditor.obj
 0001:00003865       ?qt_cast@usersEditor@@UAEPAXPBD@Z 10004865 f   moc_usersEditor.obj
 0001:00003893       ?qt_emit@usersEditor@@UAE_NHPAUQUObject@@@Z 10004893 f   moc_usersEditor.obj
 0001:000038f7       ?qt_invoke@usersEditor@@UAE_NHPAUQUObject@@@Z 100048f7 f   moc_usersEditor.obj
 0001:0000392c       ?staticMetaObject@usersEditor@@SAPAVQMetaObject@@XZ 1000492c f   moc_usersEditor.obj
 0001:000039e7       ?className@usersEditorDlgBase@@UBEPBDXZ 100049e7 f   moc_usersEditordlg.obj
 0001:000039ed       ?qt_cast@usersEditorDlgBase@@UAEPAXPBD@Z 100049ed f   moc_usersEditordlg.obj
 0001:00003a1b       ?qt_emit@usersEditorDlgBase@@UAE_NHPAUQUObject@@@Z 10004a1b f   moc_usersEditordlg.obj
 0001:00003a25       ?qt_invoke@usersEditorDlgBase@@UAE_NHPAUQUObject@@@Z 10004a25 f   moc_usersEditordlg.obj
 0001:00003a57       ?qt_property@usersEditor@@UAE_NHHPAVQVariant@@@Z 10004a57 f   moc_usersEditor.obj
 0001:00003a57       ?qt_property@usersEditorDlgBase@@UAE_NHHPAVQVariant@@@Z 10004a57 f   moc_usersEditordlg.obj
 0001:00003a61       ?staticMetaObject@usersEditorDlgBase@@SAPAVQMetaObject@@XZ 10004a61 f   moc_usersEditordlg.obj
 0001:00003aab       ?tr@usersEditorDlgBase@@SA?AVQString@@PBD0@Z 10004aab f   moc_usersEditordlg.obj
 0001:00003aee       ?className@usersEditorDlg@@UBEPBDXZ 10004aee f   moc_usersEditordlgimpl.obj
 0001:00003af4       ?command@usersEditorDlg@@IAEXVQString@@0@Z 10004af4 f   moc_usersEditordlgimpl.obj
 0001:00003bb4       ?qt_cast@usersEditorDlg@@UAEPAXPBD@Z 10004bb4 f   moc_usersEditordlgimpl.obj
 0001:00003be1       ?qt_emit@usersEditorDlg@@UAE_NHPAUQUObject@@@Z 10004be1 f   moc_usersEditordlgimpl.obj
 0001:00003c44       ?qt_invoke@usersEditorDlg@@UAE_NHPAUQUObject@@@Z 10004c44 f   moc_usersEditordlgimpl.obj
 0001:00003c92       ?qt_property@usersEditorDlg@@UAE_NHHPAVQVariant@@@Z 10004c92 f   moc_usersEditordlgimpl.obj
 0001:00003c9b       ?staticMetaObject@usersEditorDlg@@SAPAVQMetaObject@@XZ 10004c9b f   moc_usersEditordlgimpl.obj
 0001:00003d78       ?tr@usersEditorDlg@@SA?AVQString@@PBD0@Z 10004d78 f   moc_usersEditordlgimpl.obj
 0001:00003dbb       ??_EQVBoxLayout@@WCI@AEPAXI@Z 10004dbb f i toolwindow.obj
 0001:00003dc3       ??_GQVBoxLayout@@UAEPAXI@Z 10004dc3 f i toolwindow.obj
 0001:00003dc3       ??_EQVBoxLayout@@UAEPAXI@Z 10004dc3 f i toolwindow.obj
 0001:00003de3       ??0usersEditorDlgBase@@QAE@PAVQWidget@@PBDI@Z 10004de3 f   usersEditordlg.obj
 0001:00003f23       ??1usersEditorDlgBase@@UAE@XZ 10004f23 f   usersEditordlg.obj
 0001:00003f36       ??_EQLabel@@WCI@AEPAXI@Z   10004f36 f i usersEditordlg.obj
 0001:00003f3e       ??_EusersEditorDlgBase@@WCI@AEPAXI@Z 10004f3e f i usersEditordlg.obj
 0001:00003f46       ??_GQLabel@@UAEPAXI@Z      10004f46 f i usersEditordlg.obj
 0001:00003f46       ??_EQLabel@@UAEPAXI@Z      10004f46 f i usersEditordlg.obj
 0001:00003f66       ??_GusersEditorDlgBase@@UAEPAXI@Z 10004f66 f i usersEditordlg.obj
 0001:00003f66       ??_EusersEditorDlgBase@@UAEPAXI@Z 10004f66 f i usersEditordlg.obj
 0001:00003f85       ?languageChange@usersEditorDlgBase@@MAEXXZ 10004f85 f   usersEditordlg.obj
 0001:0000402a       ?metaObject@usersEditorDlgBase@@UBEPAVQMetaObject@@XZ 1000502a f i usersEditordlg.obj
 0001:00004030       ?activateNextCell@QTable@@MAEXXZ 10005030 f   qt-mt323:qt-mt323.dll
 0001:00004036       ?addChild@QScrollView@@UAEXPAVQWidget@@HH@Z 10005036 f   qt-mt323:qt-mt323.dll
 0001:0000403c       ?addSelection@QTable@@UAEHABVQTableSelection@@@Z 1000503c f   qt-mt323:qt-mt323.dll
 0001:00004042       ?adjustColumn@QTable@@UAEXH@Z 10005042 f   qt-mt323:qt-mt323.dll
 0001:00004048       ?adjustRow@QTable@@UAEXH@Z 10005048 f   qt-mt323:qt-mt323.dll
 0001:0000404e       ?adjustSize@QWidget@@UAEXXZ 1000504e f   qt-mt323:qt-mt323.dll
 0001:00004054       ?beginEdit@QTable@@MAEPAVQWidget@@HH_N@Z 10005054 f   qt-mt323:qt-mt323.dll
 0001:0000405a       ?cellGeometry@QTable@@UBE?AVQRect@@HH@Z 1000505a f   qt-mt323:qt-mt323.dll
 0001:00004060       ?cellRect@QTable@@UBE?AVQRect@@HH@Z 10005060 f   qt-mt323:qt-mt323.dll
 0001:00004066       ?cellWidget@QTable@@UBEPAVQWidget@@HH@Z 10005066 f   qt-mt323:qt-mt323.dll
 0001:0000406c       ?checkConnectArgs@QObject@@MAE_NPBDPBV1@0@Z 1000506c f   qt-mt323:qt-mt323.dll
 0001:00004072       ?childEvent@QObject@@MAEXPAVQChildEvent@@@Z 10005072 f   qt-mt323:qt-mt323.dll
 0001:00004078       ?clearCell@QTable@@UAEXHH@Z 10005078 f   qt-mt323:qt-mt323.dll
 0001:0000407e       ?clearCellWidget@QTable@@UAEXHH@Z 1000507e f   qt-mt323:qt-mt323.dll
 0001:00004084       ?close@QWidget@@UAE_N_N@Z  10005084 f   qt-mt323:qt-mt323.dll
 0001:0000408a       ?closeEvent@QWidget@@MAEXPAVQCloseEvent@@@Z 1000508a f   qt-mt323:qt-mt323.dll
 0001:00004090       ?cmd@QPaintDevice@@MAE_NHPAVQPainter@@PATQPDevCmdParam@@@Z 10005090 f   qt-mt323:qt-mt323.dll
 0001:00004096       ?columnAt@QTable@@UBEHH@Z  10005096 f   qt-mt323:qt-mt323.dll
 0001:0000409c       ?columnClicked@QTable@@MAEXH@Z 1000509c f   qt-mt323:qt-mt323.dll
 0001:000040a2       ?columnIndexChanged@QTable@@MAEXHHH@Z 100050a2 f   qt-mt323:qt-mt323.dll
 0001:000040a8       ?columnPos@QTable@@UBEHH@Z 100050a8 f   qt-mt323:qt-mt323.dll
 0001:000040ae       ?columnWidth@QTable@@UBEHH@Z 100050ae f   qt-mt323:qt-mt323.dll
 0001:000040b4       ?columnWidthChanged@QTable@@MAEXH@Z 100050b4 f   qt-mt323:qt-mt323.dll
 0001:000040ba       ?connectNotify@QObject@@MAEXPBD@Z 100050ba f   qt-mt323:qt-mt323.dll
 0001:000040c0       ?contentsContextMenuEvent@QTable@@MAEXPAVQContextMenuEvent@@@Z 100050c0 f   qt-mt323:qt-mt323.dll
 0001:000040c6       ?contentsDragEnterEvent@QTable@@MAEXPAVQDragEnterEvent@@@Z 100050c6 f   qt-mt323:qt-mt323.dll
 0001:000040cc       ?contentsDragLeaveEvent@QTable@@MAEXPAVQDragLeaveEvent@@@Z 100050cc f   qt-mt323:qt-mt323.dll
 0001:000040d2       ?contentsDragMoveEvent@QTable@@MAEXPAVQDragMoveEvent@@@Z 100050d2 f   qt-mt323:qt-mt323.dll
 0001:000040d8       ?contentsDropEvent@QTable@@MAEXPAVQDropEvent@@@Z 100050d8 f   qt-mt323:qt-mt323.dll
 0001:000040de       ?contentsMouseDoubleClickEvent@QTable@@MAEXPAVQMouseEvent@@@Z 100050de f   qt-mt323:qt-mt323.dll
 0001:000040e4       ?contentsMouseMoveEvent@QTable@@MAEXPAVQMouseEvent@@@Z 100050e4 f   qt-mt323:qt-mt323.dll
 0001:000040ea       ?contentsMousePressEvent@QTable@@MAEXPAVQMouseEvent@@@Z 100050ea f   qt-mt323:qt-mt323.dll
 0001:000040f0       ?contentsMouseReleaseEvent@QTable@@MAEXPAVQMouseEvent@@@Z 100050f0 f   qt-mt323:qt-mt323.dll
 0001:000040f6       ?contentsWheelEvent@QScrollView@@MAEXPAVQWheelEvent@@@Z 100050f6 f   qt-mt323:qt-mt323.dll
 0001:000040fc       ?contextMenuEvent@QScrollView@@MAEXPAVQContextMenuEvent@@@Z 100050fc f   qt-mt323:qt-mt323.dll
 0001:00004102       ?create@QWidget@@MAEXPAUHWND__@@_N1@Z 10005102 f   qt-mt323:qt-mt323.dll
 0001:00004108       ?createEditor@QTable@@MBEPAVQWidget@@HH_N@Z 10005108 f   qt-mt323:qt-mt323.dll
 0001:0000410e       ?currentSelection@QTable@@UBEHXZ 1000510e f   qt-mt323:qt-mt323.dll
 0001:00004114       ?customEvent@QObject@@MAEXPAVQCustomEvent@@@Z 10005114 f   qt-mt323:qt-mt323.dll
 0001:0000411a       ?customWhatsThis@QWidget@@UBE_NXZ 1000511a f   qt-mt323:qt-mt323.dll
 0001:00004120       ?destroy@QWidget@@MAEX_N0@Z 10005120 f   qt-mt323:qt-mt323.dll
 0001:00004126       ?disconnectNotify@QObject@@MAEXPBD@Z 10005126 f   qt-mt323:qt-mt323.dll
 0001:0000412c       ?dragEnterEvent@QWidget@@MAEXPAVQDragEnterEvent@@@Z 1000512c f   qt-mt323:qt-mt323.dll
 0001:00004132       ?dragLeaveEvent@QWidget@@MAEXPAVQDragLeaveEvent@@@Z 10005132 f   qt-mt323:qt-mt323.dll
 0001:00004138       ?dragMoveEvent@QWidget@@MAEXPAVQDragMoveEvent@@@Z 10005138 f   qt-mt323:qt-mt323.dll
 0001:0000413e       ?dragObject@QTable@@MAEPAVQDragObject@@XZ 1000513e f   qt-mt323:qt-mt323.dll
 0001:00004144       ?drawContents@QTable@@EAEXPAVQPainter@@@Z 10005144 f   qt-mt323:qt-mt323.dll
 0001:0000414a       ?drawContents@QTable@@MAEXPAVQPainter@@HHHH@Z 1000514a f   qt-mt323:qt-mt323.dll
 0001:00004150       ?drawContentsOffset@QScrollView@@MAEXPAVQPainter@@HHHHHH@Z 10005150 f   qt-mt323:qt-mt323.dll
 0001:00004156       ?drawFrame@QFrame@@MAEXPAVQPainter@@@Z 10005156 f   qt-mt323:qt-mt323.dll
 0001:0000415c       ?dropEvent@QWidget@@MAEXPAVQDropEvent@@@Z 1000515c f   qt-mt323:qt-mt323.dll
 0001:00004162       ?editCell@QTable@@UAEXHH_N@Z 10005162 f   qt-mt323:qt-mt323.dll
 0001:00004168       ?enabledChange@QWidget@@MAEX_N@Z 10005168 f   qt-mt323:qt-mt323.dll
 0001:0000416e       ?endEdit@QTable@@MAEXHH_N0@Z 1000516e f   qt-mt323:qt-mt323.dll
 0001:00004174       ?enterEvent@QWidget@@MAEXPAVQEvent@@@Z 10005174 f   qt-mt323:qt-mt323.dll
 0001:0000417a       ?event@QWidget@@MAE_NPAVQEvent@@@Z 1000517a f   qt-mt323:qt-mt323.dll
 0001:00004180       ?eventFilter@QTable@@UAE_NPAVQObject@@PAVQEvent@@@Z 10005180 f   qt-mt323:qt-mt323.dll
 0001:00004186       ?focusInEvent@QTable@@MAEXPAVQFocusEvent@@@Z 10005186 f   qt-mt323:qt-mt323.dll
 0001:0000418c       ?focusNextPrevChild@QScrollView@@MAE_N_N@Z 1000518c f   qt-mt323:qt-mt323.dll
 0001:00004192       ?focusOutEvent@QTable@@MAEXPAVQFocusEvent@@@Z 10005192 f   qt-mt323:qt-mt323.dll
 0001:00004198       ?fontChange@QScrollView@@MAEXABVQFont@@@Z 10005198 f   qt-mt323:qt-mt323.dll
 0001:0000419e       ?fontInf@QPaintDevice@@MBEHPAVQFont@@H@Z 1000519e f   qt-mt323:qt-mt323.dll
 0001:000041a4       ?fontMet@QPaintDevice@@MBEHPAVQFont@@HPBDH@Z 100051a4 f   qt-mt323:qt-mt323.dll
 0001:000041aa       ?frameChanged@QScrollView@@MAEXXZ 100051aa f   qt-mt323:qt-mt323.dll
 0001:000041b0       ?handle@QPaintDevice@@UBEPAUHDC__@@XZ 100051b0 f   qt-mt323:qt-mt323.dll
 0001:000041b6       ?heightForWidth@QWidget@@UBEHH@Z 100051b6 f   qt-mt323:qt-mt323.dll
 0001:000041bc       ?hide@QWidget@@UAEXXZ      100051bc f   qt-mt323:qt-mt323.dll
 0001:000041c2       ?hideColumn@QTable@@UAEXH@Z 100051c2 f   qt-mt323:qt-mt323.dll
 0001:000041c8       ?hideEvent@QWidget@@MAEXPAVQHideEvent@@@Z 100051c8 f   qt-mt323:qt-mt323.dll
 0001:000041ce       ?hideRow@QTable@@UAEXH@Z   100051ce f   qt-mt323:qt-mt323.dll
 0001:000041d4       ?imComposeEvent@QWidget@@MAEXPAVQIMEvent@@@Z 100051d4 f   qt-mt323:qt-mt323.dll
 0001:000041da       ?imEndEvent@QWidget@@MAEXPAVQIMEvent@@@Z 100051da f   qt-mt323:qt-mt323.dll
 0001:000041e0       ?imStartEvent@QWidget@@MAEXPAVQIMEvent@@@Z 100051e0 f   qt-mt323:qt-mt323.dll
 0001:000041e6       ?insertChild@QObject@@UAEXPAV1@@Z 100051e6 f   qt-mt323:qt-mt323.dll
 0001:000041ec       ?insertColumns@QTable@@UAEXHH@Z 100051ec f   qt-mt323:qt-mt323.dll
 0001:000041f2       ?insertRows@QTable@@UAEXHH@Z 100051f2 f   qt-mt323:qt-mt323.dll
 0001:000041f8       ?insertWidget@QTable@@MAEXHHPAVQWidget@@@Z 100051f8 f   qt-mt323:qt-mt323.dll
 0001:000041fe       ?item@QTable@@UBEPAVQTableItem@@HH@Z 100051fe f   qt-mt323:qt-mt323.dll
 0001:00004204       ?keyReleaseEvent@QWidget@@MAEXPAVQKeyEvent@@@Z 10005204 f   qt-mt323:qt-mt323.dll
 0001:0000420a       ?leaveEvent@QWidget@@MAEXPAVQEvent@@@Z 1000520a f   qt-mt323:qt-mt323.dll
 0001:00004210       ?metric@QWidget@@MBEHH@Z   10005210 f   qt-mt323:qt-mt323.dll
 0001:00004216       ?minimumSizeHint@QScrollView@@UBE?AVQSize@@XZ 10005216 f   qt-mt323:qt-mt323.dll
 0001:0000421c       ?mouseDoubleClickEvent@QScrollView@@MAEXPAVQMouseEvent@@@Z 1000521c f   qt-mt323:qt-mt323.dll
 0001:00004222       ?mouseMoveEvent@QScrollView@@MAEXPAVQMouseEvent@@@Z 10005222 f   qt-mt323:qt-mt323.dll
 0001:00004228       ?mousePressEvent@QScrollView@@MAEXPAVQMouseEvent@@@Z 10005228 f   qt-mt323:qt-mt323.dll
 0001:0000422e       ?mouseReleaseEvent@QScrollView@@MAEXPAVQMouseEvent@@@Z 1000522e f   qt-mt323:qt-mt323.dll
 0001:00004234       ?move@QWidget@@UAEXHH@Z    10005234 f   qt-mt323:qt-mt323.dll
 0001:0000423a       ?moveChild@QScrollView@@UAEXPAVQWidget@@HH@Z 1000523a f   qt-mt323:qt-mt323.dll
 0001:00004240       ?moveEvent@QWidget@@MAEXPAVQMoveEvent@@@Z 10005240 f   qt-mt323:qt-mt323.dll
 0001:00004246       ?numCols@QTable@@UBEHXZ    10005246 f   qt-mt323:qt-mt323.dll
 0001:0000424c       ?numRows@QTable@@UBEHXZ    1000524c f   qt-mt323:qt-mt323.dll
 0001:00004252       ?paintCell@QTable@@UAEXPAVQPainter@@HHABVQRect@@_N@Z 10005252 f   qt-mt323:qt-mt323.dll
 0001:00004258       ?paintCell@QTable@@UAEXPAVQPainter@@HHABVQRect@@_NABVQColorGroup@@@Z 10005258 f   qt-mt323:qt-mt323.dll
 0001:0000425e       ?paintEmptyArea@QTable@@MAEXPAVQPainter@@HHHH@Z 1000525e f   qt-mt323:qt-mt323.dll
 0001:00004264       ?paintEvent@QTable@@MAEXPAVQPaintEvent@@@Z 10005264 f   qt-mt323:qt-mt323.dll
 0001:0000426a       ?paintFocus@QTable@@UAEXPAVQPainter@@ABVQRect@@@Z 1000526a f   qt-mt323:qt-mt323.dll
 0001:00004270       ?paletteChange@QWidget@@MAEXABVQPalette@@@Z 10005270 f   qt-mt323:qt-mt323.dll
 0001:00004276       ?pixmap@QTable@@UBE?AVQPixmap@@HH@Z 10005276 f   qt-mt323:qt-mt323.dll
 0001:0000427c       ?polish@QWidget@@UAEXXZ    1000527c f   qt-mt323:qt-mt323.dll
 0001:00004282       ?property@QObject@@UBE?AVQVariant@@PBD@Z 10005282 f   qt-mt323:qt-mt323.dll
 0001:00004288       ?removeChild@QScrollView@@UAEXPAVQObject@@@Z 10005288 f   qt-mt323:qt-mt323.dll
 0001:0000428e       ?removeColumn@QTable@@UAEXH@Z 1000528e f   qt-mt323:qt-mt323.dll
 0001:00004294       ?removeColumns@QTable@@UAEXABV?$QMemArray@H@@@Z 10005294 f   qt-mt323:qt-mt323.dll
 0001:0000429a       ?removeRow@QTable@@UAEXH@Z 1000529a f   qt-mt323:qt-mt323.dll
 0001:000042a0       ?removeRows@QTable@@UAEXABV?$QMemArray@H@@@Z 100052a0 f   qt-mt323:qt-mt323.dll
 0001:000042a6       ?removeSelection@QTable@@UAEXABVQTableSelection@@@Z 100052a6 f   qt-mt323:qt-mt323.dll
 0001:000042ac       ?removeSelection@QTable@@UAEXH@Z 100052ac f   qt-mt323:qt-mt323.dll
 0001:000042b2       ?reparent@QWidget@@UAEXPAV1@IABVQPoint@@_N@Z 100052b2 f   qt-mt323:qt-mt323.dll
 0001:000042b8       ?resize@QScrollView@@UAEXHH@Z 100052b8 f   qt-mt323:qt-mt323.dll
 0001:000042be       ?resizeContents@QScrollView@@UAEXHH@Z 100052be f   qt-mt323:qt-mt323.dll
 0001:000042c4       ?resizeData@QTable@@MAEXH@Z 100052c4 f   qt-mt323:qt-mt323.dll
 0001:000042ca       ?resizeEvent@QScrollView@@MAEXPAVQResizeEvent@@@Z 100052ca f   qt-mt323:qt-mt323.dll
 0001:000042d0       ?resolution@QPaintDevice@@UBEHXZ 100052d0 f   qt-mt323:qt-mt323.dll
 0001:000042d6       ?rowAt@QTable@@UBEHH@Z     100052d6 f   qt-mt323:qt-mt323.dll
 0001:000042dc       ?rowHeight@QTable@@UBEHH@Z 100052dc f   qt-mt323:qt-mt323.dll
 0001:000042e2       ?rowHeightChanged@QTable@@MAEXH@Z 100052e2 f   qt-mt323:qt-mt323.dll
 0001:000042e8       ?rowIndexChanged@QTable@@MAEXHHH@Z 100052e8 f   qt-mt323:qt-mt323.dll
 0001:000042ee       ?rowPos@QTable@@UBEHH@Z    100052ee f   qt-mt323:qt-mt323.dll
 0001:000042f4       ?setAcceptDrops@QWidget@@UAEX_N@Z 100052f4 f   qt-mt323:qt-mt323.dll
 0001:000042fa       ?setActiveWindow@QWidget@@UAEXXZ 100052fa f   qt-mt323:qt-mt323.dll
 0001:00004300       ?setAutoMask@QWidget@@UAEX_N@Z 10005300 f   qt-mt323:qt-mt323.dll
 0001:00004306       ?setBackgroundColor@QWidget@@UAEXABVQColor@@@Z 10005306 f   qt-mt323:qt-mt323.dll
 0001:0000430c       ?setBackgroundMode@QWidget@@UAEXW4BackgroundMode@Qt@@@Z 1000530c f   qt-mt323:qt-mt323.dll
 0001:00004312       ?setBackgroundOrigin@QWidget@@UAEXW4BackgroundOrigin@1@@Z 10005312 f   qt-mt323:qt-mt323.dll
 0001:00004318       ?setBackgroundPixmap@QWidget@@UAEXABVQPixmap@@@Z 10005318 f   qt-mt323:qt-mt323.dll
 0001:0000431e       ?setCaption@QWidget@@UAEXABVQString@@@Z 1000531e f   qt-mt323:qt-mt323.dll
 0001:00004324       ?setCellContentFromEditor@QTable@@MAEXHH@Z 10005324 f   qt-mt323:qt-mt323.dll
 0001:0000432a       ?setCellWidget@QTable@@UAEXHHPAVQWidget@@@Z 1000532a f   qt-mt323:qt-mt323.dll
 0001:00004330       ?setColumnMovingEnabled@QTable@@UAEX_N@Z 10005330 f   qt-mt323:qt-mt323.dll
 0001:00004336       ?setColumnReadOnly@QTable@@UAEXH_N@Z 10005336 f   qt-mt323:qt-mt323.dll
 0001:0000433c       ?setColumnStretchable@QTable@@UAEXH_N@Z 1000533c f   qt-mt323:qt-mt323.dll
 0001:00004342       ?setColumnWidth@QTable@@UAEXHH@Z 10005342 f   qt-mt323:qt-mt323.dll
 0001:00004348       ?setContentsPos@QScrollView@@UAEXHH@Z 10005348 f   qt-mt323:qt-mt323.dll
 0001:0000434e       ?setCornerWidget@QScrollView@@UAEXPAVQWidget@@@Z 1000534e f   qt-mt323:qt-mt323.dll
 0001:00004354       ?setCurrentCell@QTable@@UAEXHH@Z 10005354 f   qt-mt323:qt-mt323.dll
 0001:0000435a       ?setCursor@QWidget@@UAEXABVQCursor@@@Z 1000535a f   qt-mt323:qt-mt323.dll
 0001:00004360       ?setDragAutoScroll@QScrollView@@UAEX_N@Z 10005360 f   qt-mt323:qt-mt323.dll
 0001:00004366       ?setDragEnabled@QTable@@UAEX_N@Z 10005366 f   qt-mt323:qt-mt323.dll
 0001:0000436c       ?setEnabled@QTable@@UAEX_N@Z 1000536c f   qt-mt323:qt-mt323.dll
 0001:00004372       ?setEraseColor@QWidget@@UAEXABVQColor@@@Z 10005372 f   qt-mt323:qt-mt323.dll
 0001:00004378       ?setErasePixmap@QWidget@@UAEXABVQPixmap@@@Z 10005378 f   qt-mt323:qt-mt323.dll
 0001:0000437e       ?setFocus@QWidget@@UAEXXZ  1000537e f   qt-mt323:qt-mt323.dll
 0001:00004384       ?setFocusPolicy@QWidget@@UAEXW4FocusPolicy@1@@Z 10005384 f   qt-mt323:qt-mt323.dll
 0001:0000438a       ?setFocusProxy@QWidget@@UAEXPAV1@@Z 1000538a f   qt-mt323:qt-mt323.dll
 0001:00004390       ?setFocusStyle@QTable@@UAEXW4FocusStyle@1@@Z 10005390 f   qt-mt323:qt-mt323.dll
 0001:00004396       ?setFont@QWidget@@UAEXABVQFont@@@Z 10005396 f   qt-mt323:qt-mt323.dll
 0001:0000439c       ?setFrameRect@QFrame@@UAEXABVQRect@@@Z 1000539c f   qt-mt323:qt-mt323.dll
 0001:000043a2       ?setFrameStyle@QFrame@@UAEXH@Z 100053a2 f   qt-mt323:qt-mt323.dll
 0001:000043a8       ?setGeometry@QWidget@@UAEXABVQRect@@@Z 100053a8 f   qt-mt323:qt-mt323.dll
 0001:000043ae       ?setGeometry@QWidget@@UAEXHHHH@Z 100053ae f   qt-mt323:qt-mt323.dll
 0001:000043b4       ?setHBarGeometry@QScrollView@@MAEXAAVQScrollBar@@HHHH@Z 100053b4 f   qt-mt323:qt-mt323.dll
 0001:000043ba       ?setHScrollBarMode@QScrollView@@UAEXW4ScrollBarMode@1@@Z 100053ba f   qt-mt323:qt-mt323.dll
 0001:000043c0       ?setIcon@QWidget@@UAEXABVQPixmap@@@Z 100053c0 f   qt-mt323:qt-mt323.dll
 0001:000043c6       ?setIconText@QWidget@@UAEXABVQString@@@Z 100053c6 f   qt-mt323:qt-mt323.dll
 0001:000043cc       ?setItem@QTable@@UAEXHHPAVQTableItem@@@Z 100053cc f   qt-mt323:qt-mt323.dll
 0001:000043d2       ?setKeyCompression@QWidget@@MAEX_N@Z 100053d2 f   qt-mt323:qt-mt323.dll
 0001:000043d8       ?setLeftMargin@QTable@@UAEXH@Z 100053d8 f   qt-mt323:qt-mt323.dll
 0001:000043de       ?setLineWidth@QFrame@@UAEXH@Z 100053de f   qt-mt323:qt-mt323.dll
 0001:000043e4       ?setMargin@QFrame@@UAEXH@Z 100053e4 f   qt-mt323:qt-mt323.dll
 0001:000043ea       ?setMargins@QScrollView@@MAEXHHHH@Z 100053ea f   qt-mt323:qt-mt323.dll
 0001:000043f0       ?setMask@QWidget@@UAEXABVQBitmap@@@Z 100053f0 f   qt-mt323:qt-mt323.dll
 0001:000043f6       ?setMask@QWidget@@UAEXABVQRegion@@@Z 100053f6 f   qt-mt323:qt-mt323.dll
 0001:000043fc       ?setMaximumSize@QWidget@@UAEXHH@Z 100053fc f   qt-mt323:qt-mt323.dll
 0001:00004402       ?setMicroFocusHint@QWidget@@MAEXHHHH_NPAVQFont@@@Z 10005402 f   qt-mt323:qt-mt323.dll
 0001:00004408       ?setMidLineWidth@QFrame@@UAEXH@Z 10005408 f   qt-mt323:qt-mt323.dll
 0001:0000440e       ?setMinimumSize@QWidget@@UAEXHH@Z 1000540e f   qt-mt323:qt-mt323.dll
 0001:00004414       ?setMouseTracking@QWidget@@UAEX_N@Z 10005414 f   qt-mt323:qt-mt323.dll
 0001:0000441a       ?setName@QWidget@@UAEXPBD@Z 1000541a f   qt-mt323:qt-mt323.dll
 0001:00004420       ?setNumCols@QTable@@UAEXH@Z 10005420 f   qt-mt323:qt-mt323.dll
 0001:00004426       ?setNumRows@QTable@@UAEXH@Z 10005426 f   qt-mt323:qt-mt323.dll
 0001:0000442c       ?setPalette@QWidget@@UAEXABVQPalette@@@Z 1000542c f   qt-mt323:qt-mt323.dll
 0001:00004432       ?setPaletteBackgroundColor@QWidget@@UAEXABVQColor@@@Z 10005432 f   qt-mt323:qt-mt323.dll
 0001:00004438       ?setPaletteBackgroundPixmap@QWidget@@UAEXABVQPixmap@@@Z 10005438 f   qt-mt323:qt-mt323.dll
 0001:0000443e       ?setPixmap@QTable@@UAEXHHABVQPixmap@@@Z 1000543e f   qt-mt323:qt-mt323.dll
 0001:00004444       ?setProperty@QObject@@UAE_NPBDABVQVariant@@@Z 10005444 f   qt-mt323:qt-mt323.dll
 0001:0000444a       ?setReadOnly@QTable@@UAEX_N@Z 1000544a f   qt-mt323:qt-mt323.dll
 0001:00004450       ?setResizePolicy@QScrollView@@UAEXW4ResizePolicy@1@@Z 10005450 f   qt-mt323:qt-mt323.dll
 0001:00004456       ?setResolution@QPaintDevice@@UAEXH@Z 10005456 f   qt-mt323:qt-mt323.dll
 0001:0000445c       ?setRowHeight@QTable@@UAEXHH@Z 1000545c f   qt-mt323:qt-mt323.dll
 0001:00004462       ?setRowMovingEnabled@QTable@@UAEX_N@Z 10005462 f   qt-mt323:qt-mt323.dll
 0001:00004468       ?setRowReadOnly@QTable@@UAEXH_N@Z 10005468 f   qt-mt323:qt-mt323.dll
 0001:0000446e       ?setRowStretchable@QTable@@UAEXH_N@Z 1000546e f   qt-mt323:qt-mt323.dll
 0001:00004474       ?setSelectionMode@QTable@@UAEXW4SelectionMode@1@@Z 10005474 f   qt-mt323:qt-mt323.dll
 0001:0000447a       ?setShowGrid@QTable@@UAEX_N@Z 1000547a f   qt-mt323:qt-mt323.dll
 0001:00004480       ?setSizeIncrement@QWidget@@UAEXHH@Z 10005480 f   qt-mt323:qt-mt323.dll
 0001:00004486       ?setSizePolicy@QWidget@@UAEXVQSizePolicy@@@Z 10005486 f   qt-mt323:qt-mt323.dll
 0001:0000448c       ?setSorting@QTable@@UAEX_N@Z 1000548c f   qt-mt323:qt-mt323.dll
 0001:00004492       ?setText@QTable@@UAEXHHABVQString@@@Z 10005492 f   qt-mt323:qt-mt323.dll
 0001:00004498       ?setTopMargin@QTable@@UAEXH@Z 10005498 f   qt-mt323:qt-mt323.dll
 0001:0000449e       ?setUpdatesEnabled@QWidget@@UAEX_N@Z 1000549e f   qt-mt323:qt-mt323.dll
 0001:000044a4       ?setVBarGeometry@QScrollView@@MAEXAAVQScrollBar@@HHHH@Z 100054a4 f   qt-mt323:qt-mt323.dll
 0001:000044aa       ?setVScrollBarMode@QScrollView@@UAEXW4ScrollBarMode@1@@Z 100054aa f   qt-mt323:qt-mt323.dll
 0001:000044b0       ?setWFlags@QWidget@@MAEXI@Z 100054b0 f   qt-mt323:qt-mt323.dll
 0001:000044b6       ?setWState@QWidget@@MAEXI@Z 100054b6 f   qt-mt323:qt-mt323.dll
 0001:000044bc       ?show@QScrollView@@UAEXXZ  100054bc f   qt-mt323:qt-mt323.dll
 0001:000044c2       ?showColumn@QTable@@UAEXH@Z 100054c2 f   qt-mt323:qt-mt323.dll
 0001:000044c8       ?showEvent@QTable@@MAEXPAVQShowEvent@@@Z 100054c8 f   qt-mt323:qt-mt323.dll
 0001:000044ce       ?showMaximized@QWidget@@UAEXXZ 100054ce f   qt-mt323:qt-mt323.dll
 0001:000044d4       ?showMinimized@QWidget@@UAEXXZ 100054d4 f   qt-mt323:qt-mt323.dll
 0001:000044da       ?showNormal@QWidget@@UAEXXZ 100054da f   qt-mt323:qt-mt323.dll
 0001:000044e0       ?showRow@QTable@@UAEXH@Z   100054e0 f   qt-mt323:qt-mt323.dll
 0001:000044e6       ?sizeHint@QTable@@UBE?AVQSize@@XZ 100054e6 f   qt-mt323:qt-mt323.dll
 0001:000044ec       ?sizePolicy@QWidget@@UBE?AVQSizePolicy@@XZ 100054ec f   qt-mt323:qt-mt323.dll
 0001:000044f2       ?sortColumn@QTable@@UAEXH_N0@Z 100054f2 f   qt-mt323:qt-mt323.dll
 0001:000044f8       ?startDrag@QTable@@MAEXXZ  100054f8 f   qt-mt323:qt-mt323.dll
 0001:000044fe       ?styleChange@QScrollView@@UAEXAAVQStyle@@@Z 100054fe f   qt-mt323:qt-mt323.dll
 0001:00004504       ?swapCells@QTable@@UAEXHHHH@Z 10005504 f   qt-mt323:qt-mt323.dll
 0001:0000450a       ?swapColumns@QTable@@UAEXHH_N@Z 1000550a f   qt-mt323:qt-mt323.dll
 0001:00004510       ?swapRows@QTable@@UAEXHH_N@Z 10005510 f   qt-mt323:qt-mt323.dll
 0001:00004516       ?tabletEvent@QWidget@@MAEXPAVQTabletEvent@@@Z 10005516 f   qt-mt323:qt-mt323.dll
 0001:0000451c       ?takeItem@QTable@@UAEXPAVQTableItem@@@Z 1000551c f   qt-mt323:qt-mt323.dll
 0001:00004522       ?text@QTable@@UBE?AVQString@@HH@Z 10005522 f   qt-mt323:qt-mt323.dll
 0001:00004528       ?timerEvent@QObject@@MAEXPAVQTimerEvent@@@Z 10005528 f   qt-mt323:qt-mt323.dll
 0001:0000452e       ?unsetCursor@QWidget@@UAEXXZ 1000552e f   qt-mt323:qt-mt323.dll
 0001:00004534       ?updateMask@QWidget@@MAEXXZ 10005534 f   qt-mt323:qt-mt323.dll
 0001:0000453a       ?viewportContextMenuEvent@QScrollView@@MAEXPAVQContextMenuEvent@@@Z 1000553a f   qt-mt323:qt-mt323.dll
 0001:00004540       ?viewportDragEnterEvent@QScrollView@@MAEXPAVQDragEnterEvent@@@Z 10005540 f   qt-mt323:qt-mt323.dll
 0001:00004546       ?viewportDragLeaveEvent@QScrollView@@MAEXPAVQDragLeaveEvent@@@Z 10005546 f   qt-mt323:qt-mt323.dll
 0001:0000454c       ?viewportDragMoveEvent@QScrollView@@MAEXPAVQDragMoveEvent@@@Z 1000554c f   qt-mt323:qt-mt323.dll
 0001:00004552       ?viewportDropEvent@QScrollView@@MAEXPAVQDropEvent@@@Z 10005552 f   qt-mt323:qt-mt323.dll
 0001:00004558       ?viewportMouseDoubleClickEvent@QScrollView@@MAEXPAVQMouseEvent@@@Z 10005558 f   qt-mt323:qt-mt323.dll
 0001:0000455e       ?viewportMouseMoveEvent@QScrollView@@MAEXPAVQMouseEvent@@@Z 1000555e f   qt-mt323:qt-mt323.dll
 0001:00004564       ?viewportMousePressEvent@QScrollView@@MAEXPAVQMouseEvent@@@Z 10005564 f   qt-mt323:qt-mt323.dll
 0001:0000456a       ?viewportMouseReleaseEvent@QScrollView@@MAEXPAVQMouseEvent@@@Z 1000556a f   qt-mt323:qt-mt323.dll
 0001:00004570       ?viewportPaintEvent@QScrollView@@MAEXPAVQPaintEvent@@@Z 10005570 f   qt-mt323:qt-mt323.dll
 0001:00004576       ?viewportResizeEvent@QTable@@MAEXPAVQResizeEvent@@@Z 10005576 f   qt-mt323:qt-mt323.dll
 0001:0000457c       ?viewportWheelEvent@QScrollView@@MAEXPAVQWheelEvent@@@Z 1000557c f   qt-mt323:qt-mt323.dll
 0001:00004582       ?wheelEvent@QScrollView@@MAEXPAVQWheelEvent@@@Z 10005582 f   qt-mt323:qt-mt323.dll
 0001:00004588       ?winEvent@QWidget@@MAE_NPAUtagMSG@@@Z 10005588 f   qt-mt323:qt-mt323.dll
 0001:0000458e       ?windowActivationChange@QTable@@MAEX_N@Z 1000558e f   qt-mt323:qt-mt323.dll
 0001:00004594       ?alignment@QTableItem@@UBEHXZ 10005594 f   qt-mt323:qt-mt323.dll
 0001:0000459a       ?className@QComboBox@@UBEPBDXZ 1000559a f   qt-mt323:qt-mt323.dll
 0001:000045a0       ?contextMenuEvent@QWidget@@MAEXPAVQContextMenuEvent@@@Z 100055a0 f   qt-mt323:qt-mt323.dll
 0001:000045a6       ?eventFilter@QComboBox@@UAE_NPAVQObject@@PAVQEvent@@@Z 100055a6 f   qt-mt323:qt-mt323.dll
 0001:000045ac       ?focusInEvent@QComboBox@@MAEXPAVQFocusEvent@@@Z 100055ac f   qt-mt323:qt-mt323.dll
 0001:000045b2       ?focusNextPrevChild@QWidget@@MAE_N_N@Z 100055b2 f   qt-mt323:qt-mt323.dll
 0001:000045b8       ?focusOutEvent@QComboBox@@MAEXPAVQFocusEvent@@@Z 100055b8 f   qt-mt323:qt-mt323.dll
 0001:000045be       ?fontChange@QWidget@@MAEXABVQFont@@@Z 100055be f   qt-mt323:qt-mt323.dll
 0001:000045c4       ?key@QTableItem@@UBE?AVQString@@XZ 100055c4 f   qt-mt323:qt-mt323.dll
 0001:000045ca       ?keyPressEvent@QComboBox@@MAEXPAVQKeyEvent@@@Z 100055ca f   qt-mt323:qt-mt323.dll
 0001:000045d0       ?metaObject@QComboBox@@UBEPAVQMetaObject@@XZ 100055d0 f   qt-mt323:qt-mt323.dll
 0001:000045d6       ?minimumSizeHint@QWidget@@UBE?AVQSize@@XZ 100055d6 f   qt-mt323:qt-mt323.dll
 0001:000045dc       ?mouseDoubleClickEvent@QComboBox@@MAEXPAVQMouseEvent@@@Z 100055dc f   qt-mt323:qt-mt323.dll
 0001:000045e2       ?mouseMoveEvent@QComboBox@@MAEXPAVQMouseEvent@@@Z 100055e2 f   qt-mt323:qt-mt323.dll
 0001:000045e8       ?mousePressEvent@QComboBox@@MAEXPAVQMouseEvent@@@Z 100055e8 f   qt-mt323:qt-mt323.dll
 0001:000045ee       ?mouseReleaseEvent@QComboBox@@MAEXPAVQMouseEvent@@@Z 100055ee f   qt-mt323:qt-mt323.dll
 0001:000045f4       ?paint@QTableItem@@UAEXPAVQPainter@@ABVQColorGroup@@ABVQRect@@_N@Z 100055f4 f   qt-mt323:qt-mt323.dll
 0001:000045fa       ?paintEvent@QComboBox@@MAEXPAVQPaintEvent@@@Z 100055fa f   qt-mt323:qt-mt323.dll
 0001:00004600       ?pixmap@QTableItem@@UBE?AVQPixmap@@XZ 10005600 f   qt-mt323:qt-mt323.dll
 0001:00004606       ?popup@QComboBox@@UAEXXZ   10005606 f   qt-mt323:qt-mt323.dll
 0001:0000460c       ?qt_cast@QComboBox@@UAEPAXPBD@Z 1000560c f   qt-mt323:qt-mt323.dll
 0001:00004612       ?qt_emit@QComboBox@@UAE_NHPAUQUObject@@@Z 10005612 f   qt-mt323:qt-mt323.dll
 0001:00004618       ?qt_invoke@QComboBox@@UAE_NHPAUQUObject@@@Z 10005618 f   qt-mt323:qt-mt323.dll
 0001:0000461e       ?qt_property@QComboBox@@UAE_NHHPAVQVariant@@@Z 1000561e f   qt-mt323:qt-mt323.dll
 0001:00004624       ?removeChild@QObject@@UAEXPAV1@@Z 10005624 f   qt-mt323:qt-mt323.dll
 0001:0000462a       ?resize@QWidget@@UAEXHH@Z  1000562a f   qt-mt323:qt-mt323.dll
 0001:00004630       ?resizeEvent@QComboBox@@MAEXPAVQResizeEvent@@@Z 10005630 f   qt-mt323:qt-mt323.dll
 0001:00004636       ?rtti@QTableItem@@UBEHXZ   10005636 f   qt-mt323:qt-mt323.dll
 0001:0000463c       ?setAutoCompletion@QComboBox@@UAEX_N@Z 1000563c f   qt-mt323:qt-mt323.dll
 0001:00004642       ?setAutoResize@QComboBox@@UAEX_N@Z 10005642 f   qt-mt323:qt-mt323.dll
 0001:00004648       ?setCol@QTableItem@@UAEXH@Z 10005648 f   qt-mt323:qt-mt323.dll
 0001:0000464e       ?setCurrentItem@QComboBox@@UAEXH@Z 1000564e f   qt-mt323:qt-mt323.dll
 0001:00004654       ?setCurrentText@QComboBox@@UAEXABVQString@@@Z 10005654 f   qt-mt323:qt-mt323.dll
 0001:0000465a       ?setEditText@QComboBox@@UAEXABVQString@@@Z 1000565a f   qt-mt323:qt-mt323.dll
 0001:00004660       ?setEnabled@QComboBox@@UAEX_N@Z 10005660 f   qt-mt323:qt-mt323.dll
 0001:00004666       ?setEnabled@QTableItem@@UAEX_N@Z 10005666 f   qt-mt323:qt-mt323.dll
 0001:0000466c       ?setFont@QComboBox@@UAEXABVQFont@@@Z 1000566c f   qt-mt323:qt-mt323.dll
 0001:00004672       ?setInsertionPolicy@QComboBox@@UAEXW4Policy@1@@Z 10005672 f   qt-mt323:qt-mt323.dll
 0001:00004678       ?setLineEdit@QComboBox@@UAEXPAVQLineEdit@@@Z 10005678 f   qt-mt323:qt-mt323.dll
 0001:0000467e       ?setListBox@QComboBox@@UAEXPAVQListBox@@@Z 1000567e f   qt-mt323:qt-mt323.dll
 0001:00004684       ?setMaxCount@QComboBox@@UAEXH@Z 10005684 f   qt-mt323:qt-mt323.dll
 0001:0000468a       ?setPalette@QComboBox@@UAEXABVQPalette@@@Z 1000568a f   qt-mt323:qt-mt323.dll
 0001:00004690       ?setPixmap@QTableItem@@UAEXABVQPixmap@@@Z 10005690 f   qt-mt323:qt-mt323.dll
 0001:00004696       ?setReplaceable@QTableItem@@UAEX_N@Z 10005696 f   qt-mt323:qt-mt323.dll
 0001:0000469c       ?setRow@QTableItem@@UAEXH@Z 1000569c f   qt-mt323:qt-mt323.dll
 0001:000046a2       ?setSizeLimit@QComboBox@@UAEXH@Z 100056a2 f   qt-mt323:qt-mt323.dll
 0001:000046a8       ?setSpan@QTableItem@@UAEXHH@Z 100056a8 f   qt-mt323:qt-mt323.dll
 0001:000046ae       ?setText@QTableItem@@UAEXABVQString@@@Z 100056ae f   qt-mt323:qt-mt323.dll
 0001:000046b4       ?setValidator@QComboBox@@UAEXPBVQValidator@@@Z 100056b4 f   qt-mt323:qt-mt323.dll
 0001:000046ba       ?setWordWrap@QTableItem@@UAEX_N@Z 100056ba f   qt-mt323:qt-mt323.dll
 0001:000046c0       ?show@QWidget@@UAEXXZ      100056c0 f   qt-mt323:qt-mt323.dll
 0001:000046c6       ?showEvent@QWidget@@MAEXPAVQShowEvent@@@Z 100056c6 f   qt-mt323:qt-mt323.dll
 0001:000046cc       ?sizeHint@QComboBox@@UBE?AVQSize@@XZ 100056cc f   qt-mt323:qt-mt323.dll
 0001:000046d2       ?sizeHint@QTableItem@@UBE?AVQSize@@XZ 100056d2 f   qt-mt323:qt-mt323.dll
 0001:000046d8       ?styleChange@QComboBox@@MAEXAAVQStyle@@@Z 100056d8 f   qt-mt323:qt-mt323.dll
 0001:000046de       ?text@QTableItem@@UBE?AVQString@@XZ 100056de f   qt-mt323:qt-mt323.dll
 0001:000046e4       ?updateMask@QComboBox@@MAEXXZ 100056e4 f   qt-mt323:qt-mt323.dll
 0001:000046ea       ?wheelEvent@QComboBox@@MAEXPAVQWheelEvent@@@Z 100056ea f   qt-mt323:qt-mt323.dll
 0001:000046f0       ?windowActivationChange@QWidget@@MAEX_N@Z 100056f0 f   qt-mt323:qt-mt323.dll
 0001:000046f6       ?eventFilter@QObject@@UAE_NPAV1@PAVQEvent@@@Z 100056f6 f   qt-mt323:qt-mt323.dll
 0001:000046fc       ?focusInEvent@QWidget@@MAEXPAVQFocusEvent@@@Z 100056fc f   qt-mt323:qt-mt323.dll
 0001:00004702       ?focusOutEvent@QWidget@@MAEXPAVQFocusEvent@@@Z 10005702 f   qt-mt323:qt-mt323.dll
 0001:00004708       ?keyPressEvent@QWidget@@MAEXPAVQKeyEvent@@@Z 10005708 f   qt-mt323:qt-mt323.dll
 0001:0000470e       ?mouseDoubleClickEvent@QWidget@@MAEXPAVQMouseEvent@@@Z 1000570e f   qt-mt323:qt-mt323.dll
 0001:00004714       ?mouseMoveEvent@QWidget@@MAEXPAVQMouseEvent@@@Z 10005714 f   qt-mt323:qt-mt323.dll
 0001:0000471a       ?mousePressEvent@QWidget@@MAEXPAVQMouseEvent@@@Z 1000571a f   qt-mt323:qt-mt323.dll
 0001:00004720       ?mouseReleaseEvent@QWidget@@MAEXPAVQMouseEvent@@@Z 10005720 f   qt-mt323:qt-mt323.dll
 0001:00004726       ?paintEvent@QWidget@@MAEXPAVQPaintEvent@@@Z 10005726 f   qt-mt323:qt-mt323.dll
 0001:0000472c       ?resizeEvent@QWidget@@MAEXPAVQResizeEvent@@@Z 1000572c f   qt-mt323:qt-mt323.dll
 0001:00004732       ?setEnabled@QWidget@@UAEX_N@Z 10005732 f   qt-mt323:qt-mt323.dll
 0001:00004738       ?sizeHint@QWidget@@UBE?AVQSize@@XZ 10005738 f   qt-mt323:qt-mt323.dll
 0001:0000473e       ?styleChange@QWidget@@MAEXAAVQStyle@@@Z 1000573e f   qt-mt323:qt-mt323.dll
 0001:00004744       ?wheelEvent@QWidget@@MAEXPAVQWheelEvent@@@Z 10005744 f   qt-mt323:qt-mt323.dll
 0001:0000474a       ?activateItemAt@QPopupMenu@@UAEXH@Z 1000574a f   qt-mt323:qt-mt323.dll
 0001:00004750       ?addTo@QAction@@UAE_NPAVQWidget@@@Z 10005750 f   qt-mt323:qt-mt323.dll
 0001:00004756       ?addedTo@QAction@@MAEXHPAVQPopupMenu@@@Z 10005756 f   qt-mt323:qt-mt323.dll
 0001:0000475c       ?addedTo@QAction@@MAEXPAVQWidget@@0@Z 1000575c f   qt-mt323:qt-mt323.dll
 0001:00004762       ?className@QAction@@UBEPBDXZ 10005762 f   qt-mt323:qt-mt323.dll
 0001:00004768       ?className@QGuardedPtrPrivate@@UBEPBDXZ 10005768 f   qt-mt323:qt-mt323.dll
 0001:0000476e       ?className@QPopupMenu@@UBEPBDXZ 1000576e f   qt-mt323:qt-mt323.dll
 0001:00004774       ?className@QToolBar@@UBEPBDXZ 10005774 f   qt-mt323:qt-mt323.dll
 0001:0000477a       ?className@QWidget@@UBEPBDXZ 1000577a f   qt-mt323:qt-mt323.dll
 0001:00004780       ?clear@?$QPtrList@VQDockWindow@@@@UAEXXZ 10005780 f   qt-mt323:qt-mt323.dll
 0001:00004786       ?clear@QToolBar@@UAEXXZ    10005786 f   qt-mt323:qt-mt323.dll
 0001:0000478c       ?closeEvent@QPopupMenu@@MAEXPAVQCloseEvent@@@Z 1000578c f   qt-mt323:qt-mt323.dll
 0001:00004792       ?compareItems@QGList@@MAEHPAX0@Z 10005792 f   qt-mt323:qt-mt323.dll
 0001:00004798       ?contextMenuEvent@QDockWindow@@MAEXPAVQContextMenuEvent@@@Z 10005798 f   qt-mt323:qt-mt323.dll
 0001:0000479e       ?count@?$QPtrList@VQDockWindow@@@@UBEIXZ 1000579e f   qt-mt323:qt-mt323.dll
 0001:000047a4       ?customWhatsThis@QPopupMenu@@UBE_NXZ 100057a4 f   qt-mt323:qt-mt323.dll
 0001:000047aa       ?deleteItem@?$QPtrList@VQDockWindow@@@@EAEXPAX@Z 100057aa f   qt-mt323:qt-mt323.dll
 0001:000047b0       ?dock@QDockWindow@@UAEXXZ  100057b0 f   qt-mt323:qt-mt323.dll
 0001:000047b6       ?drawContents@QDockWindow@@MAEXPAVQPainter@@@Z 100057b6 f   qt-mt323:qt-mt323.dll
 0001:000047bc       ?drawContents@QPopupMenu@@MAEXPAVQPainter@@@Z 100057bc f   qt-mt323:qt-mt323.dll
 0001:000047c2       ?drawFrame@QDockWindow@@MAEXPAVQPainter@@@Z 100057c2 f   qt-mt323:qt-mt323.dll
 0001:000047c8       ?enabledChange@QPopupMenu@@MAEX_N@Z 100057c8 f   qt-mt323:qt-mt323.dll
 0001:000047ce       ?event@QObject@@UAE_NPAVQEvent@@@Z 100057ce f   qt-mt323:qt-mt323.dll
 0001:000047d4       ?event@QToolBar@@UAE_NPAVQEvent@@@Z 100057d4 f   qt-mt323:qt-mt323.dll
 0001:000047da       ?eventFilter@QDockWindow@@UAE_NPAVQObject@@PAVQEvent@@@Z 100057da f   qt-mt323:qt-mt323.dll
 0001:000047e0       ?focusInEvent@QPopupMenu@@MAEXPAVQFocusEvent@@@Z 100057e0 f   qt-mt323:qt-mt323.dll
 0001:000047e6       ?focusNextPrevChild@QPopupMenu@@MAE_N_N@Z 100057e6 f   qt-mt323:qt-mt323.dll
 0001:000047ec       ?focusOutEvent@QPopupMenu@@MAEXPAVQFocusEvent@@@Z 100057ec f   qt-mt323:qt-mt323.dll
 0001:000047f2       ?frameChanged@QFrame@@MAEXXZ 100057f2 f   qt-mt323:qt-mt323.dll
 0001:000047f8       ?frameChanged@QPopupMenu@@EAEXXZ 100057f8 f   qt-mt323:qt-mt323.dll
 0001:000047fe       ?hide@QPopupMenu@@UAEXXZ   100057fe f   qt-mt323:qt-mt323.dll
 0001:00004804       ?hide@QToolBar@@UAEXXZ     10005804 f   qt-mt323:qt-mt323.dll
 0001:0000480a       ?hideEvent@QDockWindow@@MAEXPAVQHideEvent@@@Z 1000580a f   qt-mt323:qt-mt323.dll
 0001:00004810       ?keyPressEvent@QPopupMenu@@MAEXPAVQKeyEvent@@@Z 10005810 f   qt-mt323:qt-mt323.dll
 0001:00004816       ?leaveEvent@QPopupMenu@@MAEXPAVQEvent@@@Z 10005816 f   qt-mt323:qt-mt323.dll
 0001:0000481c       ?menuContentsChanged@QPopupMenu@@EAEXXZ 1000581c f   qt-mt323:qt-mt323.dll
 0001:00004822       ?menuDelPopup@QPopupMenu@@EAEXPAV1@@Z 10005822 f   qt-mt323:qt-mt323.dll
 0001:00004828       ?menuInsPopup@QPopupMenu@@EAEXPAV1@@Z 10005828 f   qt-mt323:qt-mt323.dll
 0001:0000482e       ?menuStateChanged@QPopupMenu@@EAEXXZ 1000582e f   qt-mt323:qt-mt323.dll
 0001:00004834       ?metaObject@QAction@@UBEPAVQMetaObject@@XZ 10005834 f   qt-mt323:qt-mt323.dll
 0001:0000483a       ?metaObject@QGuardedPtrPrivate@@UBEPAVQMetaObject@@XZ 1000583a f   qt-mt323:qt-mt323.dll
 0001:00004840       ?metaObject@QPopupMenu@@UBEPAVQMetaObject@@XZ 10005840 f   qt-mt323:qt-mt323.dll
 0001:00004846       ?metaObject@QToolBar@@UBEPAVQMetaObject@@XZ 10005846 f   qt-mt323:qt-mt323.dll
 0001:0000484c       ?metaObject@QWidget@@UBEPAVQMetaObject@@XZ 1000584c f   qt-mt323:qt-mt323.dll
 0001:00004852       ?minimumSizeHint@QToolBar@@UBE?AVQSize@@XZ 10005852 f   qt-mt323:qt-mt323.dll
 0001:00004858       ?mouseMoveEvent@QPopupMenu@@MAEXPAVQMouseEvent@@@Z 10005858 f   qt-mt323:qt-mt323.dll
 0001:0000485e       ?mousePressEvent@QPopupMenu@@MAEXPAVQMouseEvent@@@Z 1000585e f   qt-mt323:qt-mt323.dll
 0001:00004864       ?mouseReleaseEvent@QPopupMenu@@MAEXPAVQMouseEvent@@@Z 10005864 f   qt-mt323:qt-mt323.dll
 0001:0000486a       ?newItem@QPtrCollection@@MAEPAXPAX@Z 1000586a f   qt-mt323:qt-mt323.dll
 0001:00004870       ?paintEvent@QFrame@@MAEXPAVQPaintEvent@@@Z 10005870 f   qt-mt323:qt-mt323.dll
 0001:00004876       ?paintEvent@QPopupMenu@@MAEXPAVQPaintEvent@@@Z 10005876 f   qt-mt323:qt-mt323.dll
 0001:0000487c       ?qt_cast@QAction@@UAEPAXPBD@Z 1000587c f   qt-mt323:qt-mt323.dll
 0001:00004882       ?qt_cast@QGuardedPtrPrivate@@UAEPAXPBD@Z 10005882 f   qt-mt323:qt-mt323.dll
 0001:00004888       ?qt_cast@QPopupMenu@@UAEPAXPBD@Z 10005888 f   qt-mt323:qt-mt323.dll
 0001:0000488e       ?qt_cast@QToolBar@@UAEPAXPBD@Z 1000588e f   qt-mt323:qt-mt323.dll
 0001:00004894       ?qt_cast@QWidget@@UAEPAXPBD@Z 10005894 f   qt-mt323:qt-mt323.dll
 0001:0000489a       ?qt_emit@QAction@@UAE_NHPAUQUObject@@@Z 1000589a f   qt-mt323:qt-mt323.dll
 0001:000048a0       ?qt_emit@QGuardedPtrPrivate@@UAE_NHPAUQUObject@@@Z 100058a0 f   qt-mt323:qt-mt323.dll
 0001:000048a6       ?qt_emit@QPopupMenu@@UAE_NHPAUQUObject@@@Z 100058a6 f   qt-mt323:qt-mt323.dll
 0001:000048ac       ?qt_emit@QToolBar@@UAE_NHPAUQUObject@@@Z 100058ac f   qt-mt323:qt-mt323.dll
 0001:000048b2       ?qt_emit@QWidget@@UAE_NHPAUQUObject@@@Z 100058b2 f   qt-mt323:qt-mt323.dll
 0001:000048b8       ?qt_invoke@QAction@@UAE_NHPAUQUObject@@@Z 100058b8 f   qt-mt323:qt-mt323.dll
 0001:000048be       ?qt_invoke@QGuardedPtrPrivate@@UAE_NHPAUQUObject@@@Z 100058be f   qt-mt323:qt-mt323.dll
 0001:000048c4       ?qt_invoke@QPopupMenu@@UAE_NHPAUQUObject@@@Z 100058c4 f   qt-mt323:qt-mt323.dll
 0001:000048ca       ?qt_invoke@QToolBar@@UAE_NHPAUQUObject@@@Z 100058ca f   qt-mt323:qt-mt323.dll
 0001:000048d0       ?qt_invoke@QWidget@@UAE_NHPAUQUObject@@@Z 100058d0 f   qt-mt323:qt-mt323.dll
 0001:000048d6       ?qt_property@QAction@@UAE_NHHPAVQVariant@@@Z 100058d6 f   qt-mt323:qt-mt323.dll
 0001:000048dc       ?qt_property@QGuardedPtrPrivate@@UAE_NHHPAVQVariant@@@Z 100058dc f   qt-mt323:qt-mt323.dll
 0001:000048e2       ?qt_property@QPopupMenu@@UAE_NHHPAVQVariant@@@Z 100058e2 f   qt-mt323:qt-mt323.dll
 0001:000048e8       ?qt_property@QToolBar@@UAE_NHHPAVQVariant@@@Z 100058e8 f   qt-mt323:qt-mt323.dll
 0001:000048ee       ?qt_property@QWidget@@UAE_NHHPAVQVariant@@@Z 100058ee f   qt-mt323:qt-mt323.dll
 0001:000048f4       ?read@QGDict@@MAEAAVQDataStream@@AAV2@AAPAX@Z 100058f4 f   qt-mt323:qt-mt323.dll
 0001:000048fa       ?read@QGList@@MAEAAVQDataStream@@AAV2@AAPAX@Z 100058fa f   qt-mt323:qt-mt323.dll
 0001:00004900       ?removeFrom@QAction@@UAE_NPAVQWidget@@@Z 10005900 f   qt-mt323:qt-mt323.dll
 0001:00004906       ?resizeEvent@QFrame@@MAEXPAVQResizeEvent@@@Z 10005906 f   qt-mt323:qt-mt323.dll
 0001:0000490c       ?resizeEvent@QToolBar@@MAEXPAVQResizeEvent@@@Z 1000590c f   qt-mt323:qt-mt323.dll
 0001:00004912       ?setAccel@QAction@@UAEXABVQKeySequence@@@Z 10005912 f   qt-mt323:qt-mt323.dll
 0001:00004918       ?setActiveItem@QPopupMenu@@UAEXH@Z 10005918 f   qt-mt323:qt-mt323.dll
 0001:0000491e       ?setCaption@QDockWindow@@UAEXABVQString@@@Z 1000591e f   qt-mt323:qt-mt323.dll
 0001:00004924       ?setCheckable@QPopupMenu@@UAEX_N@Z 10005924 f   qt-mt323:qt-mt323.dll
 0001:0000492a       ?setCloseMode@QDockWindow@@UAEXH@Z 1000592a f   qt-mt323:qt-mt323.dll
 0001:00004930       ?setEnabled@QAction@@UAEX_N@Z 10005930 f   qt-mt323:qt-mt323.dll
 0001:00004936       ?setFirstItemActive@QPopupMenu@@EAEXXZ 10005936 f   qt-mt323:qt-mt323.dll
 0001:0000493c       ?setFixedExtentHeight@QDockWindow@@UAEXH@Z 1000593c f   qt-mt323:qt-mt323.dll
 0001:00004942       ?setFixedExtentWidth@QDockWindow@@UAEXH@Z 10005942 f   qt-mt323:qt-mt323.dll
 0001:00004948       ?setFont@QPopupMenu@@UAEXABVQFont@@@Z 10005948 f   qt-mt323:qt-mt323.dll
 0001:0000494e       ?setHorizontallyStretchable@QDockWindow@@UAEX_N@Z 1000594e f   qt-mt323:qt-mt323.dll
 0001:00004954       ?setIconSet@QAction@@UAEXABVQIconSet@@@Z 10005954 f   qt-mt323:qt-mt323.dll
 0001:0000495a       ?setId@QMenuData@@UAEXHH@Z 1000595a f   qt-mt323:qt-mt323.dll
 0001:00004960       ?setLabel@QToolBar@@UAEXABVQString@@@Z 10005960 f   qt-mt323:qt-mt323.dll
 0001:00004966       ?setMenuText@QAction@@UAEXABVQString@@@Z 10005966 f   qt-mt323:qt-mt323.dll
 0001:0000496c       ?setMinimumSize@QToolBar@@UAEXHH@Z 1000596c f   qt-mt323:qt-mt323.dll
 0001:00004972       ?setMovingEnabled@QDockWindow@@UAEX_N@Z 10005972 f   qt-mt323:qt-mt323.dll
 0001:00004978       ?setName@QObject@@UAEXPBD@Z 10005978 f   qt-mt323:qt-mt323.dll
 0001:0000497e       ?setNewLine@QDockWindow@@UAEX_N@Z 1000597e f   qt-mt323:qt-mt323.dll
 0001:00004984       ?setOffset@QDockWindow@@UAEXH@Z 10005984 f   qt-mt323:qt-mt323.dll
 0001:0000498a       ?setOn@QAction@@UAEX_N@Z   1000598a f   qt-mt323:qt-mt323.dll
 0001:00004990       ?setOpaqueMoving@QDockWindow@@UAEX_N@Z 10005990 f   qt-mt323:qt-mt323.dll
 0001:00004996       ?setOrientation@QToolBar@@UAEXW4Orientation@Qt@@@Z 10005996 f   qt-mt323:qt-mt323.dll
 0001:0000499c       ?setResizeEnabled@QDockWindow@@UAEX_N@Z 1000599c f   qt-mt323:qt-mt323.dll
 0001:000049a2       ?setStatusTip@QAction@@UAEXABVQString@@@Z 100059a2 f   qt-mt323:qt-mt323.dll
 0001:000049a8       ?setStretchableWidget@QToolBar@@UAEXPAVQWidget@@@Z 100059a8 f   qt-mt323:qt-mt323.dll
 0001:000049ae       ?setText@QAction@@UAEXABVQString@@@Z 100059ae f   qt-mt323:qt-mt323.dll
 0001:000049b4       ?setToggleAction@QAction@@UAEX_N@Z 100059b4 f   qt-mt323:qt-mt323.dll
 0001:000049ba       ?setToolTip@QAction@@UAEXABVQString@@@Z 100059ba f   qt-mt323:qt-mt323.dll
 0001:000049c0       ?setVerticallyStretchable@QDockWindow@@UAEX_N@Z 100059c0 f   qt-mt323:qt-mt323.dll
 0001:000049c6       ?setWhatsThis@QAction@@UAEXABVQString@@@Z 100059c6 f   qt-mt323:qt-mt323.dll
 0001:000049cc       ?setWidget@QDockWindow@@UAEXPAVQWidget@@@Z 100059cc f   qt-mt323:qt-mt323.dll
 0001:000049d2       ?show@QPopupMenu@@UAEXXZ   100059d2 f   qt-mt323:qt-mt323.dll
 0001:000049d8       ?show@QToolBar@@UAEXXZ     100059d8 f   qt-mt323:qt-mt323.dll
 0001:000049de       ?showEvent@QDockWindow@@MAEXPAVQShowEvent@@@Z 100059de f   qt-mt323:qt-mt323.dll
 0001:000049e4       ?sizeHint@QDockWindow@@UBE?AVQSize@@XZ 100059e4 f   qt-mt323:qt-mt323.dll
 0001:000049ea       ?sizeHint@QPopupMenu@@UBE?AVQSize@@XZ 100059ea f   qt-mt323:qt-mt323.dll
 0001:000049f0       ?styleChange@QPopupMenu@@MAEXAAVQStyle@@@Z 100059f0 f   qt-mt323:qt-mt323.dll
 0001:000049f6       ?styleChange@QToolBar@@MAEXAAVQStyle@@@Z 100059f6 f   qt-mt323:qt-mt323.dll
 0001:000049fc       ?timerEvent@QPopupMenu@@MAEXPAVQTimerEvent@@@Z 100059fc f   qt-mt323:qt-mt323.dll
 0001:00004a02       ?undock@QDockWindow@@UAEXPAVQWidget@@@Z 10005a02 f   qt-mt323:qt-mt323.dll
 0001:00004a08       ?undock@QDockWindow@@UAEXXZ 10005a08 f   qt-mt323:qt-mt323.dll
 0001:00004a0e       ?updateItem@QPopupMenu@@UAEXH@Z 10005a0e f   qt-mt323:qt-mt323.dll
 0001:00004a14       ?write@QGDict@@MBEAAVQDataStream@@AAV2@PAX@Z 10005a14 f   qt-mt323:qt-mt323.dll
 0001:00004a1a       ?write@QGList@@MBEAAVQDataStream@@AAV2@PAX@Z 10005a1a f   qt-mt323:qt-mt323.dll
 0001:00004a20       ?createEditor@QCheckTableItem@@UBEPAVQWidget@@XZ 10005a20 f   qt-mt323:qt-mt323.dll
 0001:00004a26       ?paint@QCheckTableItem@@UAEXPAVQPainter@@ABVQColorGroup@@ABVQRect@@_N@Z 10005a26 f   qt-mt323:qt-mt323.dll
 0001:00004a2c       ?rtti@QCheckTableItem@@UBEHXZ 10005a2c f   qt-mt323:qt-mt323.dll
 0001:00004a32       ?setChecked@QCheckTableItem@@UAEX_N@Z 10005a32 f   qt-mt323:qt-mt323.dll
 0001:00004a38       ?setContentFromEditor@QCheckTableItem@@UAEXPAVQWidget@@@Z 10005a38 f   qt-mt323:qt-mt323.dll
 0001:00004a3e       ?setText@QCheckTableItem@@UAEXABVQString@@@Z 10005a3e f   qt-mt323:qt-mt323.dll
 0001:00004a44       ?sizeHint@QCheckTableItem@@UBE?AVQSize@@XZ 10005a44 f   qt-mt323:qt-mt323.dll
 0001:00004a4a       ?addItem@QBoxLayout@@UAEXPAVQLayoutItem@@@Z 10005a4a f   qt-mt323:qt-mt323.dll
 0001:00004a50       ?childEvent@QLayout@@MAEXPAVQChildEvent@@@Z 10005a50 f   qt-mt323:qt-mt323.dll
 0001:00004a56       ?className@QVBoxLayout@@UBEPBDXZ 10005a56 f   qt-mt323:qt-mt323.dll
 0001:00004a5c       ?eventFilter@QLayout@@MAE_NPAVQObject@@PAVQEvent@@@Z 10005a5c f   qt-mt323:qt-mt323.dll
 0001:00004a62       ?expanding@QBoxLayout@@UBE?AW4ExpandData@QSizePolicy@@XZ 10005a62 f   qt-mt323:qt-mt323.dll
 0001:00004a68       ?geometry@QLayout@@UBE?AVQRect@@XZ 10005a68 f   qt-mt323:qt-mt323.dll
 0001:00004a6e       ?hasHeightForWidth@QBoxLayout@@UBE_NXZ 10005a6e f   qt-mt323:qt-mt323.dll
 0001:00004a74       ?heightForWidth@QBoxLayout@@UBEHH@Z 10005a74 f   qt-mt323:qt-mt323.dll
 0001:00004a7a       ?invalidate@QBoxLayout@@UAEXXZ 10005a7a f   qt-mt323:qt-mt323.dll
 0001:00004a80       ?isEmpty@QLayout@@UBE_NXZ  10005a80 f   qt-mt323:qt-mt323.dll
 0001:00004a86       ?iterator@QBoxLayout@@UAE?AVQLayoutIterator@@XZ 10005a86 f   qt-mt323:qt-mt323.dll
 0001:00004a8c       ?layout@QLayout@@UAEPAV1@XZ 10005a8c f   qt-mt323:qt-mt323.dll
 0001:00004a92       ?maximumSize@QBoxLayout@@UBE?AVQSize@@XZ 10005a92 f   qt-mt323:qt-mt323.dll
 0001:00004a98       ?metaObject@QVBoxLayout@@UBEPAVQMetaObject@@XZ 10005a98 f   qt-mt323:qt-mt323.dll
 0001:00004a9e       ?minimumSize@QBoxLayout@@UBE?AVQSize@@XZ 10005a9e f   qt-mt323:qt-mt323.dll
 0001:00004aa4       ?qt_cast@QVBoxLayout@@UAEPAXPBD@Z 10005aa4 f   qt-mt323:qt-mt323.dll
 0001:00004aaa       ?qt_emit@QVBoxLayout@@UAE_NHPAUQUObject@@@Z 10005aaa f   qt-mt323:qt-mt323.dll
 0001:00004ab0       ?qt_invoke@QVBoxLayout@@UAE_NHPAUQUObject@@@Z 10005ab0 f   qt-mt323:qt-mt323.dll
 0001:00004ab6       ?qt_property@QVBoxLayout@@UAE_NHHPAVQVariant@@@Z 10005ab6 f   qt-mt323:qt-mt323.dll
 0001:00004abc       ?setAlignment@QLayoutItem@@UAEXH@Z 10005abc f   qt-mt323:qt-mt323.dll
 0001:00004ac2       ?setAutoAdd@QLayout@@UAEX_N@Z 10005ac2 f   qt-mt323:qt-mt323.dll
 0001:00004ac8       ?setGeometry@QBoxLayout@@UAEXABVQRect@@@Z 10005ac8 f   qt-mt323:qt-mt323.dll
 0001:00004ace       ?setMargin@QLayout@@UAEXH@Z 10005ace f   qt-mt323:qt-mt323.dll
 0001:00004ad4       ?setMenuBar@QLayout@@UAEXPAVQMenuBar@@@Z 10005ad4 f   qt-mt323:qt-mt323.dll
 0001:00004ada       ?setSpacing@QLayout@@UAEXH@Z 10005ada f   qt-mt323:qt-mt323.dll
 0001:00004ae0       ?sizeHint@QBoxLayout@@UBE?AVQSize@@XZ 10005ae0 f   qt-mt323:qt-mt323.dll
 0001:00004ae6       ?spacerItem@QLayoutItem@@UAEPAVQSpacerItem@@XZ 10005ae6 f   qt-mt323:qt-mt323.dll
 0001:00004aec       ?widget@QLayoutItem@@UAEPAVQWidget@@XZ 10005aec f   qt-mt323:qt-mt323.dll
 0001:00004af2       ?className@QLabel@@UBEPBDXZ 10005af2 f   qt-mt323:qt-mt323.dll
 0001:00004af8       ?drawContents@QLabel@@MAEXPAVQPainter@@@Z 10005af8 f   qt-mt323:qt-mt323.dll
 0001:00004afe       ?fontChange@QLabel@@MAEXABVQFont@@@Z 10005afe f   qt-mt323:qt-mt323.dll
 0001:00004b04       ?heightForWidth@QLabel@@UBEHH@Z 10005b04 f   qt-mt323:qt-mt323.dll
 0001:00004b0a       ?metaObject@QLabel@@UBEPAVQMetaObject@@XZ 10005b0a f   qt-mt323:qt-mt323.dll
 0001:00004b10       ?minimumSizeHint@QLabel@@UBE?AVQSize@@XZ 10005b10 f   qt-mt323:qt-mt323.dll
 0001:00004b16       ?qt_cast@QLabel@@UAEPAXPBD@Z 10005b16 f   qt-mt323:qt-mt323.dll
 0001:00004b1c       ?qt_emit@QLabel@@UAE_NHPAUQUObject@@@Z 10005b1c f   qt-mt323:qt-mt323.dll
 0001:00004b22       ?qt_invoke@QLabel@@UAE_NHPAUQUObject@@@Z 10005b22 f   qt-mt323:qt-mt323.dll
 0001:00004b28       ?qt_property@QLabel@@UAE_NHHPAVQVariant@@@Z 10005b28 f   qt-mt323:qt-mt323.dll
 0001:00004b2e       ?resizeEvent@QLabel@@MAEXPAVQResizeEvent@@@Z 10005b2e f   qt-mt323:qt-mt323.dll
 0001:00004b34       ?setAlignment@QLabel@@UAEXH@Z 10005b34 f   qt-mt323:qt-mt323.dll
 0001:00004b3a       ?setAutoResize@QLabel@@UAEX_N@Z 10005b3a f   qt-mt323:qt-mt323.dll
 0001:00004b40       ?setBuddy@QLabel@@UAEXPAVQWidget@@@Z 10005b40 f   qt-mt323:qt-mt323.dll
 0001:00004b46       ?setFont@QLabel@@UAEXABVQFont@@@Z 10005b46 f   qt-mt323:qt-mt323.dll
 0001:00004b4c       ?setMovie@QLabel@@UAEXABVQMovie@@@Z 10005b4c f   qt-mt323:qt-mt323.dll
 0001:00004b52       ?setNum@QLabel@@UAEXH@Z    10005b52 f   qt-mt323:qt-mt323.dll
 0001:00004b58       ?setNum@QLabel@@UAEXN@Z    10005b58 f   qt-mt323:qt-mt323.dll
 0001:00004b5e       ?setPicture@QLabel@@UAEXABVQPicture@@@Z 10005b5e f   qt-mt323:qt-mt323.dll
 0001:00004b64       ?setPixmap@QLabel@@UAEXABVQPixmap@@@Z 10005b64 f   qt-mt323:qt-mt323.dll
 0001:00004b6a       ?setText@QLabel@@UAEXABVQString@@@Z 10005b6a f   qt-mt323:qt-mt323.dll
 0001:00004b70       ?sizeHint@QLabel@@UBE?AVQSize@@XZ 10005b70 f   qt-mt323:qt-mt323.dll
 0001:00004b76       ?styleChange@QFrame@@MAEXAAVQStyle@@@Z 10005b76 f   qt-mt323:qt-mt323.dll
 0001:00004b7c       ??3@YAXPAX@Z               10005b7c f   MSVCRT:MSVCR120.dll
 0001:00004b82       @__security_check_cookie@4 10005b82 f   MSVCRT:secchk.obj
 0001:00004b91       __EH_epilog3               10005b91 f   MSVCRT:ehprolg3.obj
 0001:00004ba5       __EH_epilog3_GS            10005ba5 f   MSVCRT:ehprolg3.obj
 0001:00004bb4       __EH_prolog3               10005bb4 f   MSVCRT:ehprolg3.obj
 0001:00004be7       __EH_prolog3_GS            10005be7 f   MSVCRT:ehprolg3.obj
 0001:00004c1e       ___CxxFrameHandler3        10005c1e f   MSVCRT:MSVCR120.dll
 0001:00004c24       ??_Etype_info@@UAEPAXI@Z   10005c24 f i MSVCRT:ti_inst.obj
 0001:00004c6e       ??2@YAPAXI@Z               10005c6e f   MSVCRT:MSVCR120.dll
 0001:00004c74       __purecall                 10005c74 f   MSVCRT:MSVCR120.dll
 0001:00004c7a       ___atonexitinit            10005c7a f   MSVCRT:atonexit.obj
 0001:00004cb6       __onexit                   10005cb6 f   MSVCRT:atonexit.obj
 0001:00004d5f       _atexit                    10005d5f f   MSVCRT:atonexit.obj
 0001:00004d74       ??_L@YGXPAXIHP6EX0@Z1@Z    10005d74 f   MSVCRT:ehvecctr.obj
 0001:00004dd6       ??_M@YGXPAXIHP6EX0@Z@Z     10005dd6 f   MSVCRT:ehvecdtr.obj
 0001:00004e45       ?__ArrayUnwind@@YGXPAXIHP6EX0@Z@Z 10005e45 f   MSVCRT:ehvecdtr.obj
 0001:00004ef2       __CRT_INIT@12              10005ef2 f   MSVCRT:crtdll.obj
 0001:000050e9       __DllMainCRTStartup@12     100060e9 f   MSVCRT:crtdll.obj
 0001:0000523f       ___raise_securityfailure   1000623f f   MSVCRT:gs_report.obj
 0001:0000527c       ___report_gsfailure        1000627c f   MSVCRT:gs_report.obj
 0001:00005378       ??1type_info@@UAE@XZ       10006378 f   MSVCRT:MSVCR120.dll
 0001:0000537e       __lock                     1000637e f   MSVCRT:MSVCR120.dll
 0001:00005384       __unlock                   10006384 f   MSVCRT:MSVCR120.dll
 0001:0000538a       ___dllonexit               1000638a f   MSVCRT:MSVCR120.dll
 0001:00005390       __SEH_prolog4              10006390 f   MSVCRT:sehprolg4.obj
 0001:000053d5       __SEH_epilog4              100063d5 f   MSVCRT:sehprolg4.obj
 0001:000053e9       __except_handler4          100063e9 f   MSVCRT:chandler4gs.obj
 0001:0000540c       ?terminate@@YAXXZ          1000640c f   MSVCRT:MSVCR120.dll
 0001:00005412       ___CppXcptFilter           10006412 f   MSVCRT:MSVCR120.dll
 0001:00005418       __amsg_exit                10006418 f   MSVCRT:MSVCR120.dll
 0001:00005420       __FindPESection            10006420 f   MSVCRT:pesect.obj
 0001:00005470       __IsNonwritableInCurrentImage 10006470 f   MSVCRT:pesect.obj
 0001:00005530       __ValidateImageBase        10006530 f   MSVCRT:pesect.obj
 0001:00005561       ___security_init_cookie    10006561 f   MSVCRT:gs_support.obj
 0001:000055fd       _DllMain@12                100065fd f   MSVCRT:dllmain.obj
 0001:0000561f       __RTC_Initialize           1000661f f   MSVCRT:initsect.obj
 0001:0000563f       __RTC_Terminate            1000663f f   MSVCRT:initsect.obj
 0001:00005660       __initterm                 10006660 f   MSVCRT:MSVCR120.dll
 0001:00005666       __initterm_e               10006666 f   MSVCRT:MSVCR120.dll
 0001:0000566c       ___clean_type_info_names   1000666c f   MSVCRT:tncleanup.obj
 0001:00005678       __crt_debugger_hook        10006678 f   MSVCRT:MSVCR120.dll
 0001:0000567e       ___crtUnhandledException   1000667e f   MSVCRT:MSVCR120.dll
 0001:00005684       ___crtTerminateProcess     10006684 f   MSVCRT:MSVCR120.dll
 0001:0000568a       __except_handler4_common   1000668a f   MSVCRT:MSVCR120.dll
 0001:00005690       ___clean_type_info_names_internal 10006690 f   MSVCRT:MSVCR120.dll
 0001:00005696       _IsProcessorFeaturePresent@4 10006696 f   kernel32:KERNEL32.dll
 0002:00000000       __imp__DecodePointer@4     10008000     kernel32:KERNEL32.dll
 0002:00000004       __imp__DisableThreadLibraryCalls@4 10008004     kernel32:KERNEL32.dll
 0002:00000008       __imp__GetSystemTimeAsFileTime@4 10008008     kernel32:KERNEL32.dll
 0002:0000000c       __imp__GetCurrentThreadId@0 1000800c     kernel32:KERNEL32.dll
 0002:00000010       __imp__GetCurrentProcessId@0 10008010     kernel32:KERNEL32.dll
 0002:00000014       __imp__QueryPerformanceCounter@4 10008014     kernel32:KERNEL32.dll
 0002:00000018       __imp__IsProcessorFeaturePresent@4 10008018     kernel32:KERNEL32.dll
 0002:0000001c       __imp__IsDebuggerPresent@0 1000801c     kernel32:KERNEL32.dll
 0002:00000020       __imp__EncodePointer@4     10008020     kernel32:KERNEL32.dll
 0002:00000024       \177KERNEL32_NULL_THUNK_DATA 10008024     kernel32:KERNEL32.dll
 0002:00000028       __imp____CxxFrameHandler3  10008028     MSVCRT:MSVCR120.dll
 0002:0000002c       __imp____clean_type_info_names_internal 1000802c     MSVCRT:MSVCR120.dll
 0002:00000030       __imp___except_handler4_common 10008030     MSVCRT:MSVCR120.dll
 0002:00000034       __imp____crtTerminateProcess 10008034     MSVCRT:MSVCR120.dll
 0002:00000038       __imp____crtUnhandledException 10008038     MSVCRT:MSVCR120.dll
 0002:0000003c       __imp___crt_debugger_hook  1000803c     MSVCRT:MSVCR120.dll
 0002:00000040       __imp___initterm_e         10008040     MSVCRT:MSVCR120.dll
 0002:00000044       __imp___initterm           10008044     MSVCRT:MSVCR120.dll
 0002:00000048       __imp___malloc_crt         10008048     MSVCRT:MSVCR120.dll
 0002:0000004c       __imp__free                1000804c     MSVCRT:MSVCR120.dll
 0002:00000050       __imp___amsg_exit          10008050     MSVCRT:MSVCR120.dll
 0002:00000054       __imp____CppXcptFilter     10008054     MSVCRT:MSVCR120.dll
 0002:00000058       __imp_?terminate@@YAXXZ    10008058     MSVCRT:MSVCR120.dll
 0002:0000005c       __imp___onexit             1000805c     MSVCRT:MSVCR120.dll
 0002:00000060       __imp____dllonexit         10008060     MSVCRT:MSVCR120.dll
 0002:00000064       __imp___calloc_crt         10008064     MSVCRT:MSVCR120.dll
 0002:00000068       __imp___unlock             10008068     MSVCRT:MSVCR120.dll
 0002:0000006c       __imp___lock               1000806c     MSVCRT:MSVCR120.dll
 0002:00000070       __imp_??1type_info@@UAE@XZ 10008070     MSVCRT:MSVCR120.dll
 0002:00000074       __imp___purecall           10008074     MSVCRT:MSVCR120.dll
 0002:00000078       __imp_??2@YAPAXI@Z         10008078     MSVCRT:MSVCR120.dll
 0002:0000007c       __imp_??3@YAXPAX@Z         1000807c     MSVCRT:MSVCR120.dll
 0002:00000080       \177MSVCR120_NULL_THUNK_DATA 10008080     MSVCRT:MSVCR120.dll
 0002:00000084       __imp_?fnConfig_icons@@YAPAPBDPBD@Z 10008084     config_icons:config_icons.dll
 0002:00000088       \177config_icons_NULL_THUNK_DATA 10008088     config_icons:config_icons.dll
 0002:0000008c       __imp_?columnAt@QTable@@UBEHH@Z 1000808c     qt-mt323:qt-mt323.dll
 0002:00000090       __imp_?columnClicked@QTable@@MAEXH@Z 10008090     qt-mt323:qt-mt323.dll
 0002:00000094       __imp_?columnIndexChanged@QTable@@MAEXHHH@Z 10008094     qt-mt323:qt-mt323.dll
 0002:00000098       __imp_?columnPos@QTable@@UBEHH@Z 10008098     qt-mt323:qt-mt323.dll
 0002:0000009c       __imp_?columnWidth@QTable@@UBEHH@Z 1000809c     qt-mt323:qt-mt323.dll
 0002:000000a0       __imp_?columnWidthChanged@QTable@@MAEXH@Z 100080a0     qt-mt323:qt-mt323.dll
 0002:000000a4       __imp_?connectNotify@QObject@@MAEXPBD@Z 100080a4     qt-mt323:qt-mt323.dll
 0002:000000a8       __imp_?contentsContextMenuEvent@QTable@@MAEXPAVQContextMenuEvent@@@Z 100080a8     qt-mt323:qt-mt323.dll
 0002:000000ac       __imp_?contentsDragEnterEvent@QTable@@MAEXPAVQDragEnterEvent@@@Z 100080ac     qt-mt323:qt-mt323.dll
 0002:000000b0       __imp_?contentsDragLeaveEvent@QTable@@MAEXPAVQDragLeaveEvent@@@Z 100080b0     qt-mt323:qt-mt323.dll
 0002:000000b4       __imp_?contentsDragMoveEvent@QTable@@MAEXPAVQDragMoveEvent@@@Z 100080b4     qt-mt323:qt-mt323.dll
 0002:000000b8       __imp_?contentsDropEvent@QTable@@MAEXPAVQDropEvent@@@Z 100080b8     qt-mt323:qt-mt323.dll
 0002:000000bc       __imp_?contentsMouseDoubleClickEvent@QTable@@MAEXPAVQMouseEvent@@@Z 100080bc     qt-mt323:qt-mt323.dll
 0002:000000c0       __imp_?contentsMouseMoveEvent@QTable@@MAEXPAVQMouseEvent@@@Z 100080c0     qt-mt323:qt-mt323.dll
 0002:000000c4       __imp_?contentsMousePressEvent@QTable@@MAEXPAVQMouseEvent@@@Z 100080c4     qt-mt323:qt-mt323.dll
 0002:000000c8       __imp_?contentsMouseReleaseEvent@QTable@@MAEXPAVQMouseEvent@@@Z 100080c8     qt-mt323:qt-mt323.dll
 0002:000000cc       __imp_?contentsWheelEvent@QScrollView@@MAEXPAVQWheelEvent@@@Z 100080cc     qt-mt323:qt-mt323.dll
 0002:000000d0       __imp_?contextMenuEvent@QScrollView@@MAEXPAVQContextMenuEvent@@@Z 100080d0     qt-mt323:qt-mt323.dll
 0002:000000d4       __imp_?create@QWidget@@MAEXPAUHWND__@@_N1@Z 100080d4     qt-mt323:qt-mt323.dll
 0002:000000d8       __imp_?createEditor@QTable@@MBEPAVQWidget@@HH_N@Z 100080d8     qt-mt323:qt-mt323.dll
 0002:000000dc       __imp_?currentSelection@QTable@@UBEHXZ 100080dc     qt-mt323:qt-mt323.dll
 0002:000000e0       __imp_?customEvent@QObject@@MAEXPAVQCustomEvent@@@Z 100080e0     qt-mt323:qt-mt323.dll
 0002:000000e4       __imp_?customWhatsThis@QWidget@@UBE_NXZ 100080e4     qt-mt323:qt-mt323.dll
 0002:000000e8       __imp_?destroy@QWidget@@MAEX_N0@Z 100080e8     qt-mt323:qt-mt323.dll
 0002:000000ec       __imp_?disconnectNotify@QObject@@MAEXPBD@Z 100080ec     qt-mt323:qt-mt323.dll
 0002:000000f0       __imp_?dragEnterEvent@QWidget@@MAEXPAVQDragEnterEvent@@@Z 100080f0     qt-mt323:qt-mt323.dll
 0002:000000f4       __imp_?dragLeaveEvent@QWidget@@MAEXPAVQDragLeaveEvent@@@Z 100080f4     qt-mt323:qt-mt323.dll
 0002:000000f8       __imp_?dragMoveEvent@QWidget@@MAEXPAVQDragMoveEvent@@@Z 100080f8     qt-mt323:qt-mt323.dll
 0002:000000fc       __imp_?dragObject@QTable@@MAEPAVQDragObject@@XZ 100080fc     qt-mt323:qt-mt323.dll
 0002:00000100       __imp_?drawContents@QTable@@EAEXPAVQPainter@@@Z 10008100     qt-mt323:qt-mt323.dll
 0002:00000104       __imp_?drawContents@QTable@@MAEXPAVQPainter@@HHHH@Z 10008104     qt-mt323:qt-mt323.dll
 0002:00000108       __imp_?drawContentsOffset@QScrollView@@MAEXPAVQPainter@@HHHHHH@Z 10008108     qt-mt323:qt-mt323.dll
 0002:0000010c       __imp_?drawFrame@QFrame@@MAEXPAVQPainter@@@Z 1000810c     qt-mt323:qt-mt323.dll
 0002:00000110       __imp_?dropEvent@QWidget@@MAEXPAVQDropEvent@@@Z 10008110     qt-mt323:qt-mt323.dll
 0002:00000114       __imp_?editCell@QTable@@UAEXHH_N@Z 10008114     qt-mt323:qt-mt323.dll
 0002:00000118       __imp_?enabledChange@QWidget@@MAEX_N@Z 10008118     qt-mt323:qt-mt323.dll
 0002:0000011c       __imp_?endEdit@QTable@@MAEXHH_N0@Z 1000811c     qt-mt323:qt-mt323.dll
 0002:00000120       __imp_?enterEvent@QWidget@@MAEXPAVQEvent@@@Z 10008120     qt-mt323:qt-mt323.dll
 0002:00000124       __imp_?event@QWidget@@MAE_NPAVQEvent@@@Z 10008124     qt-mt323:qt-mt323.dll
 0002:00000128       __imp_?eventFilter@QTable@@UAE_NPAVQObject@@PAVQEvent@@@Z 10008128     qt-mt323:qt-mt323.dll
 0002:0000012c       __imp_?focusInEvent@QTable@@MAEXPAVQFocusEvent@@@Z 1000812c     qt-mt323:qt-mt323.dll
 0002:00000130       __imp_?focusNextPrevChild@QScrollView@@MAE_N_N@Z 10008130     qt-mt323:qt-mt323.dll
 0002:00000134       __imp_?focusOutEvent@QTable@@MAEXPAVQFocusEvent@@@Z 10008134     qt-mt323:qt-mt323.dll
 0002:00000138       __imp_?fontChange@QScrollView@@MAEXABVQFont@@@Z 10008138     qt-mt323:qt-mt323.dll
 0002:0000013c       __imp_?fontInf@QPaintDevice@@MBEHPAVQFont@@H@Z 1000813c     qt-mt323:qt-mt323.dll
 0002:00000140       __imp_?fontMet@QPaintDevice@@MBEHPAVQFont@@HPBDH@Z 10008140     qt-mt323:qt-mt323.dll
 0002:00000144       __imp_?frameChanged@QScrollView@@MAEXXZ 10008144     qt-mt323:qt-mt323.dll
 0002:00000148       __imp_?handle@QPaintDevice@@UBEPAUHDC__@@XZ 10008148     qt-mt323:qt-mt323.dll
 0002:0000014c       __imp_?heightForWidth@QWidget@@UBEHH@Z 1000814c     qt-mt323:qt-mt323.dll
 0002:00000150       __imp_?hide@QWidget@@UAEXXZ 10008150     qt-mt323:qt-mt323.dll
 0002:00000154       __imp_?hideColumn@QTable@@UAEXH@Z 10008154     qt-mt323:qt-mt323.dll
 0002:00000158       __imp_?hideEvent@QWidget@@MAEXPAVQHideEvent@@@Z 10008158     qt-mt323:qt-mt323.dll
 0002:0000015c       __imp_?hideRow@QTable@@UAEXH@Z 1000815c     qt-mt323:qt-mt323.dll
 0002:00000160       __imp_?imComposeEvent@QWidget@@MAEXPAVQIMEvent@@@Z 10008160     qt-mt323:qt-mt323.dll
 0002:00000164       __imp_?imEndEvent@QWidget@@MAEXPAVQIMEvent@@@Z 10008164     qt-mt323:qt-mt323.dll
 0002:00000168       __imp_?imStartEvent@QWidget@@MAEXPAVQIMEvent@@@Z 10008168     qt-mt323:qt-mt323.dll
 0002:0000016c       __imp_?insertChild@QObject@@UAEXPAV1@@Z 1000816c     qt-mt323:qt-mt323.dll
 0002:00000170       __imp_?insertColumns@QTable@@UAEXHH@Z 10008170     qt-mt323:qt-mt323.dll
 0002:00000174       __imp_?insertRows@QTable@@UAEXHH@Z 10008174     qt-mt323:qt-mt323.dll
 0002:00000178       __imp_?insertWidget@QTable@@MAEXHHPAVQWidget@@@Z 10008178     qt-mt323:qt-mt323.dll
 0002:0000017c       __imp_?item@QTable@@UBEPAVQTableItem@@HH@Z 1000817c     qt-mt323:qt-mt323.dll
 0002:00000180       __imp_?keyReleaseEvent@QWidget@@MAEXPAVQKeyEvent@@@Z 10008180     qt-mt323:qt-mt323.dll
 0002:00000184       __imp_?leaveEvent@QWidget@@MAEXPAVQEvent@@@Z 10008184     qt-mt323:qt-mt323.dll
 0002:00000188       __imp_?metric@QWidget@@MBEHH@Z 10008188     qt-mt323:qt-mt323.dll
 0002:0000018c       __imp_?minimumSizeHint@QScrollView@@UBE?AVQSize@@XZ 1000818c     qt-mt323:qt-mt323.dll
 0002:00000190       __imp_?mouseDoubleClickEvent@QScrollView@@MAEXPAVQMouseEvent@@@Z 10008190     qt-mt323:qt-mt323.dll
 0002:00000194       __imp_?mouseMoveEvent@QScrollView@@MAEXPAVQMouseEvent@@@Z 10008194     qt-mt323:qt-mt323.dll
 0002:00000198       __imp_?mousePressEvent@QScrollView@@MAEXPAVQMouseEvent@@@Z 10008198     qt-mt323:qt-mt323.dll
 0002:0000019c       __imp_?mouseReleaseEvent@QScrollView@@MAEXPAVQMouseEvent@@@Z 1000819c     qt-mt323:qt-mt323.dll
 0002:000001a0       __imp_?move@QWidget@@UAEXHH@Z 100081a0     qt-mt323:qt-mt323.dll
 0002:000001a4       __imp_?moveChild@QScrollView@@UAEXPAVQWidget@@HH@Z 100081a4     qt-mt323:qt-mt323.dll
 0002:000001a8       __imp_?moveEvent@QWidget@@MAEXPAVQMoveEvent@@@Z 100081a8     qt-mt323:qt-mt323.dll
 0002:000001ac       __imp_?numCols@QTable@@UBEHXZ 100081ac     qt-mt323:qt-mt323.dll
 0002:000001b0       __imp_?numRows@QTable@@UBEHXZ 100081b0     qt-mt323:qt-mt323.dll
 0002:000001b4       __imp_?paintCell@QTable@@UAEXPAVQPainter@@HHABVQRect@@_N@Z 100081b4     qt-mt323:qt-mt323.dll
 0002:000001b8       __imp_?paintCell@QTable@@UAEXPAVQPainter@@HHABVQRect@@_NABVQColorGroup@@@Z 100081b8     qt-mt323:qt-mt323.dll
 0002:000001bc       __imp_?paintEmptyArea@QTable@@MAEXPAVQPainter@@HHHH@Z 100081bc     qt-mt323:qt-mt323.dll
 0002:000001c0       __imp_?paintEvent@QTable@@MAEXPAVQPaintEvent@@@Z 100081c0     qt-mt323:qt-mt323.dll
 0002:000001c4       __imp_?paintFocus@QTable@@UAEXPAVQPainter@@ABVQRect@@@Z 100081c4     qt-mt323:qt-mt323.dll
 0002:000001c8       __imp_?paletteChange@QWidget@@MAEXABVQPalette@@@Z 100081c8     qt-mt323:qt-mt323.dll
 0002:000001cc       __imp_?pixmap@QTable@@UBE?AVQPixmap@@HH@Z 100081cc     qt-mt323:qt-mt323.dll
 0002:000001d0       __imp_?polish@QWidget@@UAEXXZ 100081d0     qt-mt323:qt-mt323.dll
 0002:000001d4       __imp_?property@QObject@@UBE?AVQVariant@@PBD@Z 100081d4     qt-mt323:qt-mt323.dll
 0002:000001d8       __imp_?removeChild@QScrollView@@UAEXPAVQObject@@@Z 100081d8     qt-mt323:qt-mt323.dll
 0002:000001dc       __imp_?removeColumn@QTable@@UAEXH@Z 100081dc     qt-mt323:qt-mt323.dll
 0002:000001e0       __imp_?removeColumns@QTable@@UAEXABV?$QMemArray@H@@@Z 100081e0     qt-mt323:qt-mt323.dll
 0002:000001e4       __imp_?removeRow@QTable@@UAEXH@Z 100081e4     qt-mt323:qt-mt323.dll
 0002:000001e8       __imp_?removeRows@QTable@@UAEXABV?$QMemArray@H@@@Z 100081e8     qt-mt323:qt-mt323.dll
 0002:000001ec       __imp_?removeSelection@QTable@@UAEXABVQTableSelection@@@Z 100081ec     qt-mt323:qt-mt323.dll
 0002:000001f0       __imp_?removeSelection@QTable@@UAEXH@Z 100081f0     qt-mt323:qt-mt323.dll
 0002:000001f4       __imp_?reparent@QWidget@@UAEXPAV1@IABVQPoint@@_N@Z 100081f4     qt-mt323:qt-mt323.dll
 0002:000001f8       __imp_?resize@QScrollView@@UAEXHH@Z 100081f8     qt-mt323:qt-mt323.dll
 0002:000001fc       __imp_?resizeContents@QScrollView@@UAEXHH@Z 100081fc     qt-mt323:qt-mt323.dll
 0002:00000200       __imp_?resizeData@QTable@@MAEXH@Z 10008200     qt-mt323:qt-mt323.dll
 0002:00000204       __imp_?resizeEvent@QScrollView@@MAEXPAVQResizeEvent@@@Z 10008204     qt-mt323:qt-mt323.dll
 0002:00000208       __imp_?resolution@QPaintDevice@@UBEHXZ 10008208     qt-mt323:qt-mt323.dll
 0002:0000020c       __imp_?rowAt@QTable@@UBEHH@Z 1000820c     qt-mt323:qt-mt323.dll
 0002:00000210       __imp_?rowHeight@QTable@@UBEHH@Z 10008210     qt-mt323:qt-mt323.dll
 0002:00000214       __imp_?rowHeightChanged@QTable@@MAEXH@Z 10008214     qt-mt323:qt-mt323.dll
 0002:00000218       __imp_?rowIndexChanged@QTable@@MAEXHHH@Z 10008218     qt-mt323:qt-mt323.dll
 0002:0000021c       __imp_?rowPos@QTable@@UBEHH@Z 1000821c     qt-mt323:qt-mt323.dll
 0002:00000220       __imp_?setAcceptDrops@QWidget@@UAEX_N@Z 10008220     qt-mt323:qt-mt323.dll
 0002:00000224       __imp_?setActiveWindow@QWidget@@UAEXXZ 10008224     qt-mt323:qt-mt323.dll
 0002:00000228       __imp_?setAutoMask@QWidget@@UAEX_N@Z 10008228     qt-mt323:qt-mt323.dll
 0002:0000022c       __imp_?setBackgroundColor@QWidget@@UAEXABVQColor@@@Z 1000822c     qt-mt323:qt-mt323.dll
 0002:00000230       __imp_?setBackgroundMode@QWidget@@UAEXW4BackgroundMode@Qt@@@Z 10008230     qt-mt323:qt-mt323.dll
 0002:00000234       __imp_?setBackgroundOrigin@QWidget@@UAEXW4BackgroundOrigin@1@@Z 10008234     qt-mt323:qt-mt323.dll
 0002:00000238       __imp_?setBackgroundPixmap@QWidget@@UAEXABVQPixmap@@@Z 10008238     qt-mt323:qt-mt323.dll
 0002:0000023c       __imp_?setCaption@QWidget@@UAEXABVQString@@@Z 1000823c     qt-mt323:qt-mt323.dll
 0002:00000240       __imp_?setCellContentFromEditor@QTable@@MAEXHH@Z 10008240     qt-mt323:qt-mt323.dll
 0002:00000244       __imp_?setCellWidget@QTable@@UAEXHHPAVQWidget@@@Z 10008244     qt-mt323:qt-mt323.dll
 0002:00000248       __imp_?setColumnMovingEnabled@QTable@@UAEX_N@Z 10008248     qt-mt323:qt-mt323.dll
 0002:0000024c       __imp_?setColumnReadOnly@QTable@@UAEXH_N@Z 1000824c     qt-mt323:qt-mt323.dll
 0002:00000250       __imp_?setColumnStretchable@QTable@@UAEXH_N@Z 10008250     qt-mt323:qt-mt323.dll
 0002:00000254       __imp_?setColumnWidth@QTable@@UAEXHH@Z 10008254     qt-mt323:qt-mt323.dll
 0002:00000258       __imp_?setContentsPos@QScrollView@@UAEXHH@Z 10008258     qt-mt323:qt-mt323.dll
 0002:0000025c       __imp_?setCornerWidget@QScrollView@@UAEXPAVQWidget@@@Z 1000825c     qt-mt323:qt-mt323.dll
 0002:00000260       __imp_?setCurrentCell@QTable@@UAEXHH@Z 10008260     qt-mt323:qt-mt323.dll
 0002:00000264       __imp_?setCursor@QWidget@@UAEXABVQCursor@@@Z 10008264     qt-mt323:qt-mt323.dll
 0002:00000268       __imp_?setDragAutoScroll@QScrollView@@UAEX_N@Z 10008268     qt-mt323:qt-mt323.dll
 0002:0000026c       __imp_?setDragEnabled@QTable@@UAEX_N@Z 1000826c     qt-mt323:qt-mt323.dll
 0002:00000270       __imp_?setEnabled@QTable@@UAEX_N@Z 10008270     qt-mt323:qt-mt323.dll
 0002:00000274       __imp_?setEraseColor@QWidget@@UAEXABVQColor@@@Z 10008274     qt-mt323:qt-mt323.dll
 0002:00000278       __imp_?setErasePixmap@QWidget@@UAEXABVQPixmap@@@Z 10008278     qt-mt323:qt-mt323.dll
 0002:0000027c       __imp_?setFocus@QWidget@@UAEXXZ 1000827c     qt-mt323:qt-mt323.dll
 0002:00000280       __imp_?setFocusPolicy@QWidget@@UAEXW4FocusPolicy@1@@Z 10008280     qt-mt323:qt-mt323.dll
 0002:00000284       __imp_?setFocusProxy@QWidget@@UAEXPAV1@@Z 10008284     qt-mt323:qt-mt323.dll
 0002:00000288       __imp_?setFocusStyle@QTable@@UAEXW4FocusStyle@1@@Z 10008288     qt-mt323:qt-mt323.dll
 0002:0000028c       __imp_?setFont@QWidget@@UAEXABVQFont@@@Z 1000828c     qt-mt323:qt-mt323.dll
 0002:00000290       __imp_?setFrameRect@QFrame@@UAEXABVQRect@@@Z 10008290     qt-mt323:qt-mt323.dll
 0002:00000294       __imp_?setFrameStyle@QFrame@@UAEXH@Z 10008294     qt-mt323:qt-mt323.dll
 0002:00000298       __imp_?setGeometry@QWidget@@UAEXABVQRect@@@Z 10008298     qt-mt323:qt-mt323.dll
 0002:0000029c       __imp_?setGeometry@QWidget@@UAEXHHHH@Z 1000829c     qt-mt323:qt-mt323.dll
 0002:000002a0       __imp_?setHBarGeometry@QScrollView@@MAEXAAVQScrollBar@@HHHH@Z 100082a0     qt-mt323:qt-mt323.dll
 0002:000002a4       __imp_?setHScrollBarMode@QScrollView@@UAEXW4ScrollBarMode@1@@Z 100082a4     qt-mt323:qt-mt323.dll
 0002:000002a8       __imp_?setIcon@QWidget@@UAEXABVQPixmap@@@Z 100082a8     qt-mt323:qt-mt323.dll
 0002:000002ac       __imp_?setIconText@QWidget@@UAEXABVQString@@@Z 100082ac     qt-mt323:qt-mt323.dll
 0002:000002b0       __imp_?setItem@QTable@@UAEXHHPAVQTableItem@@@Z 100082b0     qt-mt323:qt-mt323.dll
 0002:000002b4       __imp_?setKeyCompression@QWidget@@MAEX_N@Z 100082b4     qt-mt323:qt-mt323.dll
 0002:000002b8       __imp_?setLeftMargin@QTable@@UAEXH@Z 100082b8     qt-mt323:qt-mt323.dll
 0002:000002bc       __imp_?setLineWidth@QFrame@@UAEXH@Z 100082bc     qt-mt323:qt-mt323.dll
 0002:000002c0       __imp_?setMargin@QFrame@@UAEXH@Z 100082c0     qt-mt323:qt-mt323.dll
 0002:000002c4       __imp_?setMargins@QScrollView@@MAEXHHHH@Z 100082c4     qt-mt323:qt-mt323.dll
 0002:000002c8       __imp_?setMask@QWidget@@UAEXABVQBitmap@@@Z 100082c8     qt-mt323:qt-mt323.dll
 0002:000002cc       __imp_?setMask@QWidget@@UAEXABVQRegion@@@Z 100082cc     qt-mt323:qt-mt323.dll
 0002:000002d0       __imp_?setMaximumSize@QWidget@@UAEXHH@Z 100082d0     qt-mt323:qt-mt323.dll
 0002:000002d4       __imp_?setMicroFocusHint@QWidget@@MAEXHHHH_NPAVQFont@@@Z 100082d4     qt-mt323:qt-mt323.dll
 0002:000002d8       __imp_?setMidLineWidth@QFrame@@UAEXH@Z 100082d8     qt-mt323:qt-mt323.dll
 0002:000002dc       __imp_?setMinimumSize@QWidget@@UAEXHH@Z 100082dc     qt-mt323:qt-mt323.dll
 0002:000002e0       __imp_?setMouseTracking@QWidget@@UAEX_N@Z 100082e0     qt-mt323:qt-mt323.dll
 0002:000002e4       __imp_?setName@QWidget@@UAEXPBD@Z 100082e4     qt-mt323:qt-mt323.dll
 0002:000002e8       __imp_?setNumCols@QTable@@UAEXH@Z 100082e8     qt-mt323:qt-mt323.dll
 0002:000002ec       __imp_?setNumRows@QTable@@UAEXH@Z 100082ec     qt-mt323:qt-mt323.dll
 0002:000002f0       __imp_?setPalette@QWidget@@UAEXABVQPalette@@@Z 100082f0     qt-mt323:qt-mt323.dll
 0002:000002f4       __imp_?setPaletteBackgroundColor@QWidget@@UAEXABVQColor@@@Z 100082f4     qt-mt323:qt-mt323.dll
 0002:000002f8       __imp_?setPaletteBackgroundPixmap@QWidget@@UAEXABVQPixmap@@@Z 100082f8     qt-mt323:qt-mt323.dll
 0002:000002fc       __imp_?setPixmap@QTable@@UAEXHHABVQPixmap@@@Z 100082fc     qt-mt323:qt-mt323.dll
 0002:00000300       __imp_?setProperty@QObject@@UAE_NPBDABVQVariant@@@Z 10008300     qt-mt323:qt-mt323.dll
 0002:00000304       __imp_?setReadOnly@QTable@@UAEX_N@Z 10008304     qt-mt323:qt-mt323.dll
 0002:00000308       __imp_?setResizePolicy@QScrollView@@UAEXW4ResizePolicy@1@@Z 10008308     qt-mt323:qt-mt323.dll
 0002:0000030c       __imp_?setResolution@QPaintDevice@@UAEXH@Z 1000830c     qt-mt323:qt-mt323.dll
 0002:00000310       __imp_?setRowHeight@QTable@@UAEXHH@Z 10008310     qt-mt323:qt-mt323.dll
 0002:00000314       __imp_?setRowMovingEnabled@QTable@@UAEX_N@Z 10008314     qt-mt323:qt-mt323.dll
 0002:00000318       __imp_?setRowReadOnly@QTable@@UAEXH_N@Z 10008318     qt-mt323:qt-mt323.dll
 0002:0000031c       __imp_?setRowStretchable@QTable@@UAEXH_N@Z 1000831c     qt-mt323:qt-mt323.dll
 0002:00000320       __imp_?setSelectionMode@QTable@@UAEXW4SelectionMode@1@@Z 10008320     qt-mt323:qt-mt323.dll
 0002:00000324       __imp_?setShowGrid@QTable@@UAEX_N@Z 10008324     qt-mt323:qt-mt323.dll
 0002:00000328       __imp_?setSizeIncrement@QWidget@@UAEXHH@Z 10008328     qt-mt323:qt-mt323.dll
 0002:0000032c       __imp_?setSizePolicy@QWidget@@UAEXVQSizePolicy@@@Z 1000832c     qt-mt323:qt-mt323.dll
 0002:00000330       __imp_?setSorting@QTable@@UAEX_N@Z 10008330     qt-mt323:qt-mt323.dll
 0002:00000334       __imp_?setText@QTable@@UAEXHHABVQString@@@Z 10008334     qt-mt323:qt-mt323.dll
 0002:00000338       __imp_?setTopMargin@QTable@@UAEXH@Z 10008338     qt-mt323:qt-mt323.dll
 0002:0000033c       __imp_?setUpdatesEnabled@QWidget@@UAEX_N@Z 1000833c     qt-mt323:qt-mt323.dll
 0002:00000340       __imp_?setVBarGeometry@QScrollView@@MAEXAAVQScrollBar@@HHHH@Z 10008340     qt-mt323:qt-mt323.dll
 0002:00000344       __imp_?setVScrollBarMode@QScrollView@@UAEXW4ScrollBarMode@1@@Z 10008344     qt-mt323:qt-mt323.dll
 0002:00000348       __imp_?setWFlags@QWidget@@MAEXI@Z 10008348     qt-mt323:qt-mt323.dll
 0002:0000034c       __imp_?setWState@QWidget@@MAEXI@Z 1000834c     qt-mt323:qt-mt323.dll
 0002:00000350       __imp_?show@QScrollView@@UAEXXZ 10008350     qt-mt323:qt-mt323.dll
 0002:00000354       __imp_?showColumn@QTable@@UAEXH@Z 10008354     qt-mt323:qt-mt323.dll
 0002:00000358       __imp_?showEvent@QTable@@MAEXPAVQShowEvent@@@Z 10008358     qt-mt323:qt-mt323.dll
 0002:0000035c       __imp_?showMaximized@QWidget@@UAEXXZ 1000835c     qt-mt323:qt-mt323.dll
 0002:00000360       __imp_?showMinimized@QWidget@@UAEXXZ 10008360     qt-mt323:qt-mt323.dll
 0002:00000364       __imp_?showNormal@QWidget@@UAEXXZ 10008364     qt-mt323:qt-mt323.dll
 0002:00000368       __imp_?showRow@QTable@@UAEXH@Z 10008368     qt-mt323:qt-mt323.dll
 0002:0000036c       __imp_?sizeHint@QTable@@UBE?AVQSize@@XZ 1000836c     qt-mt323:qt-mt323.dll
 0002:00000370       __imp_?sizePolicy@QWidget@@UBE?AVQSizePolicy@@XZ 10008370     qt-mt323:qt-mt323.dll
 0002:00000374       __imp_?sortColumn@QTable@@UAEXH_N0@Z 10008374     qt-mt323:qt-mt323.dll
 0002:00000378       __imp_?startDrag@QTable@@MAEXXZ 10008378     qt-mt323:qt-mt323.dll
 0002:0000037c       __imp_?styleChange@QScrollView@@UAEXAAVQStyle@@@Z 1000837c     qt-mt323:qt-mt323.dll
 0002:00000380       __imp_?swapCells@QTable@@UAEXHHHH@Z 10008380     qt-mt323:qt-mt323.dll
 0002:00000384       __imp_?swapColumns@QTable@@UAEXHH_N@Z 10008384     qt-mt323:qt-mt323.dll
 0002:00000388       __imp_?swapRows@QTable@@UAEXHH_N@Z 10008388     qt-mt323:qt-mt323.dll
 0002:0000038c       __imp_?tabletEvent@QWidget@@MAEXPAVQTabletEvent@@@Z 1000838c     qt-mt323:qt-mt323.dll
 0002:00000390       __imp_?takeItem@QTable@@UAEXPAVQTableItem@@@Z 10008390     qt-mt323:qt-mt323.dll
 0002:00000394       __imp_?text@QTable@@UBE?AVQString@@HH@Z 10008394     qt-mt323:qt-mt323.dll
 0002:00000398       __imp_?timerEvent@QObject@@MAEXPAVQTimerEvent@@@Z 10008398     qt-mt323:qt-mt323.dll
 0002:0000039c       __imp_?unsetCursor@QWidget@@UAEXXZ 1000839c     qt-mt323:qt-mt323.dll
 0002:000003a0       __imp_?updateMask@QWidget@@MAEXXZ 100083a0     qt-mt323:qt-mt323.dll
 0002:000003a4       __imp_?viewportContextMenuEvent@QScrollView@@MAEXPAVQContextMenuEvent@@@Z 100083a4     qt-mt323:qt-mt323.dll
 0002:000003a8       __imp_?viewportDragEnterEvent@QScrollView@@MAEXPAVQDragEnterEvent@@@Z 100083a8     qt-mt323:qt-mt323.dll
 0002:000003ac       __imp_?viewportDragLeaveEvent@QScrollView@@MAEXPAVQDragLeaveEvent@@@Z 100083ac     qt-mt323:qt-mt323.dll
 0002:000003b0       __imp_?viewportDragMoveEvent@QScrollView@@MAEXPAVQDragMoveEvent@@@Z 100083b0     qt-mt323:qt-mt323.dll
 0002:000003b4       __imp_?viewportDropEvent@QScrollView@@MAEXPAVQDropEvent@@@Z 100083b4     qt-mt323:qt-mt323.dll
 0002:000003b8       __imp_?viewportMouseDoubleClickEvent@QScrollView@@MAEXPAVQMouseEvent@@@Z 100083b8     qt-mt323:qt-mt323.dll
 0002:000003bc       __imp_?viewportMouseMoveEvent@QScrollView@@MAEXPAVQMouseEvent@@@Z 100083bc     qt-mt323:qt-mt323.dll
 0002:000003c0       __imp_?viewportMousePressEvent@QScrollView@@MAEXPAVQMouseEvent@@@Z 100083c0     qt-mt323:qt-mt323.dll
 0002:000003c4       __imp_?viewportMouseReleaseEvent@QScrollView@@MAEXPAVQMouseEvent@@@Z 100083c4     qt-mt323:qt-mt323.dll
 0002:000003c8       __imp_?viewportPaintEvent@QScrollView@@MAEXPAVQPaintEvent@@@Z 100083c8     qt-mt323:qt-mt323.dll
 0002:000003cc       __imp_?viewportResizeEvent@QTable@@MAEXPAVQResizeEvent@@@Z 100083cc     qt-mt323:qt-mt323.dll
 0002:000003d0       __imp_?viewportWheelEvent@QScrollView@@MAEXPAVQWheelEvent@@@Z 100083d0     qt-mt323:qt-mt323.dll
 0002:000003d4       __imp_?wheelEvent@QScrollView@@MAEXPAVQWheelEvent@@@Z 100083d4     qt-mt323:qt-mt323.dll
 0002:000003d8       __imp_?winEvent@QWidget@@MAE_NPAUtagMSG@@@Z 100083d8     qt-mt323:qt-mt323.dll
 0002:000003dc       __imp_?windowActivationChange@QTable@@MAEX_N@Z 100083dc     qt-mt323:qt-mt323.dll
 0002:000003e0       __imp_??0QString@@QAE@PBD@Z 100083e0     qt-mt323:qt-mt323.dll
 0002:000003e4       __imp_?ascii@QString@@QBEPBDXZ 100083e4     qt-mt323:qt-mt323.dll
 0002:000003e8       __imp_??8@YA_NABVQString@@PBD@Z 100083e8     qt-mt323:qt-mt323.dll
 0002:000003ec       __imp_??H@YA?BVQString@@ABV0@PBD@Z 100083ec     qt-mt323:qt-mt323.dll
 0002:000003f0       __imp_?inherits@QObject@@QBE_NPBD@Z 100083f0     qt-mt323:qt-mt323.dll
 0002:000003f4       __imp_?connect@QObject@@SA_NPBV1@PBD01@Z 100083f4     qt-mt323:qt-mt323.dll
 0002:000003f8       __imp_?viewport@QScrollView@@QBEPAVQWidget@@XZ 100083f8     qt-mt323:qt-mt323.dll
 0002:000003fc       __imp_??0QTableItem@@QAE@PAVQTable@@W4EditType@0@ABVQString@@@Z 100083fc     qt-mt323:qt-mt323.dll
 0002:00000400       __imp_??1QTableItem@@UAE@XZ 10008400     qt-mt323:qt-mt323.dll
 0002:00000404       __imp_?setContentFromEditor@QTableItem@@UAEXPAVQWidget@@@Z 10008404     qt-mt323:qt-mt323.dll
 0002:00000408       __imp_??0QComboBox@@QAE@PAVQWidget@@PBD@Z 10008408     qt-mt323:qt-mt323.dll
 0002:0000040c       __imp_??1QComboBox@@UAE@XZ 1000840c     qt-mt323:qt-mt323.dll
 0002:00000410       __imp_?insertItem@QComboBox@@QAEXABVQString@@H@Z 10008410     qt-mt323:qt-mt323.dll
 0002:00000414       __imp_?currentText@QComboBox@@QBE?AVQString@@XZ 10008414     qt-mt323:qt-mt323.dll
 0002:00000418       __imp_??4QDomNode@@QAEAAV0@ABV0@@Z 10008418     qt-mt323:qt-mt323.dll
 0002:0000041c       __imp_??1QDomNode@@UAE@XZ  1000841c     qt-mt323:qt-mt323.dll
 0002:00000420       __imp_?firstChild@QDomNode@@UBE?AV1@XZ 10008420     qt-mt323:qt-mt323.dll
 0002:00000424       __imp_?nextSibling@QDomNode@@UBE?AV1@XZ 10008424     qt-mt323:qt-mt323.dll
 0002:00000428       __imp_?isNull@QDomNode@@QBE_NXZ 10008428     qt-mt323:qt-mt323.dll
 0002:0000042c       __imp_?toElement@QDomNode@@QAE?AVQDomElement@@XZ 1000842c     qt-mt323:qt-mt323.dll
 0002:00000430       __imp_??0QDomDocument@@QAE@ABVQString@@@Z 10008430     qt-mt323:qt-mt323.dll
 0002:00000434       __imp_??1QDomDocument@@UAE@XZ 10008434     qt-mt323:qt-mt323.dll
 0002:00000438       __imp_?documentElement@QDomDocument@@QBE?AVQDomElement@@XZ 10008438     qt-mt323:qt-mt323.dll
 0002:0000043c       __imp_?setContent@QDomDocument@@QAE_NPAVQIODevice@@PAVQString@@PAH2@Z 1000843c     qt-mt323:qt-mt323.dll
 0002:00000440       __imp_??1QDomElement@@UAE@XZ 10008440     qt-mt323:qt-mt323.dll
 0002:00000444       __imp_?attribute@QDomElement@@QBE?AVQString@@ABV2@0@Z 10008444     qt-mt323:qt-mt323.dll
 0002:00000448       __imp_??0QFile@@QAE@ABVQString@@@Z 10008448     qt-mt323:qt-mt323.dll
 0002:0000044c       __imp_??1QFile@@UAE@XZ     1000844c     qt-mt323:qt-mt323.dll
 0002:00000450       __imp_?open@QFile@@UAE_NH@Z 10008450     qt-mt323:qt-mt323.dll
 0002:00000454       __imp_?close@QFile@@UAEXXZ 10008454     qt-mt323:qt-mt323.dll
 0002:00000458       __imp_?alignment@QTableItem@@UBEHXZ 10008458     qt-mt323:qt-mt323.dll
 0002:0000045c       __imp_?className@QComboBox@@UBEPBDXZ 1000845c     qt-mt323:qt-mt323.dll
 0002:00000460       __imp_?contextMenuEvent@QWidget@@MAEXPAVQContextMenuEvent@@@Z 10008460     qt-mt323:qt-mt323.dll
 0002:00000464       __imp_?eventFilter@QComboBox@@UAE_NPAVQObject@@PAVQEvent@@@Z 10008464     qt-mt323:qt-mt323.dll
 0002:00000468       __imp_?focusInEvent@QComboBox@@MAEXPAVQFocusEvent@@@Z 10008468     qt-mt323:qt-mt323.dll
 0002:0000046c       __imp_?focusNextPrevChild@QWidget@@MAE_N_N@Z 1000846c     qt-mt323:qt-mt323.dll
 0002:00000470       __imp_?focusOutEvent@QComboBox@@MAEXPAVQFocusEvent@@@Z 10008470     qt-mt323:qt-mt323.dll
 0002:00000474       __imp_?fontChange@QWidget@@MAEXABVQFont@@@Z 10008474     qt-mt323:qt-mt323.dll
 0002:00000478       __imp_?key@QTableItem@@UBE?AVQString@@XZ 10008478     qt-mt323:qt-mt323.dll
 0002:0000047c       __imp_?keyPressEvent@QComboBox@@MAEXPAVQKeyEvent@@@Z 1000847c     qt-mt323:qt-mt323.dll
 0002:00000480       __imp_?metaObject@QComboBox@@UBEPAVQMetaObject@@XZ 10008480     qt-mt323:qt-mt323.dll
 0002:00000484       __imp_?minimumSizeHint@QWidget@@UBE?AVQSize@@XZ 10008484     qt-mt323:qt-mt323.dll
 0002:00000488       __imp_?mouseDoubleClickEvent@QComboBox@@MAEXPAVQMouseEvent@@@Z 10008488     qt-mt323:qt-mt323.dll
 0002:0000048c       __imp_?mouseMoveEvent@QComboBox@@MAEXPAVQMouseEvent@@@Z 1000848c     qt-mt323:qt-mt323.dll
 0002:00000490       __imp_?mousePressEvent@QComboBox@@MAEXPAVQMouseEvent@@@Z 10008490     qt-mt323:qt-mt323.dll
 0002:00000494       __imp_?mouseReleaseEvent@QComboBox@@MAEXPAVQMouseEvent@@@Z 10008494     qt-mt323:qt-mt323.dll
 0002:00000498       __imp_?paint@QTableItem@@UAEXPAVQPainter@@ABVQColorGroup@@ABVQRect@@_N@Z 10008498     qt-mt323:qt-mt323.dll
 0002:0000049c       __imp_?paintEvent@QComboBox@@MAEXPAVQPaintEvent@@@Z 1000849c     qt-mt323:qt-mt323.dll
 0002:000004a0       __imp_?pixmap@QTableItem@@UBE?AVQPixmap@@XZ 100084a0     qt-mt323:qt-mt323.dll
 0002:000004a4       __imp_?popup@QComboBox@@UAEXXZ 100084a4     qt-mt323:qt-mt323.dll
 0002:000004a8       __imp_?qt_cast@QComboBox@@UAEPAXPBD@Z 100084a8     qt-mt323:qt-mt323.dll
 0002:000004ac       __imp_?qt_emit@QComboBox@@UAE_NHPAUQUObject@@@Z 100084ac     qt-mt323:qt-mt323.dll
 0002:000004b0       __imp_?qt_invoke@QComboBox@@UAE_NHPAUQUObject@@@Z 100084b0     qt-mt323:qt-mt323.dll
 0002:000004b4       __imp_?qt_property@QComboBox@@UAE_NHHPAVQVariant@@@Z 100084b4     qt-mt323:qt-mt323.dll
 0002:000004b8       __imp_?removeChild@QObject@@UAEXPAV1@@Z 100084b8     qt-mt323:qt-mt323.dll
 0002:000004bc       __imp_?resize@QWidget@@UAEXHH@Z 100084bc     qt-mt323:qt-mt323.dll
 0002:000004c0       __imp_?resizeEvent@QComboBox@@MAEXPAVQResizeEvent@@@Z 100084c0     qt-mt323:qt-mt323.dll
 0002:000004c4       __imp_?rtti@QTableItem@@UBEHXZ 100084c4     qt-mt323:qt-mt323.dll
 0002:000004c8       __imp_?setAutoCompletion@QComboBox@@UAEX_N@Z 100084c8     qt-mt323:qt-mt323.dll
 0002:000004cc       __imp_?setAutoResize@QComboBox@@UAEX_N@Z 100084cc     qt-mt323:qt-mt323.dll
 0002:000004d0       __imp_?setCol@QTableItem@@UAEXH@Z 100084d0     qt-mt323:qt-mt323.dll
 0002:000004d4       __imp_?setCurrentItem@QComboBox@@UAEXH@Z 100084d4     qt-mt323:qt-mt323.dll
 0002:000004d8       __imp_?setCurrentText@QComboBox@@UAEXABVQString@@@Z 100084d8     qt-mt323:qt-mt323.dll
 0002:000004dc       __imp_?setEditText@QComboBox@@UAEXABVQString@@@Z 100084dc     qt-mt323:qt-mt323.dll
 0002:000004e0       __imp_?setEnabled@QComboBox@@UAEX_N@Z 100084e0     qt-mt323:qt-mt323.dll
 0002:000004e4       __imp_?setEnabled@QTableItem@@UAEX_N@Z 100084e4     qt-mt323:qt-mt323.dll
 0002:000004e8       __imp_?setFont@QComboBox@@UAEXABVQFont@@@Z 100084e8     qt-mt323:qt-mt323.dll
 0002:000004ec       __imp_?setInsertionPolicy@QComboBox@@UAEXW4Policy@1@@Z 100084ec     qt-mt323:qt-mt323.dll
 0002:000004f0       __imp_?setLineEdit@QComboBox@@UAEXPAVQLineEdit@@@Z 100084f0     qt-mt323:qt-mt323.dll
 0002:000004f4       __imp_?setListBox@QComboBox@@UAEXPAVQListBox@@@Z 100084f4     qt-mt323:qt-mt323.dll
 0002:000004f8       __imp_?setMaxCount@QComboBox@@UAEXH@Z 100084f8     qt-mt323:qt-mt323.dll
 0002:000004fc       __imp_?setPalette@QComboBox@@UAEXABVQPalette@@@Z 100084fc     qt-mt323:qt-mt323.dll
 0002:00000500       __imp_?setPixmap@QTableItem@@UAEXABVQPixmap@@@Z 10008500     qt-mt323:qt-mt323.dll
 0002:00000504       __imp_?setReplaceable@QTableItem@@UAEX_N@Z 10008504     qt-mt323:qt-mt323.dll
 0002:00000508       __imp_?setRow@QTableItem@@UAEXH@Z 10008508     qt-mt323:qt-mt323.dll
 0002:0000050c       __imp_?setSizeLimit@QComboBox@@UAEXH@Z 1000850c     qt-mt323:qt-mt323.dll
 0002:00000510       __imp_?setSpan@QTableItem@@UAEXHH@Z 10008510     qt-mt323:qt-mt323.dll
 0002:00000514       __imp_?setText@QTableItem@@UAEXABVQString@@@Z 10008514     qt-mt323:qt-mt323.dll
 0002:00000518       __imp_?setValidator@QComboBox@@UAEXPBVQValidator@@@Z 10008518     qt-mt323:qt-mt323.dll
 0002:0000051c       __imp_?setWordWrap@QTableItem@@UAEX_N@Z 1000851c     qt-mt323:qt-mt323.dll
 0002:00000520       __imp_?show@QWidget@@UAEXXZ 10008520     qt-mt323:qt-mt323.dll
 0002:00000524       __imp_?showEvent@QWidget@@MAEXPAVQShowEvent@@@Z 10008524     qt-mt323:qt-mt323.dll
 0002:00000528       __imp_?sizeHint@QComboBox@@UBE?AVQSize@@XZ 10008528     qt-mt323:qt-mt323.dll
 0002:0000052c       __imp_?sizeHint@QTableItem@@UBE?AVQSize@@XZ 1000852c     qt-mt323:qt-mt323.dll
 0002:00000530       __imp_?styleChange@QComboBox@@MAEXAAVQStyle@@@Z 10008530     qt-mt323:qt-mt323.dll
 0002:00000534       __imp_?text@QTableItem@@UBE?AVQString@@XZ 10008534     qt-mt323:qt-mt323.dll
 0002:00000538       __imp_?updateMask@QComboBox@@MAEXXZ 10008538     qt-mt323:qt-mt323.dll
 0002:0000053c       __imp_?wheelEvent@QComboBox@@MAEXPAVQWheelEvent@@@Z 1000853c     qt-mt323:qt-mt323.dll
 0002:00000540       __imp_?windowActivationChange@QWidget@@MAEX_N@Z 10008540     qt-mt323:qt-mt323.dll
 0002:00000544       __imp_?null@QString@@2V1@A 10008544     qt-mt323:qt-mt323.dll
 0002:00000548       __imp_??6?$QValueList@VQString@@@@QAEAAV0@ABVQString@@@Z 10008548     qt-mt323:qt-mt323.dll
 0002:0000054c       __imp_??0QStringList@@QAE@XZ 1000854c     qt-mt323:qt-mt323.dll
 0002:00000550       __imp_??1QStringList@@QAE@XZ 10008550     qt-mt323:qt-mt323.dll
 0002:00000554       __imp_??0QPixmap@@QAE@QAPBD@Z 10008554     qt-mt323:qt-mt323.dll
 0002:00000558       __imp_?eventFilter@QObject@@UAE_NPAV1@PAVQEvent@@@Z 10008558     qt-mt323:qt-mt323.dll
 0002:0000055c       __imp_?focusInEvent@QWidget@@MAEXPAVQFocusEvent@@@Z 1000855c     qt-mt323:qt-mt323.dll
 0002:00000560       __imp_?focusOutEvent@QWidget@@MAEXPAVQFocusEvent@@@Z 10008560     qt-mt323:qt-mt323.dll
 0002:00000564       __imp_?keyPressEvent@QWidget@@MAEXPAVQKeyEvent@@@Z 10008564     qt-mt323:qt-mt323.dll
 0002:00000568       __imp_?mouseDoubleClickEvent@QWidget@@MAEXPAVQMouseEvent@@@Z 10008568     qt-mt323:qt-mt323.dll
 0002:0000056c       __imp_?mouseMoveEvent@QWidget@@MAEXPAVQMouseEvent@@@Z 1000856c     qt-mt323:qt-mt323.dll
 0002:00000570       __imp_?mousePressEvent@QWidget@@MAEXPAVQMouseEvent@@@Z 10008570     qt-mt323:qt-mt323.dll
 0002:00000574       __imp_?mouseReleaseEvent@QWidget@@MAEXPAVQMouseEvent@@@Z 10008574     qt-mt323:qt-mt323.dll
 0002:00000578       __imp_?paintEvent@QWidget@@MAEXPAVQPaintEvent@@@Z 10008578     qt-mt323:qt-mt323.dll
 0002:0000057c       __imp_?resizeEvent@QWidget@@MAEXPAVQResizeEvent@@@Z 1000857c     qt-mt323:qt-mt323.dll
 0002:00000580       __imp_?setEnabled@QWidget@@UAEX_N@Z 10008580     qt-mt323:qt-mt323.dll
 0002:00000584       __imp_?sizeHint@QWidget@@UBE?AVQSize@@XZ 10008584     qt-mt323:qt-mt323.dll
 0002:00000588       __imp_?styleChange@QWidget@@MAEXAAVQStyle@@@Z 10008588     qt-mt323:qt-mt323.dll
 0002:0000058c       __imp_?wheelEvent@QWidget@@MAEXPAVQWheelEvent@@@Z 1000858c     qt-mt323:qt-mt323.dll
 0002:00000590       __imp_??0QString@@QAE@ABV0@@Z 10008590     qt-mt323:qt-mt323.dll
 0002:00000594       __imp_??4QString@@QAEAAV0@PBD@Z 10008594     qt-mt323:qt-mt323.dll
 0002:00000598       __imp_?arg@QString@@QBE?AV1@ABV1@H@Z 10008598     qt-mt323:qt-mt323.dll
 0002:0000059c       __imp_??8@YA_NABVQString@@0@Z 1000859c     qt-mt323:qt-mt323.dll
 0002:000005a0       __imp_??H@YA?BVQString@@PBDABV0@@Z 100085a0     qt-mt323:qt-mt323.dll
 0002:000005a4       __imp_??0QGList@@IAE@XZ    100085a4     qt-mt323:qt-mt323.dll
 0002:000005a8       __imp_?cmd@QPaintDevice@@MAE_NHPAVQPainter@@PATQPDevCmdParam@@@Z 100085a8     qt-mt323:qt-mt323.dll
 0002:000005ac       __imp_??1QGList@@MAE@XZ    100085ac     qt-mt323:qt-mt323.dll
 0002:000005b0       __imp_?append@QGList@@IAEXPAX@Z 100085b0     qt-mt323:qt-mt323.dll
 0002:000005b4       __imp_?clear@QGList@@MAEXXZ 100085b4     qt-mt323:qt-mt323.dll
 0002:000005b8       __imp_??0QWidget@@QAE@PAV0@PBDI@Z 100085b8     qt-mt323:qt-mt323.dll
 0002:000005bc       __imp_??1QWidget@@UAE@XZ   100085bc     qt-mt323:qt-mt323.dll
 0002:000005c0       __imp_?rect@QWidget@@QBE?AVQRect@@XZ 100085c0     qt-mt323:qt-mt323.dll
 0002:000005c4       __imp_?information@QMessageBox@@SAHPAVQWidget@@ABVQString@@1111HH@Z 100085c4     qt-mt323:qt-mt323.dll
 0002:000005c8       __imp_??0QKeySequence@@QAE@H@Z 100085c8     qt-mt323:qt-mt323.dll
 0002:000005cc       __imp_??1QPixmap@@UAE@XZ   100085cc     qt-mt323:qt-mt323.dll
 0002:000005d0       __imp_??0QIconSet@@QAE@ABVQPixmap@@W4Size@0@@Z 100085d0     qt-mt323:qt-mt323.dll
 0002:000005d4       __imp_??1QIconSet@@UAE@XZ  100085d4     qt-mt323:qt-mt323.dll
 0002:000005d8       __imp_??0QAction@@QAE@ABVQString@@ABVQIconSet@@0VQKeySequence@@PAVQObject@@PBD_N@Z 100085d8     qt-mt323:qt-mt323.dll
 0002:000005dc       __imp_??1QAction@@UAE@XZ   100085dc     qt-mt323:qt-mt323.dll
 0002:000005e0       __imp_??1?$QPtrList@VQDockWindow@@@@UAE@XZ 100085e0     qt-mt323:qt-mt323.dll
 0002:000005e4       __imp_??0QToolBar@@QAE@PAVQMainWindow@@PBD@Z 100085e4     qt-mt323:qt-mt323.dll
 0002:000005e8       __imp_??1QToolBar@@UAE@XZ  100085e8     qt-mt323:qt-mt323.dll
 0002:000005ec       __imp_??9QDateTime@@QBE_NABV0@@Z 100085ec     qt-mt323:qt-mt323.dll
 0002:000005f0       __imp_??0QFileInfo@@QAE@ABVQString@@@Z 100085f0     qt-mt323:qt-mt323.dll
 0002:000005f4       __imp_??1QFileInfo@@QAE@XZ 100085f4     qt-mt323:qt-mt323.dll
 0002:000005f8       __imp_?lastModified@QFileInfo@@QBE?AVQDateTime@@XZ 100085f8     qt-mt323:qt-mt323.dll
 0002:000005fc       __imp_??0QGuardedPtrPrivate@@QAE@PAVQObject@@@Z 100085fc     qt-mt323:qt-mt323.dll
 0002:00000600       __imp_??1QGuardedPtrPrivate@@UAE@XZ 10008600     qt-mt323:qt-mt323.dll
 0002:00000604       __imp_?reconnect@QGuardedPtrPrivate@@QAEXPAVQObject@@@Z 10008604     qt-mt323:qt-mt323.dll
 0002:00000608       __imp_??0QPopupMenu@@QAE@PAVQWidget@@PBD@Z 10008608     qt-mt323:qt-mt323.dll
 0002:0000060c       __imp_??1QPopupMenu@@UAE@XZ 1000860c     qt-mt323:qt-mt323.dll
 0002:00000610       __imp_?look_string@QGDict@@QAEPAXABVQString@@PAXH@Z 10008610     qt-mt323:qt-mt323.dll
 0002:00000614       __imp_??0QGDict@@IAE@IW4KeyType@0@_N1@Z 10008614     qt-mt323:qt-mt323.dll
 0002:00000618       __imp_??1QGDict@@MAE@XZ    10008618     qt-mt323:qt-mt323.dll
 0002:0000061c       __imp_?clear@QGDict@@MAEXXZ 1000861c     qt-mt323:qt-mt323.dll
 0002:00000620       __imp_?activateItemAt@QPopupMenu@@UAEXH@Z 10008620     qt-mt323:qt-mt323.dll
 0002:00000624       __imp_?addTo@QAction@@UAE_NPAVQWidget@@@Z 10008624     qt-mt323:qt-mt323.dll
 0002:00000628       __imp_?addedTo@QAction@@MAEXHPAVQPopupMenu@@@Z 10008628     qt-mt323:qt-mt323.dll
 0002:0000062c       __imp_?addedTo@QAction@@MAEXPAVQWidget@@0@Z 1000862c     qt-mt323:qt-mt323.dll
 0002:00000630       __imp_?className@QAction@@UBEPBDXZ 10008630     qt-mt323:qt-mt323.dll
 0002:00000634       __imp_?className@QGuardedPtrPrivate@@UBEPBDXZ 10008634     qt-mt323:qt-mt323.dll
 0002:00000638       __imp_?className@QPopupMenu@@UBEPBDXZ 10008638     qt-mt323:qt-mt323.dll
 0002:0000063c       __imp_?className@QToolBar@@UBEPBDXZ 1000863c     qt-mt323:qt-mt323.dll
 0002:00000640       __imp_?className@QWidget@@UBEPBDXZ 10008640     qt-mt323:qt-mt323.dll
 0002:00000644       __imp_?clear@?$QPtrList@VQDockWindow@@@@UAEXXZ 10008644     qt-mt323:qt-mt323.dll
 0002:00000648       __imp_?clear@QToolBar@@UAEXXZ 10008648     qt-mt323:qt-mt323.dll
 0002:0000064c       __imp_?closeEvent@QPopupMenu@@MAEXPAVQCloseEvent@@@Z 1000864c     qt-mt323:qt-mt323.dll
 0002:00000650       __imp_?compareItems@QGList@@MAEHPAX0@Z 10008650     qt-mt323:qt-mt323.dll
 0002:00000654       __imp_?contextMenuEvent@QDockWindow@@MAEXPAVQContextMenuEvent@@@Z 10008654     qt-mt323:qt-mt323.dll
 0002:00000658       __imp_?count@?$QPtrList@VQDockWindow@@@@UBEIXZ 10008658     qt-mt323:qt-mt323.dll
 0002:0000065c       __imp_?customWhatsThis@QPopupMenu@@UBE_NXZ 1000865c     qt-mt323:qt-mt323.dll
 0002:00000660       __imp_?deleteItem@?$QPtrList@VQDockWindow@@@@EAEXPAX@Z 10008660     qt-mt323:qt-mt323.dll
 0002:00000664       __imp_?dock@QDockWindow@@UAEXXZ 10008664     qt-mt323:qt-mt323.dll
 0002:00000668       __imp_?drawContents@QDockWindow@@MAEXPAVQPainter@@@Z 10008668     qt-mt323:qt-mt323.dll
 0002:0000066c       __imp_?drawContents@QPopupMenu@@MAEXPAVQPainter@@@Z 1000866c     qt-mt323:qt-mt323.dll
 0002:00000670       __imp_?drawFrame@QDockWindow@@MAEXPAVQPainter@@@Z 10008670     qt-mt323:qt-mt323.dll
 0002:00000674       __imp_?enabledChange@QPopupMenu@@MAEX_N@Z 10008674     qt-mt323:qt-mt323.dll
 0002:00000678       __imp_?event@QObject@@UAE_NPAVQEvent@@@Z 10008678     qt-mt323:qt-mt323.dll
 0002:0000067c       __imp_?event@QToolBar@@UAE_NPAVQEvent@@@Z 1000867c     qt-mt323:qt-mt323.dll
 0002:00000680       __imp_?eventFilter@QDockWindow@@UAE_NPAVQObject@@PAVQEvent@@@Z 10008680     qt-mt323:qt-mt323.dll
 0002:00000684       __imp_?focusInEvent@QPopupMenu@@MAEXPAVQFocusEvent@@@Z 10008684     qt-mt323:qt-mt323.dll
 0002:00000688       __imp_?focusNextPrevChild@QPopupMenu@@MAE_N_N@Z 10008688     qt-mt323:qt-mt323.dll
 0002:0000068c       __imp_?focusOutEvent@QPopupMenu@@MAEXPAVQFocusEvent@@@Z 1000868c     qt-mt323:qt-mt323.dll
 0002:00000690       __imp_?frameChanged@QFrame@@MAEXXZ 10008690     qt-mt323:qt-mt323.dll
 0002:00000694       __imp_?frameChanged@QPopupMenu@@EAEXXZ 10008694     qt-mt323:qt-mt323.dll
 0002:00000698       __imp_?hide@QPopupMenu@@UAEXXZ 10008698     qt-mt323:qt-mt323.dll
 0002:0000069c       __imp_?hide@QToolBar@@UAEXXZ 1000869c     qt-mt323:qt-mt323.dll
 0002:000006a0       __imp_?hideEvent@QDockWindow@@MAEXPAVQHideEvent@@@Z 100086a0     qt-mt323:qt-mt323.dll
 0002:000006a4       __imp_?keyPressEvent@QPopupMenu@@MAEXPAVQKeyEvent@@@Z 100086a4     qt-mt323:qt-mt323.dll
 0002:000006a8       __imp_?leaveEvent@QPopupMenu@@MAEXPAVQEvent@@@Z 100086a8     qt-mt323:qt-mt323.dll
 0002:000006ac       __imp_?menuContentsChanged@QPopupMenu@@EAEXXZ 100086ac     qt-mt323:qt-mt323.dll
 0002:000006b0       __imp_?menuDelPopup@QPopupMenu@@EAEXPAV1@@Z 100086b0     qt-mt323:qt-mt323.dll
 0002:000006b4       __imp_?menuInsPopup@QPopupMenu@@EAEXPAV1@@Z 100086b4     qt-mt323:qt-mt323.dll
 0002:000006b8       __imp_?menuStateChanged@QPopupMenu@@EAEXXZ 100086b8     qt-mt323:qt-mt323.dll
 0002:000006bc       __imp_?metaObject@QAction@@UBEPAVQMetaObject@@XZ 100086bc     qt-mt323:qt-mt323.dll
 0002:000006c0       __imp_?metaObject@QGuardedPtrPrivate@@UBEPAVQMetaObject@@XZ 100086c0     qt-mt323:qt-mt323.dll
 0002:000006c4       __imp_?metaObject@QPopupMenu@@UBEPAVQMetaObject@@XZ 100086c4     qt-mt323:qt-mt323.dll
 0002:000006c8       __imp_?metaObject@QToolBar@@UBEPAVQMetaObject@@XZ 100086c8     qt-mt323:qt-mt323.dll
 0002:000006cc       __imp_?metaObject@QWidget@@UBEPAVQMetaObject@@XZ 100086cc     qt-mt323:qt-mt323.dll
 0002:000006d0       __imp_?minimumSizeHint@QToolBar@@UBE?AVQSize@@XZ 100086d0     qt-mt323:qt-mt323.dll
 0002:000006d4       __imp_?mouseMoveEvent@QPopupMenu@@MAEXPAVQMouseEvent@@@Z 100086d4     qt-mt323:qt-mt323.dll
 0002:000006d8       __imp_?mousePressEvent@QPopupMenu@@MAEXPAVQMouseEvent@@@Z 100086d8     qt-mt323:qt-mt323.dll
 0002:000006dc       __imp_?mouseReleaseEvent@QPopupMenu@@MAEXPAVQMouseEvent@@@Z 100086dc     qt-mt323:qt-mt323.dll
 0002:000006e0       __imp_?newItem@QPtrCollection@@MAEPAXPAX@Z 100086e0     qt-mt323:qt-mt323.dll
 0002:000006e4       __imp_?paintEvent@QFrame@@MAEXPAVQPaintEvent@@@Z 100086e4     qt-mt323:qt-mt323.dll
 0002:000006e8       __imp_?paintEvent@QPopupMenu@@MAEXPAVQPaintEvent@@@Z 100086e8     qt-mt323:qt-mt323.dll
 0002:000006ec       __imp_?qt_cast@QAction@@UAEPAXPBD@Z 100086ec     qt-mt323:qt-mt323.dll
 0002:000006f0       __imp_?qt_cast@QGuardedPtrPrivate@@UAEPAXPBD@Z 100086f0     qt-mt323:qt-mt323.dll
 0002:000006f4       __imp_?qt_cast@QPopupMenu@@UAEPAXPBD@Z 100086f4     qt-mt323:qt-mt323.dll
 0002:000006f8       __imp_?qt_cast@QToolBar@@UAEPAXPBD@Z 100086f8     qt-mt323:qt-mt323.dll
 0002:000006fc       __imp_?qt_cast@QWidget@@UAEPAXPBD@Z 100086fc     qt-mt323:qt-mt323.dll
 0002:00000700       __imp_?qt_emit@QAction@@UAE_NHPAUQUObject@@@Z 10008700     qt-mt323:qt-mt323.dll
 0002:00000704       __imp_?qt_emit@QGuardedPtrPrivate@@UAE_NHPAUQUObject@@@Z 10008704     qt-mt323:qt-mt323.dll
 0002:00000708       __imp_?qt_emit@QPopupMenu@@UAE_NHPAUQUObject@@@Z 10008708     qt-mt323:qt-mt323.dll
 0002:0000070c       __imp_?qt_emit@QToolBar@@UAE_NHPAUQUObject@@@Z 1000870c     qt-mt323:qt-mt323.dll
 0002:00000710       __imp_?qt_emit@QWidget@@UAE_NHPAUQUObject@@@Z 10008710     qt-mt323:qt-mt323.dll
 0002:00000714       __imp_?qt_invoke@QAction@@UAE_NHPAUQUObject@@@Z 10008714     qt-mt323:qt-mt323.dll
 0002:00000718       __imp_?qt_invoke@QGuardedPtrPrivate@@UAE_NHPAUQUObject@@@Z 10008718     qt-mt323:qt-mt323.dll
 0002:0000071c       __imp_?qt_invoke@QPopupMenu@@UAE_NHPAUQUObject@@@Z 1000871c     qt-mt323:qt-mt323.dll
 0002:00000720       __imp_?qt_invoke@QToolBar@@UAE_NHPAUQUObject@@@Z 10008720     qt-mt323:qt-mt323.dll
 0002:00000724       __imp_?qt_invoke@QWidget@@UAE_NHPAUQUObject@@@Z 10008724     qt-mt323:qt-mt323.dll
 0002:00000728       __imp_?qt_property@QAction@@UAE_NHHPAVQVariant@@@Z 10008728     qt-mt323:qt-mt323.dll
 0002:0000072c       __imp_?qt_property@QGuardedPtrPrivate@@UAE_NHHPAVQVariant@@@Z 1000872c     qt-mt323:qt-mt323.dll
 0002:00000730       __imp_?qt_property@QPopupMenu@@UAE_NHHPAVQVariant@@@Z 10008730     qt-mt323:qt-mt323.dll
 0002:00000734       __imp_?qt_property@QToolBar@@UAE_NHHPAVQVariant@@@Z 10008734     qt-mt323:qt-mt323.dll
 0002:00000738       __imp_?qt_property@QWidget@@UAE_NHHPAVQVariant@@@Z 10008738     qt-mt323:qt-mt323.dll
 0002:0000073c       __imp_?read@QGDict@@MAEAAVQDataStream@@AAV2@AAPAX@Z 1000873c     qt-mt323:qt-mt323.dll
 0002:00000740       __imp_?read@QGList@@MAEAAVQDataStream@@AAV2@AAPAX@Z 10008740     qt-mt323:qt-mt323.dll
 0002:00000744       __imp_?removeFrom@QAction@@UAE_NPAVQWidget@@@Z 10008744     qt-mt323:qt-mt323.dll
 0002:00000748       __imp_?resizeEvent@QFrame@@MAEXPAVQResizeEvent@@@Z 10008748     qt-mt323:qt-mt323.dll
 0002:0000074c       __imp_?resizeEvent@QToolBar@@MAEXPAVQResizeEvent@@@Z 1000874c     qt-mt323:qt-mt323.dll
 0002:00000750       __imp_?setAccel@QAction@@UAEXABVQKeySequence@@@Z 10008750     qt-mt323:qt-mt323.dll
 0002:00000754       __imp_?setActiveItem@QPopupMenu@@UAEXH@Z 10008754     qt-mt323:qt-mt323.dll
 0002:00000758       __imp_?setCaption@QDockWindow@@UAEXABVQString@@@Z 10008758     qt-mt323:qt-mt323.dll
 0002:0000075c       __imp_?setCheckable@QPopupMenu@@UAEX_N@Z 1000875c     qt-mt323:qt-mt323.dll
 0002:00000760       __imp_?setCloseMode@QDockWindow@@UAEXH@Z 10008760     qt-mt323:qt-mt323.dll
 0002:00000764       __imp_?setEnabled@QAction@@UAEX_N@Z 10008764     qt-mt323:qt-mt323.dll
 0002:00000768       __imp_?setFirstItemActive@QPopupMenu@@EAEXXZ 10008768     qt-mt323:qt-mt323.dll
 0002:0000076c       __imp_?setFixedExtentHeight@QDockWindow@@UAEXH@Z 1000876c     qt-mt323:qt-mt323.dll
 0002:00000770       __imp_?setFixedExtentWidth@QDockWindow@@UAEXH@Z 10008770     qt-mt323:qt-mt323.dll
 0002:00000774       __imp_?setFont@QPopupMenu@@UAEXABVQFont@@@Z 10008774     qt-mt323:qt-mt323.dll
 0002:00000778       __imp_?setHorizontallyStretchable@QDockWindow@@UAEX_N@Z 10008778     qt-mt323:qt-mt323.dll
 0002:0000077c       __imp_?setIconSet@QAction@@UAEXABVQIconSet@@@Z 1000877c     qt-mt323:qt-mt323.dll
 0002:00000780       __imp_?setId@QMenuData@@UAEXHH@Z 10008780     qt-mt323:qt-mt323.dll
 0002:00000784       __imp_?setLabel@QToolBar@@UAEXABVQString@@@Z 10008784     qt-mt323:qt-mt323.dll
 0002:00000788       __imp_?setMenuText@QAction@@UAEXABVQString@@@Z 10008788     qt-mt323:qt-mt323.dll
 0002:0000078c       __imp_?setMinimumSize@QToolBar@@UAEXHH@Z 1000878c     qt-mt323:qt-mt323.dll
 0002:00000790       __imp_?setMovingEnabled@QDockWindow@@UAEX_N@Z 10008790     qt-mt323:qt-mt323.dll
 0002:00000794       __imp_?setName@QObject@@UAEXPBD@Z 10008794     qt-mt323:qt-mt323.dll
 0002:00000798       __imp_?setNewLine@QDockWindow@@UAEX_N@Z 10008798     qt-mt323:qt-mt323.dll
 0002:0000079c       __imp_?setOffset@QDockWindow@@UAEXH@Z 1000879c     qt-mt323:qt-mt323.dll
 0002:000007a0       __imp_?setOn@QAction@@UAEX_N@Z 100087a0     qt-mt323:qt-mt323.dll
 0002:000007a4       __imp_?setOpaqueMoving@QDockWindow@@UAEX_N@Z 100087a4     qt-mt323:qt-mt323.dll
 0002:000007a8       __imp_?setOrientation@QToolBar@@UAEXW4Orientation@Qt@@@Z 100087a8     qt-mt323:qt-mt323.dll
 0002:000007ac       __imp_?setResizeEnabled@QDockWindow@@UAEX_N@Z 100087ac     qt-mt323:qt-mt323.dll
 0002:000007b0       __imp_?setStatusTip@QAction@@UAEXABVQString@@@Z 100087b0     qt-mt323:qt-mt323.dll
 0002:000007b4       __imp_?setStretchableWidget@QToolBar@@UAEXPAVQWidget@@@Z 100087b4     qt-mt323:qt-mt323.dll
 0002:000007b8       __imp_?setText@QAction@@UAEXABVQString@@@Z 100087b8     qt-mt323:qt-mt323.dll
 0002:000007bc       __imp_?setToggleAction@QAction@@UAEX_N@Z 100087bc     qt-mt323:qt-mt323.dll
 0002:000007c0       __imp_?setToolTip@QAction@@UAEXABVQString@@@Z 100087c0     qt-mt323:qt-mt323.dll
 0002:000007c4       __imp_?setVerticallyStretchable@QDockWindow@@UAEX_N@Z 100087c4     qt-mt323:qt-mt323.dll
 0002:000007c8       __imp_?setWhatsThis@QAction@@UAEXABVQString@@@Z 100087c8     qt-mt323:qt-mt323.dll
 0002:000007cc       __imp_?setWidget@QDockWindow@@UAEXPAVQWidget@@@Z 100087cc     qt-mt323:qt-mt323.dll
 0002:000007d0       __imp_?show@QPopupMenu@@UAEXXZ 100087d0     qt-mt323:qt-mt323.dll
 0002:000007d4       __imp_?show@QToolBar@@UAEXXZ 100087d4     qt-mt323:qt-mt323.dll
 0002:000007d8       __imp_?showEvent@QDockWindow@@MAEXPAVQShowEvent@@@Z 100087d8     qt-mt323:qt-mt323.dll
 0002:000007dc       __imp_?sizeHint@QDockWindow@@UBE?AVQSize@@XZ 100087dc     qt-mt323:qt-mt323.dll
 0002:000007e0       __imp_?sizeHint@QPopupMenu@@UBE?AVQSize@@XZ 100087e0     qt-mt323:qt-mt323.dll
 0002:000007e4       __imp_?styleChange@QPopupMenu@@MAEXAAVQStyle@@@Z 100087e4     qt-mt323:qt-mt323.dll
 0002:000007e8       __imp_?styleChange@QToolBar@@MAEXAAVQStyle@@@Z 100087e8     qt-mt323:qt-mt323.dll
 0002:000007ec       __imp_?timerEvent@QPopupMenu@@MAEXPAVQTimerEvent@@@Z 100087ec     qt-mt323:qt-mt323.dll
 0002:000007f0       __imp_?undock@QDockWindow@@UAEXPAVQWidget@@@Z 100087f0     qt-mt323:qt-mt323.dll
 0002:000007f4       __imp_?undock@QDockWindow@@UAEXXZ 100087f4     qt-mt323:qt-mt323.dll
 0002:000007f8       __imp_?updateItem@QPopupMenu@@UAEXH@Z 100087f8     qt-mt323:qt-mt323.dll
 0002:000007fc       __imp_?write@QGDict@@MBEAAVQDataStream@@AAV2@PAX@Z 100087fc     qt-mt323:qt-mt323.dll
 0002:00000800       __imp_?write@QGList@@MBEAAVQDataStream@@AAV2@PAX@Z 10008800     qt-mt323:qt-mt323.dll
 0002:00000804       __imp_??_7?$QPtrList@VQDockWindow@@@@6B@ 10008804     qt-mt323:qt-mt323.dll
 0002:00000808       __imp_?arg@QString@@QBE?AV1@HHH@Z 10008808     qt-mt323:qt-mt323.dll
 0002:0000080c       __imp_?replace@QString@@QAEAAV1@ABV1@0@Z 1000880c     qt-mt323:qt-mt323.dll
 0002:00000810       __imp_??0QTextStream@@QAE@PAVQIODevice@@@Z 10008810     qt-mt323:qt-mt323.dll
 0002:00000814       __imp_??1QTextStream@@UAE@XZ 10008814     qt-mt323:qt-mt323.dll
 0002:00000818       __imp_??6QTextStream@@QAEAAV0@PBD@Z 10008818     qt-mt323:qt-mt323.dll
 0002:0000081c       __imp_??6QTextStream@@QAEAAV0@ABVQString@@@Z 1000881c     qt-mt323:qt-mt323.dll
 0002:00000820       __imp_?first@QGList@@IAEPAXXZ 10008820     qt-mt323:qt-mt323.dll
 0002:00000824       __imp_?next@QGList@@IAEPAXXZ 10008824     qt-mt323:qt-mt323.dll
 0002:00000828       __imp_?blockSignals@QObject@@QAEX_N@Z 10008828     qt-mt323:qt-mt323.dll
 0002:0000082c       __imp_?setPaletteForegroundColor@QWidget@@QAEXABVQColor@@@Z 1000882c     qt-mt323:qt-mt323.dll
 0002:00000830       __imp_??0QCheckTableItem@@QAE@PAVQTable@@ABVQString@@@Z 10008830     qt-mt323:qt-mt323.dll
 0002:00000834       __imp_?isRowSelected@QTable@@QBE_NH_N@Z 10008834     qt-mt323:qt-mt323.dll
 0002:00000838       __imp_?addWidget@QBoxLayout@@QAEXPAVQWidget@@HH@Z 10008838     qt-mt323:qt-mt323.dll
 0002:0000083c       __imp_?add@QWhatsThis@@SAXPAVQWidget@@ABVQString@@@Z 1000883c     qt-mt323:qt-mt323.dll
 0002:00000840       __imp_?createEditor@QCheckTableItem@@UBEPAVQWidget@@XZ 10008840     qt-mt323:qt-mt323.dll
 0002:00000844       __imp_?paint@QCheckTableItem@@UAEXPAVQPainter@@ABVQColorGroup@@ABVQRect@@_N@Z 10008844     qt-mt323:qt-mt323.dll
 0002:00000848       __imp_?rtti@QCheckTableItem@@UBEHXZ 10008848     qt-mt323:qt-mt323.dll
 0002:0000084c       __imp_?setChecked@QCheckTableItem@@UAEX_N@Z 1000884c     qt-mt323:qt-mt323.dll
 0002:00000850       __imp_?setContentFromEditor@QCheckTableItem@@UAEXPAVQWidget@@@Z 10008850     qt-mt323:qt-mt323.dll
 0002:00000854       __imp_?setText@QCheckTableItem@@UAEXABVQString@@@Z 10008854     qt-mt323:qt-mt323.dll
 0002:00000858       __imp_?sizeHint@QCheckTableItem@@UBE?AVQSize@@XZ 10008858     qt-mt323:qt-mt323.dll
 0002:0000085c       __imp_?black@Qt@@2AAVQColor@@A 1000885c     qt-mt323:qt-mt323.dll
 0002:00000860       __imp_?gray@Qt@@2AAVQColor@@A 10008860     qt-mt323:qt-mt323.dll
 0002:00000864       __imp_?qstrcmp@@YAHPBD0@Z  10008864     qt-mt323:qt-mt323.dll
 0002:00000868       __imp_?fromLatin1@QString@@SA?AV1@PBDH@Z 10008868     qt-mt323:qt-mt323.dll
 0002:0000086c       __imp_?qt_cast@QTable@@UAEPAXPBD@Z 1000886c     qt-mt323:qt-mt323.dll
 0002:00000870       __imp_?qt_invoke@QTable@@UAE_NHPAUQUObject@@@Z 10008870     qt-mt323:qt-mt323.dll
 0002:00000874       __imp_?qt_emit@QTable@@UAE_NHPAUQUObject@@@Z 10008874     qt-mt323:qt-mt323.dll
 0002:00000878       __imp_?qt_property@QTable@@UAE_NHHPAVQVariant@@@Z 10008878     qt-mt323:qt-mt323.dll
 0002:0000087c       __imp_?staticMetaObject@QTable@@SAPAVQMetaObject@@XZ 1000887c     qt-mt323:qt-mt323.dll
 0002:00000880       __imp_?new_metaobject@QMetaObject@@SAPAV1@PBDPAV1@QBUQMetaData@@H2HQBVQMetaProperty@@HQBUQMetaEnum@@HQBUQClassInfo@@H@Z 10008880     qt-mt323:qt-mt323.dll
 0002:00000884       __imp_??0QMetaObjectCleanUp@@QAE@PBDP6APAVQMetaObject@@XZ@Z 10008884     qt-mt323:qt-mt323.dll
 0002:00000888       __imp_??1QMetaObjectCleanUp@@QAE@XZ 10008888     qt-mt323:qt-mt323.dll
 0002:0000088c       __imp_?setMetaObject@QMetaObjectCleanUp@@QAEXAAPAVQMetaObject@@@Z 1000888c     qt-mt323:qt-mt323.dll
 0002:00000890       __imp_?translate@QApplication@@QBE?AVQString@@PBD00W4Encoding@1@@Z 10008890     qt-mt323:qt-mt323.dll
 0002:00000894       __imp_?qApp@@3PAVQApplication@@A 10008894     qt-mt323:qt-mt323.dll
 0002:00000898       __imp_?staticMetaObject@QWidget@@SAPAVQMetaObject@@XZ 10008898     qt-mt323:qt-mt323.dll
 0002:0000089c       __imp_?static_QUType_ptr@@3UQUType_ptr@@A 1000889c     qt-mt323:qt-mt323.dll
 0002:000008a0       __imp_?static_QUType_QString@@3UQUType_QString@@A 100088a0     qt-mt323:qt-mt323.dll
 0002:000008a4       __imp_?receivers@QObject@@IBEPAVQConnectionList@@H@Z 100088a4     qt-mt323:qt-mt323.dll
 0002:000008a8       __imp_?activate_signal@QObject@@IAEXPAVQConnectionList@@PAUQUObject@@@Z 100088a8     qt-mt323:qt-mt323.dll
 0002:000008ac       __imp_??0QUObject@@QAE@XZ  100088ac     qt-mt323:qt-mt323.dll
 0002:000008b0       __imp_??1QUObject@@QAE@XZ  100088b0     qt-mt323:qt-mt323.dll
 0002:000008b4       __imp_?set@QUType_QString@@QAEXPAUQUObject@@ABVQString@@@Z 100088b4     qt-mt323:qt-mt323.dll
 0002:000008b8       __imp_?static_QUType_int@@3UQUType_int@@A 100088b8     qt-mt323:qt-mt323.dll
 0002:000008bc       __imp_?resize@QWidget@@QAEXABVQSize@@@Z 100088bc     qt-mt323:qt-mt323.dll
 0002:000008c0       __imp_??0QVBoxLayout@@QAE@PAVQWidget@@HHPBD@Z 100088c0     qt-mt323:qt-mt323.dll
 0002:000008c4       __imp_??1QVBoxLayout@@UAE@XZ 100088c4     qt-mt323:qt-mt323.dll
 0002:000008c8       __imp_?addItem@QBoxLayout@@UAEXPAVQLayoutItem@@@Z 100088c8     qt-mt323:qt-mt323.dll
 0002:000008cc       __imp_?childEvent@QLayout@@MAEXPAVQChildEvent@@@Z 100088cc     qt-mt323:qt-mt323.dll
 0002:000008d0       __imp_?className@QVBoxLayout@@UBEPBDXZ 100088d0     qt-mt323:qt-mt323.dll
 0002:000008d4       __imp_?eventFilter@QLayout@@MAE_NPAVQObject@@PAVQEvent@@@Z 100088d4     qt-mt323:qt-mt323.dll
 0002:000008d8       __imp_?expanding@QBoxLayout@@UBE?AW4ExpandData@QSizePolicy@@XZ 100088d8     qt-mt323:qt-mt323.dll
 0002:000008dc       __imp_?geometry@QLayout@@UBE?AVQRect@@XZ 100088dc     qt-mt323:qt-mt323.dll
 0002:000008e0       __imp_?hasHeightForWidth@QBoxLayout@@UBE_NXZ 100088e0     qt-mt323:qt-mt323.dll
 0002:000008e4       __imp_?heightForWidth@QBoxLayout@@UBEHH@Z 100088e4     qt-mt323:qt-mt323.dll
 0002:000008e8       __imp_?invalidate@QBoxLayout@@UAEXXZ 100088e8     qt-mt323:qt-mt323.dll
 0002:000008ec       __imp_?isEmpty@QLayout@@UBE_NXZ 100088ec     qt-mt323:qt-mt323.dll
 0002:000008f0       __imp_?iterator@QBoxLayout@@UAE?AVQLayoutIterator@@XZ 100088f0     qt-mt323:qt-mt323.dll
 0002:000008f4       __imp_?layout@QLayout@@UAEPAV1@XZ 100088f4     qt-mt323:qt-mt323.dll
 0002:000008f8       __imp_?maximumSize@QBoxLayout@@UBE?AVQSize@@XZ 100088f8     qt-mt323:qt-mt323.dll
 0002:000008fc       __imp_?metaObject@QVBoxLayout@@UBEPAVQMetaObject@@XZ 100088fc     qt-mt323:qt-mt323.dll
 0002:00000900       __imp_?minimumSize@QBoxLayout@@UBE?AVQSize@@XZ 10008900     qt-mt323:qt-mt323.dll
 0002:00000904       __imp_?qt_cast@QVBoxLayout@@UAEPAXPBD@Z 10008904     qt-mt323:qt-mt323.dll
 0002:00000908       __imp_?qt_emit@QVBoxLayout@@UAE_NHPAUQUObject@@@Z 10008908     qt-mt323:qt-mt323.dll
 0002:0000090c       __imp_?qt_invoke@QVBoxLayout@@UAE_NHPAUQUObject@@@Z 1000890c     qt-mt323:qt-mt323.dll
 0002:00000910       __imp_?qt_property@QVBoxLayout@@UAE_NHHPAVQVariant@@@Z 10008910     qt-mt323:qt-mt323.dll
 0002:00000914       __imp_?setAlignment@QLayoutItem@@UAEXH@Z 10008914     qt-mt323:qt-mt323.dll
 0002:00000918       __imp_?setAutoAdd@QLayout@@UAEX_N@Z 10008918     qt-mt323:qt-mt323.dll
 0002:0000091c       __imp_?setGeometry@QBoxLayout@@UAEXABVQRect@@@Z 1000891c     qt-mt323:qt-mt323.dll
 0002:00000920       __imp_?setMargin@QLayout@@UAEXH@Z 10008920     qt-mt323:qt-mt323.dll
 0002:00000924       __imp_?setMenuBar@QLayout@@UAEXPAVQMenuBar@@@Z 10008924     qt-mt323:qt-mt323.dll
 0002:00000928       __imp_?setSpacing@QLayout@@UAEXH@Z 10008928     qt-mt323:qt-mt323.dll
 0002:0000092c       __imp_?sizeHint@QBoxLayout@@UBE?AVQSize@@XZ 1000892c     qt-mt323:qt-mt323.dll
 0002:00000930       __imp_?spacerItem@QLayoutItem@@UAEPAVQSpacerItem@@XZ 10008930     qt-mt323:qt-mt323.dll
 0002:00000934       __imp_?widget@QLayoutItem@@UAEPAVQWidget@@XZ 10008934     qt-mt323:qt-mt323.dll
 0002:00000938       __imp_?setFrameShape@QFrame@@QAEXW4Shape@1@@Z 10008938     qt-mt323:qt-mt323.dll
 0002:0000093c       __imp_?setFrameShadow@QFrame@@QAEXW4Shadow@1@@Z 1000893c     qt-mt323:qt-mt323.dll
 0002:00000940       __imp_??0QLabel@@QAE@PAVQWidget@@PBDI@Z 10008940     qt-mt323:qt-mt323.dll
 0002:00000944       __imp_??1QLabel@@UAE@XZ    10008944     qt-mt323:qt-mt323.dll
 0002:00000948       __imp_?className@QLabel@@UBEPBDXZ 10008948     qt-mt323:qt-mt323.dll
 0002:0000094c       __imp_?drawContents@QLabel@@MAEXPAVQPainter@@@Z 1000894c     qt-mt323:qt-mt323.dll
 0002:00000950       __imp_?fontChange@QLabel@@MAEXABVQFont@@@Z 10008950     qt-mt323:qt-mt323.dll
 0002:00000954       __imp_?heightForWidth@QLabel@@UBEHH@Z 10008954     qt-mt323:qt-mt323.dll
 0002:00000958       __imp_?metaObject@QLabel@@UBEPAVQMetaObject@@XZ 10008958     qt-mt323:qt-mt323.dll
 0002:0000095c       __imp_?minimumSizeHint@QLabel@@UBE?AVQSize@@XZ 1000895c     qt-mt323:qt-mt323.dll
 0002:00000960       __imp_?qt_cast@QLabel@@UAEPAXPBD@Z 10008960     qt-mt323:qt-mt323.dll
 0002:00000964       __imp_?qt_emit@QLabel@@UAE_NHPAUQUObject@@@Z 10008964     qt-mt323:qt-mt323.dll
 0002:00000968       __imp_?qt_invoke@QLabel@@UAE_NHPAUQUObject@@@Z 10008968     qt-mt323:qt-mt323.dll
 0002:0000096c       __imp_?qt_property@QLabel@@UAE_NHHPAVQVariant@@@Z 1000896c     qt-mt323:qt-mt323.dll
 0002:00000970       __imp_?resizeEvent@QLabel@@MAEXPAVQResizeEvent@@@Z 10008970     qt-mt323:qt-mt323.dll
 0002:00000974       __imp_?setAlignment@QLabel@@UAEXH@Z 10008974     qt-mt323:qt-mt323.dll
 0002:00000978       __imp_?setAutoResize@QLabel@@UAEX_N@Z 10008978     qt-mt323:qt-mt323.dll
 0002:0000097c       __imp_?setBuddy@QLabel@@UAEXPAVQWidget@@@Z 1000897c     qt-mt323:qt-mt323.dll
 0002:00000980       __imp_?setFont@QLabel@@UAEXABVQFont@@@Z 10008980     qt-mt323:qt-mt323.dll
 0002:00000984       __imp_?setMovie@QLabel@@UAEXABVQMovie@@@Z 10008984     qt-mt323:qt-mt323.dll
 0002:00000988       __imp_?setNum@QLabel@@UAEXH@Z 10008988     qt-mt323:qt-mt323.dll
 0002:0000098c       __imp_?setNum@QLabel@@UAEXN@Z 1000898c     qt-mt323:qt-mt323.dll
 0002:00000990       __imp_?setPicture@QLabel@@UAEXABVQPicture@@@Z 10008990     qt-mt323:qt-mt323.dll
 0002:00000994       __imp_?setPixmap@QLabel@@UAEXABVQPixmap@@@Z 10008994     qt-mt323:qt-mt323.dll
 0002:00000998       __imp_?setText@QLabel@@UAEXABVQString@@@Z 10008998     qt-mt323:qt-mt323.dll
 0002:0000099c       __imp_?sizeHint@QLabel@@UBE?AVQSize@@XZ 1000899c     qt-mt323:qt-mt323.dll
 0002:000009a0       __imp_?styleChange@QFrame@@MAEXAAVQStyle@@@Z 100089a0     qt-mt323:qt-mt323.dll
 0002:000009a4       __imp_?closeEvent@QWidget@@MAEXPAVQCloseEvent@@@Z 100089a4     qt-mt323:qt-mt323.dll
 0002:000009a8       __imp_?close@QWidget@@UAE_N_N@Z 100089a8     qt-mt323:qt-mt323.dll
 0002:000009ac       __imp_?clearCellWidget@QTable@@UAEXHH@Z 100089ac     qt-mt323:qt-mt323.dll
 0002:000009b0       __imp_?clearCell@QTable@@UAEXHH@Z 100089b0     qt-mt323:qt-mt323.dll
 0002:000009b4       __imp_?childEvent@QObject@@MAEXPAVQChildEvent@@@Z 100089b4     qt-mt323:qt-mt323.dll
 0002:000009b8       __imp_?checkConnectArgs@QObject@@MAE_NPBDPBV1@0@Z 100089b8     qt-mt323:qt-mt323.dll
 0002:000009bc       __imp_?cellWidget@QTable@@UBEPAVQWidget@@HH@Z 100089bc     qt-mt323:qt-mt323.dll
 0002:000009c0       __imp_?cellRect@QTable@@UBE?AVQRect@@HH@Z 100089c0     qt-mt323:qt-mt323.dll
 0002:000009c4       __imp_?cellGeometry@QTable@@UBE?AVQRect@@HH@Z 100089c4     qt-mt323:qt-mt323.dll
 0002:000009c8       __imp_?beginEdit@QTable@@MAEPAVQWidget@@HH_N@Z 100089c8     qt-mt323:qt-mt323.dll
 0002:000009cc       __imp_?adjustSize@QWidget@@UAEXXZ 100089cc     qt-mt323:qt-mt323.dll
 0002:000009d0       __imp_?adjustRow@QTable@@UAEXH@Z 100089d0     qt-mt323:qt-mt323.dll
 0002:000009d4       __imp_?adjustColumn@QTable@@UAEXH@Z 100089d4     qt-mt323:qt-mt323.dll
 0002:000009d8       __imp_?addSelection@QTable@@UAEHABVQTableSelection@@@Z 100089d8     qt-mt323:qt-mt323.dll
 0002:000009dc       __imp_?addChild@QScrollView@@UAEXPAVQWidget@@HH@Z 100089dc     qt-mt323:qt-mt323.dll
 0002:000009e0       __imp_?activateNextCell@QTable@@MAEXXZ 100089e0     qt-mt323:qt-mt323.dll
 0002:000009e4       __imp_?setText@QClipboard@@QAEXABVQString@@W4Mode@1@@Z 100089e4     qt-mt323:qt-mt323.dll
 0002:000009e8       __imp_?clipboard@QApplication@@SAPAVQClipboard@@XZ 100089e8     qt-mt323:qt-mt323.dll
 0002:000009ec       __imp_?keyPressEvent@QTable@@MAEXPAVQKeyEvent@@@Z 100089ec     qt-mt323:qt-mt323.dll
 0002:000009f0       __imp_?selection@QTable@@QBE?AVQTableSelection@@H@Z 100089f0     qt-mt323:qt-mt323.dll
 0002:000009f4       __imp_?numSelections@QTable@@QBEHXZ 100089f4     qt-mt323:qt-mt323.dll
 0002:000009f8       __imp_?horizontalHeader@QTable@@QBEPAVQHeader@@XZ 100089f8     qt-mt323:qt-mt323.dll
 0002:000009fc       __imp_??1QTable@@UAE@XZ    100089fc     qt-mt323:qt-mt323.dll
 0002:00000a00       __imp_??0QTable@@QAE@PAVQWidget@@PBD@Z 10008a00     qt-mt323:qt-mt323.dll
 0002:00000a04       __imp_?isChecked@QCheckTableItem@@QBE_NXZ 10008a04     qt-mt323:qt-mt323.dll
 0002:00000a08       __imp_?label@QHeader@@QBE?AVQString@@H@Z 10008a08     qt-mt323:qt-mt323.dll
 0002:00000a0c       __imp_??H@YA?BVQString@@ABV0@0@Z 10008a0c     qt-mt323:qt-mt323.dll
 0002:00000a10       __imp_??YQString@@QAEAAV0@PBD@Z 10008a10     qt-mt323:qt-mt323.dll
 0002:00000a14       __imp_??4QString@@QAEAAV0@ABV0@@Z 10008a14     qt-mt323:qt-mt323.dll
 0002:00000a18       __imp_??1QString@@QAE@XZ   10008a18     qt-mt323:qt-mt323.dll
 0002:00000a1c       __imp_??0QString@@QAE@XZ   10008a1c     qt-mt323:qt-mt323.dll
 0002:00000a20       __imp_?qDebug@@YAXPBDZZ    10008a20     qt-mt323:qt-mt323.dll
 0002:00000a24       \177qt-mt323_NULL_THUNK_DATA 10008a24     qt-mt323:qt-mt323.dll
 0002:00000a28       ___xc_a                    10008a28     MSVCRT:cinitexe.obj
 0002:00000a44       ___xc_z                    10008a44     MSVCRT:cinitexe.obj
 0002:00000a48       ___xi_a                    10008a48     MSVCRT:cinitexe.obj
 0002:00000a54       ___xi_z                    10008a54     MSVCRT:cinitexe.obj
 0002:00000a5c       ??_7bncsTable@@6BQObject@@@ 10008a5c     bncsTable.obj
 0002:00000e00       ??_7bncsTable@@6BQPaintDevice@@@ 10008e00     bncsTable.obj
 0002:00000e20       ??_C@_0BH@DEJAMDON@key?5press?5event?3?5?$CFc?5?$CFd?$AA@ 10008e20     bncsTable.obj
 0002:00000e38       ??_C@_01GPOEFGEJ@?7?$AA@   10008e38     bncsTable.obj
 0002:00000e3c       ??_C@_01EEMJAFIK@?6?$AA@   10008e3c     bncsTable.obj
 0002:00000e44       ??_7panelsetsTableItem@@6B@ 10008e44     panelsetsTableItem.obj
 0002:00000e94       ??_SQComboBox@@6BQObject@@@ 10008e94     panelsetsTableItem.obj
 0002:00001078       ??_SQComboBox@@6BQPaintDevice@@@ 10009078     panelsetsTableItem.obj
 0002:00001098       ??_C@_0BC@NAAGCOBJ@1doValueChanged?$CI?$CJ?$AA@ 10009098     panelsetsTableItem.obj
 0002:000010ac       ??_C@_0BC@BGJFBFF@2activated?$CI?5int?5?$CJ?$AA@ 100090ac     panelsetsTableItem.obj
 0002:000010c0       ??_C@_0N@LIKKKKKK@1destroyed?$CI?$CJ?$AA@ 100090c0     panelsetsTableItem.obj
 0002:000010d0       ??_C@_0N@FGAMGGE@2destroyed?$CI?$CJ?$AA@ 100090d0     panelsetsTableItem.obj
 0002:000010e0       ??_C@_0L@IINBHNNO@mydocument?$AA@ 100090e0     panelsetsTableItem.obj
 0002:000010ec       ??_C@_0BG@BOFIIFLN@?2config?2panelsets?4xml?$AA@ 100090ec     panelsetsTableItem.obj
 0002:00001104       ??_C@_0CI@JONOEMHN@usersEditor?3?5can?8t?5open?5panelset@ 10009104     panelsetsTableItem.obj
 0002:0000112c       ??_C@_0CO@HGDELOGB@usersEditor?3?5can?8t?5read?5into?5DOM@ 1000912c     panelsetsTableItem.obj
 0002:0000115c       ??_C@_06GGPOMPNM@?$CInone?$CJ?$AA@ 1000915c     panelsetsTableItem.obj
 0002:00001164       ??_C@_02EGCJHIOB@id?$AA@   10009164     panelsetsTableItem.obj
 0002:00001168       ??_C@_09IFDIHLJH@QComboBox?$AA@ 10009168     panelsetsTableItem.obj
 0002:00001172       ??_C@_00CNPNBAHC@?$AA@     10009172     panelsetsTableItem.obj
 0002:00001174       ??_C@_09OFODDICG@14?514?52?51?$AA@ 10009174     plugindesc.obj
 0002:00001180       ??_C@_0M@KEPPNGJB@?$CD?5c?5?$CD000000?$AA@ 10009180     plugindesc.obj
 0002:0000118c       ??_C@_08IMFNEMJ@?4?5c?5none?$AA@ 1000918c     plugindesc.obj
 0002:00001198       ??_C@_0P@HFKAALMG@?4?4?4?4?4?4?4?4?4?4?4?4?4?4?$AA@ 10009198     plugindesc.obj
 0002:000011ac       ??_7config_plugin_desc_base@@6B@ 100091ac     plugindesc.obj
 0002:000011c0       ??_7plugindesc@@6B@        100091c0     plugindesc.obj
 0002:000011d0       ??_C@_0BC@BGJNCJMC@Home?1System?1Users?$AA@ 100091d0     plugindesc.obj
 0002:000011e8       ??_7userLevelTableItem@@6B@ 100091e8     userLevelTableItem.obj
 0002:00001230       ??_C@_09GNBOHHKB@Read?5Only?$AA@ 10009230     userLevelTableItem.obj
 0002:0000123c       ??_C@_04ODLBFFJE@User?$AA@ 1000923c     userLevelTableItem.obj
 0002:00001244       ??_C@_0L@BIEKHEBJ@Supervisor?$AA@ 10009244     userLevelTableItem.obj
 0002:00001250       ??_C@_0O@PMKNNGMO@Administrator?$AA@ 10009250     userLevelTableItem.obj
 0002:00001260       ??_C@_09HCBPJCHD@Developer?$AA@ 10009260     userLevelTableItem.obj
 0002:0000126c       ??_C@_02GIPFHKNO@OK?$AA@   1000926c     usersEditor.obj
 0002:00001274       ??_SQAction@@6B@           10009274     usersEditor.obj
 0002:00001304       ??_SQToolBar@@6BQObject@@@ 10009304     usersEditor.obj
 0002:00001520       ??_SQToolBar@@6BQPaintDevice@@@ 10009520     usersEditor.obj
 0002:00001544       ??_SQGuardedPtrPrivate@@6B@ 10009544     usersEditor.obj
 0002:00001598       ??_7QDockWindowList@@6B@   10009598     usersEditor.obj
 0002:000015bc       ??_SQPopupMenu@@6BQObject@@@ 100095bc     usersEditor.obj
 0002:0000179c       ??_SQPopupMenu@@6BQPaintDevice@@@ 1000979c     usersEditor.obj
 0002:000017c0       ??_SQPopupMenu@@6B@        100097c0     usersEditor.obj
 0002:000017e4       ??_7?$QPtrList@VQPopupMenu@@@@6B@ 100097e4     usersEditor.obj
 0002:00001808       ??_7QPopupMenuList@@6B@    10009808     usersEditor.obj
 0002:00001828       ??_C@_04OOEBCMBF@FAIL?$AA@ 10009828     usersEditor.obj
 0002:00001830       ??_C@_08OBALAKLA@READONLY?$AA@ 10009830     usersEditor.obj
 0002:0000183c       ??_C@_04KANDKFIK@DONE?$AA@ 1000983c     usersEditor.obj
 0002:00001844       ??_C@_07NFANNNEC@UNKNOWN?$AA@ 10009844     usersEditor.obj
 0002:00001850       ??_7config_plugin_base@@6BQObject@@@ 10009850     usersEditor.obj
 0002:00001a28       ??_7config_plugin_base@@6BQPaintDevice@@@ 10009a28     usersEditor.obj
 0002:00001a48       ??_C@_0EB@GNDACMDJ@?$CC?5?9?5the?5author?5should?5have?5defin@ 10009a48     usersEditor.obj
 0002:00001a8c       ??_C@_0CH@BDPDPLDP@This?5is?5the?5default?5?$CCAbout?$CC?5text@ 10009a8c     usersEditor.obj
 0002:00001ab8       ??_7?$QDict@VQAction@@@@6B@ 10009ab8     usersEditor.obj
 0002:00001ad8       ??_7usersEditor@@6BQObject@@@ 10009ad8     usersEditor.obj
 0002:00001cb0       ??_7usersEditor@@6BQPaintDevice@@@ 10009cb0     usersEditor.obj
 0002:00001cd0       ??_C@_0O@GEGCOHGM@usersEditor?3?5?$AA@ 10009cd0     usersEditor.obj
 0002:00001ce0       ??_C@_0BB@FEGHJLOM@config?1users?4xml?$AA@ 10009ce0     usersEditor.obj
 0002:00001cf4       ??_C@_0BN@CEGLABJP@2command?$CI?5QString?0?5QString?5?$CJ?$AA@ 10009cf4     usersEditor.obj
 0002:00001d14       ??_C@_0BI@DJGPDCG@Template?5Plugin?5Toolbar?$AA@ 10009d14     usersEditor.obj
 0002:00001d2c       ??_C@_05LHMKEDEH@?$CGEdit?$AA@ 10009d2c     usersEditor.obj
 0002:00001d34       ??_C@_03CLCAEGCJ@new?$AA@  10009d34     usersEditor.obj
 0002:00001d38       ??_C@_04CCPFBLLC@?$CGNew?$AA@ 10009d38     usersEditor.obj
 0002:00001d40       ??_C@_07EJAINBEK@filenew?$AA@ 10009d40     usersEditor.obj
 0002:00001d48       ??_C@_08GDKCCLPO@New?5User?$AA@ 10009d48     usersEditor.obj
 0002:00001d54       ??_C@_06FOBLBEIN@delete?$AA@ 10009d54     usersEditor.obj
 0002:00001d5c       ??_C@_0L@BPDPNFLB@filedelete?$AA@ 10009d5c     usersEditor.obj
 0002:00001d68       ??_C@_0M@GHLHALBI@Delete?5User?$AA@ 10009d68     usersEditor.obj
 0002:00001d74       ??_C@_0L@IDAGKIO@1addUser?$CI?$CJ?$AA@ 10009d74     usersEditor.obj
 0002:00001d80       ??_C@_0N@KCMOKDBB@2activated?$CI?$CJ?$AA@ 10009d80     usersEditor.obj
 0002:00001d90       ??_C@_0O@CAMFNOAB@1deleteUser?$CI?$CJ?$AA@ 10009d90     usersEditor.obj
 0002:00001da0       ??_C@_06BNCCALCL@unlock?$AA@ 10009da0     usersEditor.obj
 0002:00001da8       ??_C@_09JLEOPMAJ@?5?9?5error?$DN?$AA@ 10009da8     usersEditor.obj
 0002:00001db4       ??_C@_09LBCHCBIC@?5?9?5value?$DN?$AA@ 10009db4     usersEditor.obj
 0002:00001dc0       ??_C@_0P@ELNNACEA@?5?9?5textStatus?$DN?$AA@ 10009dc0     usersEditor.obj
 0002:00001dd0       ??_C@_0L@LEAPMKGP@Reply?3?5op?$DN?$AA@ 10009dd0     usersEditor.obj
 0002:00001ddc       ??_C@_08HNIAHLMM@download?$AA@ 10009ddc     usersEditor.obj
 0002:00001de8       ??_C@_01KMDKNFGN@?1?$AA@   10009de8     usersEditor.obj
 0002:00001dec       ??_C@_06KAOCKAGB@upload?$AA@ 10009dec     usersEditor.obj
 0002:00001df4       ??_C@_05CCAMFJOL@clean?$AA@ 10009df4     usersEditor.obj
 0002:00001dfc       ??_C@_0M@EBFEGAAI@Information?$AA@ 10009dfc     usersEditor.obj
 0002:00001e08       ??_C@_0CO@GKAEALGF@Being?5asked?5to?5navigate?5to?5?$CF1?5wi@ 10009e08     usersEditor.obj
 0002:00001e38       ??_C@_0N@EHHLDFOB@checkoutFile?$AA@ 10009e38     usersEditor.obj
 0002:00001e48       ??_C@_0BF@GGAPJNIF@config?1panelsets?4xml?$AA@ 10009e48     usersEditor.obj
 0002:00001e60       ??_C@_0N@LJNCPLAD@downloadFile?$AA@ 10009e60     usersEditor.obj
 0002:00001e70       ??_C@_0L@CIKGEHEG@uploadFile?$AA@ 10009e70     usersEditor.obj
 0002:00001e7c       ??_C@_0DP@NPFMHNGF@?$DMh3?$DOTemplate?5Configuration?5Plugi@ 10009e7c     usersEditor.obj
 0002:00001ebc       ??_C@_08IJEMJLKG@13?324?359?$AA@ 10009ebc     usersEditor.obj
 0002:00001ec8       ??_C@_0M@JEDEHNP@Sep?523?52021?$AA@ 10009ec8     usersEditor.obj
 0002:00001edc       ??_SQCheckTableItem@@6B@   10009edc     usersEditordlgimpl.obj
 0002:00001f2c       ??_7usersEditorDlg@@6BQObject@@@ 10009f2c     usersEditordlgimpl.obj
 0002:000020e4       ??_7usersEditorDlg@@6BQPaintDevice@@@ 1000a0e4     usersEditordlgimpl.obj
 0002:00002104       ??_C@_06KDFPGKKJ@table1?$AA@ 1000a104     usersEditordlgimpl.obj
 0002:0000210c       ??_C@_04FABLJDN@Name?$AA@  1000a10c     usersEditordlgimpl.obj
 0002:00002114       ??_C@_08FJIAHGMM@Password?$AA@ 1000a114     usersEditordlgimpl.obj
 0002:00002120       ??_C@_05KOHFLOFG@Level?$AA@ 1000a120     usersEditordlgimpl.obj
 0002:00002128       ??_C@_0BB@GMNBEHBM@Default?5Panelset?$AA@ 1000a128     usersEditordlgimpl.obj
 0002:0000213c       ??_C@_0BG@ELFBGIHJ@Default?5Eng?4?5Panelset?$AA@ 1000a13c     usersEditordlgimpl.obj
 0002:00002154       ??_C@_0M@FFDLKKOC@System?5User?$AA@ 1000a154     usersEditordlgimpl.obj
 0002:00002160       ??_C@_0M@LMNJGDDI@Config?5User?$AA@ 1000a160     usersEditordlgimpl.obj
 0002:00002170       ??_C@_0DDC@OCAHGNNJ@?$DMp?$DO?$DMb?$DOUsers?5for?5this?5Colledia?5Co@ 1000a170     usersEditordlgimpl.obj
 0002:000024a4       ??_C@_0BJ@MLJPFPGN@1textChanged?$CI?5int?0?5int?5?$CJ?$AA@ 1000a4a4     usersEditordlgimpl.obj
 0002:000024c0       ??_C@_0BK@OCHKEFCC@2valueChanged?$CI?5int?0?5int?5?$CJ?$AA@ 1000a4c0     usersEditordlgimpl.obj
 0002:000024dc       ??_C@_0CH@FEFACFFL@usersEditorDlg?3?5loading?5users?5fi@ 1000a4dc     usersEditordlgimpl.obj
 0002:00002504       ??_C@_08NLHBPEGP@password?$AA@ 1000a504     usersEditordlgimpl.obj
 0002:00002510       ??_C@_05KJNJLLGA@level?$AA@ 1000a510     usersEditordlgimpl.obj
 0002:00002518       ??_C@_08FGKDABPH@panelset?$AA@ 1000a518     usersEditordlgimpl.obj
 0002:00002524       ??_C@_06NODEDMPP@engset?$AA@ 1000a524     usersEditordlgimpl.obj
 0002:0000252c       ??_C@_01HIHLOKLC@1?$AA@    1000a52c     usersEditordlgimpl.obj
 0002:00002530       ??_C@_06FHFOAHML@system?$AA@ 1000a530     usersEditordlgimpl.obj
 0002:00002538       ??_C@_06HEJKKHEK@config?$AA@ 1000a538     usersEditordlgimpl.obj
 0002:00002540       ??_C@_0BC@BFIEMEJM@?2config?2users?4xml?$AA@ 1000a540     usersEditordlgimpl.obj
 0002:00002558       ??_C@_0FD@PLAOHPOJ@?$DM?$DPxml?5version?$DN?$CC1?40?$CC?5encoding?$DN?$CCUT@ 1000a558     usersEditordlgimpl.obj
 0002:000025ac       ??_C@_02PIGFKFFE@?$CF1?$AA@ 1000a5ac     usersEditordlgimpl.obj
 0002:000025b0       ??_C@_0M@KNIKEEHG@?7?$DMuser?5id?$DN?$CC?$AA@ 1000a5b0     usersEditordlgimpl.obj
 0002:000025bc       ??_C@_0N@HMFEHINH@?$CC?5password?$DN?$CC?$AA@ 1000a5bc     usersEditordlgimpl.obj
 0002:000025cc       ??_C@_0N@IBLPDIE@?$CC?5panelset?$DN?$CC?$AA@ 1000a5cc     usersEditordlgimpl.obj
 0002:000025dc       ??_C@_0L@CLGJPPKG@?$CC?5engset?$DN?$CC?$AA@ 1000a5dc     usersEditordlgimpl.obj
 0002:000025e8       ??_C@_09PNLOHOMI@?$CC?5level?$DN?$CC?$AA@ 1000a5e8     usersEditordlgimpl.obj
 0002:000025f4       ??_C@_0L@CBEIGMBP@?$CC?5system?$DN?$CC?$AA@ 1000a5f4     usersEditordlgimpl.obj
 0002:00002600       ??_C@_0L@NFAGEFDJ@?$CC?5config?$DN?$CC?$AA@ 1000a600     usersEditordlgimpl.obj
 0002:0000260c       ??_C@_05OJNDEKBN@?$CC?5?1?$DO?6?$AA@ 1000a60c     usersEditordlgimpl.obj
 0002:00002614       ??_C@_08EFNFHFNA@?$DM?1users?$DO?$AA@ 1000a614     usersEditordlgimpl.obj
 0002:00002620       ??_C@_05CFEJGMAI@dirty?$AA@ 1000a620     usersEditordlgimpl.obj
 0002:00002628       ??_C@_06DDLNFFBN@?$CGquot?$DL?$AA@ 1000a628     usersEditordlgimpl.obj
 0002:00002630       ??_C@_01BJJEKLCA@?$CC?$AA@ 1000a630     usersEditordlgimpl.obj
 0002:00002634       ??_C@_04GJOGLFEJ@?$CGlt?$DL?$AA@ 1000a634     usersEditordlgimpl.obj
 0002:0000263c       ??_C@_01MNNFJEPP@?$DM?$AA@ 1000a63c     usersEditordlgimpl.obj
 0002:00002640       ??_C@_04LOOHDCEI@?$CGgt?$DL?$AA@ 1000a640     usersEditordlgimpl.obj
 0002:00002648       ??_C@_01PPODPGHN@?$DO?$AA@ 1000a648     usersEditordlgimpl.obj
 0002:0000264c       ??_C@_05JKJFEODM@?$CGamp?$DL?$AA@ 1000a64c     usersEditordlgimpl.obj
 0002:00002654       ??_C@_01HNPIGOCE@?$CG?$AA@ 1000a654     usersEditordlgimpl.obj
 0002:00002658       ??_C@_06PNMEMOHD@?$CGapos?$DL?$AA@ 1000a658     usersEditordlgimpl.obj
 0002:00002660       ??_C@_01GEODFPGF@?8?$AA@   1000a660     usersEditordlgimpl.obj
 0002:00002668       ??_7?$QPtrList@H@@6B@      1000a668     usersEditordlgimpl.obj
 0002:00002688       ??_C@_09CFAHPCCO@bncsTable?$AA@ 1000a688     moc_bncsTable.obj
 0002:000026a0       ??_C@_06DCNCJKNL@doCopy?$AA@ 1000a6a0     moc_bncsTable.obj
 0002:000026b4       ??_C@_07CJKGLEMN@doPaste?$AA@ 1000a6b4     moc_bncsTable.obj
 0002:000026c8       ??_C@_06GCHJCBOH@doUndo?$AA@ 1000a6c8     moc_bncsTable.obj
 0002:000026dc       ??_C@_08OCIHIEHO@doDelete?$AA@ 1000a6dc     moc_bncsTable.obj
 0002:00002718       ??_C@_08ONMOP@doCopy?$CI?$CJ?$AA@ 1000a718     moc_bncsTable.obj
 0002:00002724       ??_C@_09MAEAHPID@doPaste?$CI?$CJ?$AA@ 1000a724     moc_bncsTable.obj
 0002:00002730       ??_C@_08CPEOJPLP@doUndo?$CI?$CJ?$AA@ 1000a730     moc_bncsTable.obj
 0002:0000273c       ??_C@_0L@CJHBHJHF@doDelete?$CI?$CJ?$AA@ 1000a73c     moc_bncsTable.obj
 0002:00002748       ??_C@_0P@ECKEJGFB@toolWindowBase?$AA@ 1000a748     moc_toolwindow.obj
 0002:00002764       ??_C@_0P@DMEOIADN@languageChange?$AA@ 1000a764     moc_toolwindow.obj
 0002:00002780       ??_C@_0BB@PFEIHPGD@languageChange?$CI?$CJ?$AA@ 1000a780     moc_toolwindow.obj
 0002:00002794       ??_C@_0L@IGMLIIOB@toolWindow?$AA@ 1000a794     moc_toolwindowimpl.obj
 0002:000027a0       ??_C@_0O@NDCCBDNA@QIconViewItem?$AA@ 1000a7a0     moc_toolwindowimpl.obj
 0002:000027bc       ??_C@_0BB@FFKPNNIH@selectionChanged?$AA@ 1000a7bc     moc_toolwindowimpl.obj
 0002:000027dc       ??_C@_0CB@DONPBGFK@selectionChanged?$CIQIconViewItem?$CK?$CJ@ 1000a7dc     moc_toolwindowimpl.obj
 0002:0000280c       ??_C@_0N@DENPNHIG@fileSelected?$AA@ 1000a80c     moc_toolwindowimpl.obj
 0002:00002828       ??_C@_0BN@NHBBIGHD@fileSelected?$CIconst?5QString?$CG?$CJ?$AA@ 1000a828     moc_toolwindowimpl.obj
 0002:00002848       ??_C@_0M@DPOMOLJO@usersEditor?$AA@ 1000a848     moc_usersEditor.obj
 0002:00002854       ??_C@_08BABJIOEM@filename?$AA@ 1000a854     moc_usersEditor.obj
 0002:00002884       ??_C@_07KMMNMMFF@command?$AA@ 1000a884     moc_usersEditor.obj
 0002:00002898       ??_C@_0BJ@FEFNJDLM@command?$CIQString?0QString?$CJ?$AA@ 1000a898     moc_usersEditor.obj
 0002:000028b4       ??_C@_0BD@JNLMCDMJ@usersEditorDlgBase?$AA@ 1000a8b4     moc_usersEditordlg.obj
 0002:000028e0       ??_C@_0P@JMLMBBPP@usersEditorDlg?$AA@ 1000a8e0     moc_usersEditordlgimpl.obj
 0002:000028f0       ??_C@_03DMHICLNI@row?$AA@  1000a8f0     moc_usersEditordlgimpl.obj
 0002:000028f4       ??_C@_03HNOLNALI@col?$AA@  1000a8f4     moc_usersEditordlgimpl.obj
 0002:00002904       ??_C@_0M@NJKJFEFJ@textChanged?$AA@ 1000a904     moc_usersEditordlgimpl.obj
 0002:0000291c       ??_C@_07LAGMPIHP@addUser?$AA@ 1000a91c     moc_usersEditordlgimpl.obj
 0002:00002930       ??_C@_0L@PLJFIPFF@deleteUser?$AA@ 1000a930     moc_usersEditordlgimpl.obj
 0002:00002960       ??_C@_0BF@LBJIOMAH@textChanged?$CIint?0int?$CJ?$AA@ 1000a960     moc_usersEditordlgimpl.obj
 0002:00002978       ??_C@_09GJNJCHMI@addUser?$CI?$CJ?$AA@ 1000a978     moc_usersEditordlgimpl.obj
 0002:00002984       ??_C@_0N@MINDEEIG@deleteUser?$CI?$CJ?$AA@ 1000a984     moc_usersEditordlgimpl.obj
 0002:000029b4       ??_SQVBoxLayout@@6BQObject@@@ 1000a9b4     toolwindow.obj
 0002:00002a1c       ??_SQVBoxLayout@@6BQLayoutItem@@@ 1000aa1c     toolwindow.obj
 0002:00002a60       ??_7usersEditorDlgBase@@6BQObject@@@ 1000aa60     usersEditordlg.obj
 0002:00002c18       ??_7usersEditorDlgBase@@6BQPaintDevice@@@ 1000ac18     usersEditordlg.obj
 0002:00002c3c       ??_SQLabel@@6BQObject@@@   1000ac3c     usersEditordlg.obj
 0002:00002e34       ??_SQLabel@@6BQPaintDevice@@@ 1000ae34     usersEditordlg.obj
 0002:00002e54       ??_C@_0BJ@NMAEHAHJ@usersEditorDlgBaseLayout?$AA@ 1000ae54     usersEditordlg.obj
 0002:00002e70       ??_C@_0N@CJBMCOMC@textLabel1_4?$AA@ 1000ae70     usersEditordlg.obj
 0002:00002e80       ??_C@_0P@KCEMFHPK@?$DMh1?$DOUsers?$DM?1h1?$DO?$AA@ 1000ae80     usersEditordlg.obj
 0002:00002e90       ??_C@_0CH@PKLDHJEL@Users?5for?5this?5Colledia?5Control?5@ 1000ae90     usersEditordlg.obj
 0002:00002ebc       ??_7type_info@@6B@         1000aebc     MSVCRT:ti_inst.obj
 0002:00002ec0       __pDefaultRawDllMain       1000aec0     MSVCRT:crtdll.obj
 0002:00002ec0       __pRawDllMain              1000aec0     MSVCRT:crtdll.obj
 0002:00002ed0       __load_config_used         1000aed0     MSVCRT:loadcfg.obj
 0002:00002f18       ??_R4bncsTable@@6BQObject@@@ 1000af18     bncsTable.obj
 0002:00002f2c       ??_R3bncsTable@@8          1000af2c     bncsTable.obj
 0002:00002f3c       ??_R2bncsTable@@8          1000af3c     bncsTable.obj
 0002:00002f60       ??_R1A@?0A@EA@bncsTable@@8 1000af60     bncsTable.obj
 0002:00002f7c       ??_R1A@?0A@EA@QTable@@8    1000af7c     bncsTable.obj
 0002:00002f98       ??_R3QTable@@8             1000af98     bncsTable.obj
 0002:00002fa8       ??_R2QTable@@8             1000afa8     bncsTable.obj
 0002:00002fc8       ??_R1A@?0A@EA@QScrollView@@8 1000afc8     bncsTable.obj
 0002:00002fe4       ??_R3QScrollView@@8        1000afe4     bncsTable.obj
 0002:00002ff4       ??_R2QScrollView@@8        1000aff4     bncsTable.obj
 0002:00003010       ??_R1A@?0A@EA@QFrame@@8    1000b010     bncsTable.obj
 0002:0000302c       ??_R3QFrame@@8             1000b02c     bncsTable.obj
 0002:0000303c       ??_R2QFrame@@8             1000b03c     bncsTable.obj
 0002:00003054       ??_R1A@?0A@EA@QWidget@@8   1000b054     bncsTable.obj
 0002:00003070       ??_R3QWidget@@8            1000b070     bncsTable.obj
 0002:00003080       ??_R2QWidget@@8            1000b080     bncsTable.obj
 0002:00003094       ??_R1A@?0A@EA@QObject@@8   1000b094     bncsTable.obj
 0002:000030b0       ??_R3QObject@@8            1000b0b0     bncsTable.obj
 0002:000030c0       ??_R2QObject@@8            1000b0c0     bncsTable.obj
 0002:000030cc       ??_R13?0A@EA@Qt@@8         1000b0cc     bncsTable.obj
 0002:000030e8       ??_R3Qt@@8                 1000b0e8     bncsTable.obj
 0002:000030f8       ??_R2Qt@@8                 1000b0f8     bncsTable.obj
 0002:00003100       ??_R1A@?0A@EA@Qt@@8        1000b100     bncsTable.obj
 0002:0000311c       ??_R1CI@?0A@EA@QPaintDevice@@8 1000b11c     bncsTable.obj
 0002:00003138       ??_R3QPaintDevice@@8       1000b138     bncsTable.obj
 0002:00003148       ??_R2QPaintDevice@@8       1000b148     bncsTable.obj
 0002:00003150       ??_R1A@?0A@EA@QPaintDevice@@8 1000b150     bncsTable.obj
 0002:0000316c       ??_R4bncsTable@@6BQPaintDevice@@@ 1000b16c     bncsTable.obj
 0002:00003180       ??_R4QComboBox@@6BQObject@@@ 1000b180     panelsetsTableItem.obj
 0002:00003194       ??_R3QComboBox@@8          1000b194     panelsetsTableItem.obj
 0002:000031a4       ??_R2QComboBox@@8          1000b1a4     panelsetsTableItem.obj
 0002:000031bc       ??_R1A@?0A@EA@QComboBox@@8 1000b1bc     panelsetsTableItem.obj
 0002:000031d8       ??_R4QComboBox@@6BQPaintDevice@@@ 1000b1d8     panelsetsTableItem.obj
 0002:000031ec       ??_R4panelsetsTableItem@@6B@ 1000b1ec     panelsetsTableItem.obj
 0002:00003200       ??_R3panelsetsTableItem@@8 1000b200     panelsetsTableItem.obj
 0002:00003210       ??_R2panelsetsTableItem@@8 1000b210     panelsetsTableItem.obj
 0002:00003220       ??_R1A@?0A@EA@panelsetsTableItem@@8 1000b220     panelsetsTableItem.obj
 0002:0000323c       ??_R1A@?0A@EA@QTableItem@@8 1000b23c     panelsetsTableItem.obj
 0002:00003258       ??_R3QTableItem@@8         1000b258     panelsetsTableItem.obj
 0002:00003268       ??_R2QTableItem@@8         1000b268     panelsetsTableItem.obj
 0002:00003274       ??_R4config_plugin_desc_base@@6B@ 1000b274     plugindesc.obj
 0002:00003288       ??_R3config_plugin_desc_base@@8 1000b288     plugindesc.obj
 0002:00003298       ??_R2config_plugin_desc_base@@8 1000b298     plugindesc.obj
 0002:000032a0       ??_R1A@?0A@EA@config_plugin_desc_base@@8 1000b2a0     plugindesc.obj
 0002:000032bc       ??_R4plugindesc@@6B@       1000b2bc     plugindesc.obj
 0002:000032d0       ??_R3plugindesc@@8         1000b2d0     plugindesc.obj
 0002:000032e0       ??_R2plugindesc@@8         1000b2e0     plugindesc.obj
 0002:000032ec       ??_R1A@?0A@EA@plugindesc@@8 1000b2ec     plugindesc.obj
 0002:00003308       ??_R4userLevelTableItem@@6B@ 1000b308     userLevelTableItem.obj
 0002:0000331c       ??_R3userLevelTableItem@@8 1000b31c     userLevelTableItem.obj
 0002:0000332c       ??_R2userLevelTableItem@@8 1000b32c     userLevelTableItem.obj
 0002:0000333c       ??_R1A@?0A@EA@userLevelTableItem@@8 1000b33c     userLevelTableItem.obj
 0002:00003358       ??_R3QShared@@8            1000b358     usersEditor.obj
 0002:00003368       ??_R2QShared@@8            1000b368     usersEditor.obj
 0002:00003370       ??_R1A@?0A@EA@QShared@@8   1000b370     usersEditor.obj
 0002:0000338c       ??_R1A@?0A@EA@QGList@@8    1000b38c     usersEditor.obj
 0002:000033a8       ??_R3QGList@@8             1000b3a8     usersEditor.obj
 0002:000033b8       ??_R2QGList@@8             1000b3b8     usersEditor.obj
 0002:000033c4       ??_R1A@?0A@EA@QPtrCollection@@8 1000b3c4     usersEditor.obj
 0002:000033e0       ??_R3QPtrCollection@@8     1000b3e0     usersEditor.obj
 0002:000033f0       ??_R2QPtrCollection@@8     1000b3f0     usersEditor.obj
 0002:000033f8       ??_R4QToolBar@@6BQObject@@@ 1000b3f8     usersEditor.obj
 0002:0000340c       ??_R3QToolBar@@8           1000b40c     usersEditor.obj
 0002:0000341c       ??_R2QToolBar@@8           1000b41c     usersEditor.obj
 0002:0000343c       ??_R1A@?0A@EA@QToolBar@@8  1000b43c     usersEditor.obj
 0002:00003458       ??_R1A@?0A@EA@QDockWindow@@8 1000b458     usersEditor.obj
 0002:00003474       ??_R3QDockWindow@@8        1000b474     usersEditor.obj
 0002:00003484       ??_R2QDockWindow@@8        1000b484     usersEditor.obj
 0002:000034a0       ??_R4QToolBar@@6BQPaintDevice@@@ 1000b4a0     usersEditor.obj
 0002:000034b4       ??_R4QPopupMenu@@6BQObject@@@ 1000b4b4     usersEditor.obj
 0002:000034c8       ??_R3QPopupMenu@@8         1000b4c8     usersEditor.obj
 0002:000034d8       ??_R2QPopupMenu@@8         1000b4d8     usersEditor.obj
 0002:000034f8       ??_R1A@?0A@EA@QPopupMenu@@8 1000b4f8     usersEditor.obj
 0002:00003514       ??_R1IM@?0A@EA@QMenuData@@8 1000b514     usersEditor.obj
 0002:00003530       ??_R3QMenuData@@8          1000b530     usersEditor.obj
 0002:00003540       ??_R2QMenuData@@8          1000b540     usersEditor.obj
 0002:00003548       ??_R1A@?0A@EA@QMenuData@@8 1000b548     usersEditor.obj
 0002:00003564       ??_R4QPopupMenu@@6BQPaintDevice@@@ 1000b564     usersEditor.obj
 0002:00003578       ??_R4QPopupMenu@@6B@       1000b578     usersEditor.obj
 0002:0000358c       ??_R4QAction@@6B@          1000b58c     usersEditor.obj
 0002:000035a0       ??_R3QAction@@8            1000b5a0     usersEditor.obj
 0002:000035b0       ??_R2QAction@@8            1000b5b0     usersEditor.obj
 0002:000035c0       ??_R1A@?0A@EA@QAction@@8   1000b5c0     usersEditor.obj
 0002:000035dc       ??_R4QGuardedPtrPrivate@@6B@ 1000b5dc     usersEditor.obj
 0002:000035f0       ??_R3QGuardedPtrPrivate@@8 1000b5f0     usersEditor.obj
 0002:00003600       ??_R2QGuardedPtrPrivate@@8 1000b600     usersEditor.obj
 0002:00003614       ??_R1A@?0A@EA@QGuardedPtrPrivate@@8 1000b614     usersEditor.obj
 0002:00003630       ??_R1CI@?0A@EA@QShared@@8  1000b630     usersEditor.obj
 0002:0000364c       ??_R4QDockWindowList@@6B@  1000b64c     usersEditor.obj
 0002:00003660       ??_R3QDockWindowList@@8    1000b660     usersEditor.obj
 0002:00003670       ??_R2QDockWindowList@@8    1000b670     usersEditor.obj
 0002:00003684       ??_R1A@?0A@EA@QDockWindowList@@8 1000b684     usersEditor.obj
 0002:000036a0       ??_R1A@?0A@EA@?$QPtrList@VQDockWindow@@@@8 1000b6a0     usersEditor.obj
 0002:000036bc       ??_R3?$QPtrList@VQDockWindow@@@@8 1000b6bc     usersEditor.obj
 0002:000036cc       ??_R2?$QPtrList@VQDockWindow@@@@8 1000b6cc     usersEditor.obj
 0002:000036dc       ??_R4QPopupMenuList@@6B@   1000b6dc     usersEditor.obj
 0002:000036f0       ??_R3QPopupMenuList@@8     1000b6f0     usersEditor.obj
 0002:00003700       ??_R2QPopupMenuList@@8     1000b700     usersEditor.obj
 0002:00003714       ??_R1A@?0A@EA@QPopupMenuList@@8 1000b714     usersEditor.obj
 0002:00003730       ??_R1A@?0A@EA@?$QPtrList@VQPopupMenu@@@@8 1000b730     usersEditor.obj
 0002:0000374c       ??_R3?$QPtrList@VQPopupMenu@@@@8 1000b74c     usersEditor.obj
 0002:0000375c       ??_R2?$QPtrList@VQPopupMenu@@@@8 1000b75c     usersEditor.obj
 0002:0000376c       ??_R4?$QPtrList@VQPopupMenu@@@@6B@ 1000b76c     usersEditor.obj
 0002:00003780       ??_R4config_plugin_base@@6BQObject@@@ 1000b780     usersEditor.obj
 0002:00003794       ??_R3config_plugin_base@@8 1000b794     usersEditor.obj
 0002:000037a4       ??_R2config_plugin_base@@8 1000b7a4     usersEditor.obj
 0002:000037bc       ??_R1A@?0A@EA@config_plugin_base@@8 1000b7bc     usersEditor.obj
 0002:000037d8       ??_R4config_plugin_base@@6BQPaintDevice@@@ 1000b7d8     usersEditor.obj
 0002:000037ec       ??_R1A@?0A@EA@QGDict@@8    1000b7ec     usersEditor.obj
 0002:00003808       ??_R3QGDict@@8             1000b808     usersEditor.obj
 0002:00003818       ??_R2QGDict@@8             1000b818     usersEditor.obj
 0002:00003824       ??_R4usersEditor@@6BQObject@@@ 1000b824     usersEditor.obj
 0002:00003838       ??_R3usersEditor@@8        1000b838     usersEditor.obj
 0002:00003848       ??_R2usersEditor@@8        1000b848     usersEditor.obj
 0002:00003864       ??_R1A@?0A@EA@usersEditor@@8 1000b864     usersEditor.obj
 0002:00003880       ??_R4usersEditor@@6BQPaintDevice@@@ 1000b880     usersEditor.obj
 0002:00003894       ??_R4?$QDict@VQAction@@@@6B@ 1000b894     usersEditor.obj
 0002:000038a8       ??_R3?$QDict@VQAction@@@@8 1000b8a8     usersEditor.obj
 0002:000038b8       ??_R2?$QDict@VQAction@@@@8 1000b8b8     usersEditor.obj
 0002:000038c8       ??_R1A@?0A@EA@?$QDict@VQAction@@@@8 1000b8c8     usersEditor.obj
 0002:000038e4       ??_R4QCheckTableItem@@6B@  1000b8e4     usersEditordlgimpl.obj
 0002:000038f8       ??_R3QCheckTableItem@@8    1000b8f8     usersEditordlgimpl.obj
 0002:00003908       ??_R2QCheckTableItem@@8    1000b908     usersEditordlgimpl.obj
 0002:00003918       ??_R1A@?0A@EA@QCheckTableItem@@8 1000b918     usersEditordlgimpl.obj
 0002:00003934       ??_R4usersEditorDlg@@6BQObject@@@ 1000b934     usersEditordlgimpl.obj
 0002:00003948       ??_R3usersEditorDlg@@8     1000b948     usersEditordlgimpl.obj
 0002:00003958       ??_R2usersEditorDlg@@8     1000b958     usersEditordlgimpl.obj
 0002:00003974       ??_R1A@?0A@EA@usersEditorDlg@@8 1000b974     usersEditordlgimpl.obj
 0002:00003990       ??_R1A@?0A@EA@usersEditorDlgBase@@8 1000b990     usersEditordlgimpl.obj
 0002:000039ac       ??_R3usersEditorDlgBase@@8 1000b9ac     usersEditordlgimpl.obj
 0002:000039bc       ??_R2usersEditorDlgBase@@8 1000b9bc     usersEditordlgimpl.obj
 0002:000039d4       ??_R4usersEditorDlg@@6BQPaintDevice@@@ 1000b9d4     usersEditordlgimpl.obj
 0002:000039e8       ??_R4?$QPtrList@H@@6B@     1000b9e8     usersEditordlgimpl.obj
 0002:000039fc       ??_R3?$QPtrList@H@@8       1000b9fc     usersEditordlgimpl.obj
 0002:00003a0c       ??_R2?$QPtrList@H@@8       1000ba0c     usersEditordlgimpl.obj
 0002:00003a1c       ??_R1A@?0A@EA@?$QPtrList@H@@8 1000ba1c     usersEditordlgimpl.obj
 0002:00003a38       ??_R4QVBoxLayout@@6BQObject@@@ 1000ba38     toolwindow.obj
 0002:00003a4c       ??_R3QVBoxLayout@@8        1000ba4c     toolwindow.obj
 0002:00003a5c       ??_R2QVBoxLayout@@8        1000ba5c     toolwindow.obj
 0002:00003a78       ??_R1A@?0A@EA@QVBoxLayout@@8 1000ba78     toolwindow.obj
 0002:00003a94       ??_R1A@?0A@EA@QBoxLayout@@8 1000ba94     toolwindow.obj
 0002:00003ab0       ??_R3QBoxLayout@@8         1000bab0     toolwindow.obj
 0002:00003ac0       ??_R2QBoxLayout@@8         1000bac0     toolwindow.obj
 0002:00003ad8       ??_R1A@?0A@EA@QLayout@@8   1000bad8     toolwindow.obj
 0002:00003af4       ??_R3QLayout@@8            1000baf4     toolwindow.obj
 0002:00003b04       ??_R2QLayout@@8            1000bb04     toolwindow.obj
 0002:00003b18       ??_R1CI@?0A@EA@QLayoutItem@@8 1000bb18     toolwindow.obj
 0002:00003b34       ??_R3QLayoutItem@@8        1000bb34     toolwindow.obj
 0002:00003b44       ??_R2QLayoutItem@@8        1000bb44     toolwindow.obj
 0002:00003b4c       ??_R1A@?0A@EA@QLayoutItem@@8 1000bb4c     toolwindow.obj
 0002:00003b68       ??_R4QVBoxLayout@@6BQLayoutItem@@@ 1000bb68     toolwindow.obj
 0002:00003b7c       ??_R4QLabel@@6BQObject@@@  1000bb7c     usersEditordlg.obj
 0002:00003b90       ??_R3QLabel@@8             1000bb90     usersEditordlg.obj
 0002:00003ba0       ??_R2QLabel@@8             1000bba0     usersEditordlg.obj
 0002:00003bbc       ??_R1A@?0A@EA@QLabel@@8    1000bbbc     usersEditordlg.obj
 0002:00003bd8       ??_R4QLabel@@6BQPaintDevice@@@ 1000bbd8     usersEditordlg.obj
 0002:00003bec       ??_R4usersEditorDlgBase@@6BQObject@@@ 1000bbec     usersEditordlg.obj
 0002:00003c00       ??_R4usersEditorDlgBase@@6BQPaintDevice@@@ 1000bc00     usersEditordlg.obj
 0002:00003c14       ??_R4type_info@@6B@        1000bc14     MSVCRT:ti_inst.obj
 0002:00003c28       ??_R3type_info@@8          1000bc28     MSVCRT:ti_inst.obj
 0002:00003c38       ??_R2type_info@@8          1000bc38     MSVCRT:ti_inst.obj
 0002:00003c40       ??_R1A@?0A@EA@type_info@@8 1000bc40     MSVCRT:ti_inst.obj
 0002:00003c5c       ___rtc_iaa                 1000bc5c     MSVCRT:initsect.obj
 0002:00003c60       ___rtc_izz                 1000bc60     MSVCRT:initsect.obj
 0002:00003c64       ___rtc_taa                 1000bc64     MSVCRT:initsect.obj
 0002:00003c68       ___rtc_tzz                 1000bc68     MSVCRT:initsect.obj
 0002:00004ab0       __IMPORT_DESCRIPTOR_config_icons 1000cab0     config_icons:config_icons.dll
 0002:00004ac4       __IMPORT_DESCRIPTOR_qt-mt323 1000cac4     qt-mt323:qt-mt323.dll
 0002:00004ad8       __IMPORT_DESCRIPTOR_MSVCR120 1000cad8     MSVCRT:MSVCR120.dll
 0002:00004aec       __IMPORT_DESCRIPTOR_KERNEL32 1000caec     kernel32:KERNEL32.dll
 0002:00004b00       __NULL_IMPORT_DESCRIPTOR   1000cb00     config_icons:config_icons.dll
 0003:00000074       ___security_cookie         10014074     MSVCRT:gs_cookie.obj
 0003:00000078       ___security_cookie_complement 10014078     MSVCRT:gs_cookie.obj
 0003:00000080       ___native_dllmain_reason   10014080     MSVCRT:natstart.obj
 0003:00000084       ??_R0?AVbncsTable@@@8      10014084     bncsTable.obj
 0003:0000009c       ??_R0?AVQTable@@@8         1001409c     bncsTable.obj
 0003:000000b4       ??_R0?AVQScrollView@@@8    100140b4     bncsTable.obj
 0003:000000d0       ??_R0?AVQFrame@@@8         100140d0     bncsTable.obj
 0003:000000e8       ??_R0?AVQWidget@@@8        100140e8     bncsTable.obj
 0003:00000100       ??_R0?AVQObject@@@8        10014100     bncsTable.obj
 0003:00000118       ??_R0?AVQt@@@8             10014118     bncsTable.obj
 0003:0000012c       ??_R0?AVQPaintDevice@@@8   1001412c     bncsTable.obj
 0003:00000148       ??_R0?AVQComboBox@@@8      10014148     panelsetsTableItem.obj
 0003:00000160       ??_R0?AVpanelsetsTableItem@@@8 10014160     panelsetsTableItem.obj
 0003:00000184       ??_R0?AVQTableItem@@@8     10014184     panelsetsTableItem.obj
 0003:000001a0       ??_R0?AVconfig_plugin_desc_base@@@8 100141a0     plugindesc.obj
 0003:000001c8       ??_R0?AVplugindesc@@@8     100141c8     plugindesc.obj
 0003:000001e4       ??_R0?AVuserLevelTableItem@@@8 100141e4     userLevelTableItem.obj
 0003:00000208       ??_R0?AUQShared@@@8        10014208     usersEditor.obj
 0003:00000220       ??_R0?AVQGList@@@8         10014220     usersEditor.obj
 0003:00000238       ??_R0?AVQPtrCollection@@@8 10014238     usersEditor.obj
 0003:00000258       ??_R0?AVQToolBar@@@8       10014258     usersEditor.obj
 0003:00000270       ??_R0?AVQDockWindow@@@8    10014270     usersEditor.obj
 0003:0000028c       ??_R0?AVQPopupMenu@@@8     1001428c     usersEditor.obj
 0003:000002a8       ??_R0?AVQMenuData@@@8      100142a8     usersEditor.obj
 0003:000002c0       ??_R0?AVQAction@@@8        100142c0     usersEditor.obj
 0003:000002d8       ??_R0?AVQGuardedPtrPrivate@@@8 100142d8     usersEditor.obj
 0003:000002fc       ??_R0?AVQDockWindowList@@@8 100142fc     usersEditor.obj
 0003:0000031c       ??_R0?AV?$QPtrList@VQDockWindow@@@@@8 1001431c     usersEditor.obj
 0003:00000344       ??_R0?AVQPopupMenuList@@@8 10014344     usersEditor.obj
 0003:00000364       ??_R0?AV?$QPtrList@VQPopupMenu@@@@@8 10014364     usersEditor.obj
 0003:0000038c       ??_R0?AVconfig_plugin_base@@@8 1001438c     usersEditor.obj
 0003:000003b0       ??_R0?AVQGDict@@@8         100143b0     usersEditor.obj
 0003:000003c8       ??_R0?AVusersEditor@@@8    100143c8     usersEditor.obj
 0003:000003e4       ??_R0?AV?$QDict@VQAction@@@@@8 100143e4     usersEditor.obj
 0003:00000408       ??_R0?AVQCheckTableItem@@@8 10014408     usersEditordlgimpl.obj
 0003:00000428       ??_R0?AVusersEditorDlg@@@8 10014428     usersEditordlgimpl.obj
 0003:00000448       ??_R0?AVusersEditorDlgBase@@@8 10014448     usersEditordlgimpl.obj
 0003:0000046c       ??_R0?AV?$QPtrList@H@@@8   1001446c     usersEditordlgimpl.obj
 0003:00000488       ??_R0?AVQVBoxLayout@@@8    10014488     toolwindow.obj
 0003:000004a4       ??_R0?AVQBoxLayout@@@8     100144a4     toolwindow.obj
 0003:000004c0       ??_R0?AVQLayout@@@8        100144c0     toolwindow.obj
 0003:000004d8       ??_R0?AVQLayoutItem@@@8    100144d8     toolwindow.obj
 0003:000004f4       ??_R0?AVQLabel@@@8         100144f4     usersEditordlg.obj
 0003:0000050c       ??_R0?AVtype_info@@@8      1001450c     MSVCRT:ti_inst.obj
 0003:00000528       ?metaObj@bncsTable@@0PAVQMetaObject@@A 10014528     moc_bncsTable.obj
 0003:00000530       ?metaObj@toolWindowBase@@0PAVQMetaObject@@A 10014530     moc_toolwindow.obj
 0003:00000538       ?metaObj@toolWindow@@0PAVQMetaObject@@A 10014538     moc_toolwindowimpl.obj
 0003:00000564       ?metaObj@usersEditor@@0PAVQMetaObject@@A 10014564     moc_usersEditor.obj
 0003:00000590       ?metaObj@usersEditorDlgBase@@0PAVQMetaObject@@A 10014590     moc_usersEditordlg.obj
 0003:00000598       ?metaObj@usersEditorDlg@@0PAVQMetaObject@@A 10014598     moc_usersEditordlgimpl.obj
 0003:000008e8       ?__type_info_root_node@@3U__type_info_node@@A 100148e8     MSVCRT:tncleanup.obj
 0003:000008f0       ___native_startup_lock     100148f0     <common>
 0003:000008f4       ___native_startup_state    100148f4     <common>
 0003:000008f8       ___dyn_tls_init_callback   100148f8     <common>
 0003:000008fc       ___onexitend               100148fc     <common>
 0003:00000900       ___onexitbegin             10014900     <common>

 entry point at        0001:000050e9

 Static symbols

 0001:00000000       ??__EcleanUp_bncsTable@@YAXXZ 10001000 f   moc_bncsTable.obj
 0001:00000021       ??__EcleanUp_toolWindowBase@@YAXXZ 10001021 f   moc_toolwindow.obj
 0001:00000042       ??__EcleanUp_toolWindow@@YAXXZ 10001042 f   moc_toolwindowimpl.obj
 0001:00000063       ??__EcleanUp_usersEditor@@YAXXZ 10001063 f   moc_usersEditor.obj
 0001:00000084       ??__EcleanUp_usersEditorDlgBase@@YAXXZ 10001084 f   moc_usersEditordlg.obj
 0001:000000a5       ??__EcleanUp_usersEditorDlg@@YAXXZ 100010a5 f   moc_usersEditordlgimpl.obj
 0001:00004ea3       _pre_c_init                10005ea3 f   MSVCRT:crtdll.obj
 0001:0000510c       ___DllMainCRTStartup       1000610c f   MSVCRT:crtdll.obj
 0001:00005390       $$000000                   10006390     MSVCRT:sehprolg4.obj
 0001:0000569c       __unwindfunclet$?doCopy@bncsTable@@QAEXXZ$0 1000669c f   bncsTable.obj
 0001:000056a5       __unwindfunclet$?doCopy@bncsTable@@QAEXXZ$1 100066a5 f   bncsTable.obj
 0001:000056ae       __unwindfunclet$?doCopy@bncsTable@@QAEXXZ$2 100066ae f   bncsTable.obj
 0001:000056b7       __unwindfunclet$?doCopy@bncsTable@@QAEXXZ$3 100066b7 f   bncsTable.obj
 0001:000056c0       __unwindfunclet$?doCopy@bncsTable@@QAEXXZ$4 100066c0 f   bncsTable.obj
 0001:000056c9       __ehhandler$?doCopy@bncsTable@@QAEXXZ 100066c9 f   bncsTable.obj
 0001:000056e4       __unwindfunclet$??1panelsetsTableItem@@UAE@XZ$0 100066e4 f   panelsetsTableItem.obj
 0001:000056e4       __unwindfunclet$??1userLevelTableItem@@UAE@XZ$0 100066e4 f   panelsetsTableItem.obj
 0001:000056ed       __ehhandler$??1panelsetsTableItem@@UAE@XZ 100066ed f   panelsetsTableItem.obj
 0001:000056ed       __ehhandler$??1userLevelTableItem@@UAE@XZ 100066ed f   panelsetsTableItem.obj
 0001:00005708       __unwindfunclet$?createEditor@panelsetsTableItem@@UBEPAVQWidget@@XZ$0 10006708 f   panelsetsTableItem.obj
 0001:00005712       __unwindfunclet$?createEditor@panelsetsTableItem@@UBEPAVQWidget@@XZ$1 10006712 f   panelsetsTableItem.obj
 0001:0000571b       __unwindfunclet$?createEditor@panelsetsTableItem@@UBEPAVQWidget@@XZ$2 1000671b f   panelsetsTableItem.obj
 0001:00005724       __unwindfunclet$?createEditor@panelsetsTableItem@@UBEPAVQWidget@@XZ$3 10006724 f   panelsetsTableItem.obj
 0001:0000572d       __unwindfunclet$?createEditor@panelsetsTableItem@@UBEPAVQWidget@@XZ$4 1000672d f   panelsetsTableItem.obj
 0001:00005736       __unwindfunclet$?createEditor@panelsetsTableItem@@UBEPAVQWidget@@XZ$5 10006736 f   panelsetsTableItem.obj
 0001:0000573f       __unwindfunclet$?createEditor@panelsetsTableItem@@UBEPAVQWidget@@XZ$6 1000673f f   panelsetsTableItem.obj
 0001:00005748       __unwindfunclet$?createEditor@panelsetsTableItem@@UBEPAVQWidget@@XZ$7 10006748 f   panelsetsTableItem.obj
 0001:00005751       __unwindfunclet$?createEditor@panelsetsTableItem@@UBEPAVQWidget@@XZ$8 10006751 f   panelsetsTableItem.obj
 0001:0000575a       __unwindfunclet$?createEditor@panelsetsTableItem@@UBEPAVQWidget@@XZ$9 1000675a f   panelsetsTableItem.obj
 0001:00005763       __unwindfunclet$?createEditor@panelsetsTableItem@@UBEPAVQWidget@@XZ$10 10006763 f   panelsetsTableItem.obj
 0001:0000576c       __unwindfunclet$?createEditor@panelsetsTableItem@@UBEPAVQWidget@@XZ$11 1000676c f   panelsetsTableItem.obj
 0001:00005775       __unwindfunclet$?createEditor@panelsetsTableItem@@UBEPAVQWidget@@XZ$12 10006775 f   panelsetsTableItem.obj
 0001:0000577e       __ehhandler$?createEditor@panelsetsTableItem@@UBEPAVQWidget@@XZ 1000677e f   panelsetsTableItem.obj
 0001:00005799       __unwindfunclet$?keys@plugindesc@@UAE?AVQStringList@@ABVQString@@0@Z$0 10006799 f   plugindesc.obj
 0001:000057b3       __unwindfunclet$?keys@plugindesc@@UAE?AVQStringList@@ABVQString@@0@Z$1 100067b3 f   plugindesc.obj
 0001:000057bc       __ehhandler$?keys@plugindesc@@UAE?AVQStringList@@ABVQString@@0@Z 100067bc f   plugindesc.obj
 0001:000057d7       __unwindfunclet$??0userLevelTableItem@@QAE@ABVQString@@PAVQTable@@W4EditType@QTableItem@@0@Z$0 100067d7 f   userLevelTableItem.obj
 0001:000057d7       __unwindfunclet$??0panelsetsTableItem@@QAE@ABVQString@@PAVQTable@@W4EditType@QTableItem@@0@Z$0 100067d7 f   userLevelTableItem.obj
 0001:000057e0       __unwindfunclet$??0userLevelTableItem@@QAE@ABVQString@@PAVQTable@@W4EditType@QTableItem@@0@Z$1 100067e0 f   userLevelTableItem.obj
 0001:000057e0       __unwindfunclet$??0panelsetsTableItem@@QAE@ABVQString@@PAVQTable@@W4EditType@QTableItem@@0@Z$1 100067e0 f   userLevelTableItem.obj
 0001:000057ec       __ehhandler$??0userLevelTableItem@@QAE@ABVQString@@PAVQTable@@W4EditType@QTableItem@@0@Z 100067ec f   userLevelTableItem.obj
 0001:000057ec       __ehhandler$??0panelsetsTableItem@@QAE@ABVQString@@PAVQTable@@W4EditType@QTableItem@@0@Z 100067ec f   userLevelTableItem.obj
 0001:00005807       __unwindfunclet$?createEditor@userLevelTableItem@@UBEPAVQWidget@@XZ$0 10006807 f   userLevelTableItem.obj
 0001:00005811       __unwindfunclet$?createEditor@userLevelTableItem@@UBEPAVQWidget@@XZ$1 10006811 f   userLevelTableItem.obj
 0001:0000581a       __unwindfunclet$?createEditor@userLevelTableItem@@UBEPAVQWidget@@XZ$2 1000681a f   userLevelTableItem.obj
 0001:00005823       __unwindfunclet$?createEditor@userLevelTableItem@@UBEPAVQWidget@@XZ$3 10006823 f   userLevelTableItem.obj
 0001:0000582c       __unwindfunclet$?createEditor@userLevelTableItem@@UBEPAVQWidget@@XZ$4 1000682c f   userLevelTableItem.obj
 0001:00005835       __unwindfunclet$?createEditor@userLevelTableItem@@UBEPAVQWidget@@XZ$5 10006835 f   userLevelTableItem.obj
 0001:0000583e       __unwindfunclet$?createEditor@userLevelTableItem@@UBEPAVQWidget@@XZ$6 1000683e f   userLevelTableItem.obj
 0001:00005847       __unwindfunclet$?createEditor@userLevelTableItem@@UBEPAVQWidget@@XZ$7 10006847 f   userLevelTableItem.obj
 0001:00005850       __ehhandler$?createEditor@userLevelTableItem@@UBEPAVQWidget@@XZ 10006850 f   userLevelTableItem.obj
 0001:0000586b       __unwindfunclet$?setContentFromEditor@panelsetsTableItem@@UAEXPAVQWidget@@@Z$0 1000686b f   userLevelTableItem.obj
 0001:0000586b       __unwindfunclet$?setContentFromEditor@userLevelTableItem@@UAEXPAVQWidget@@@Z$0 1000686b f   userLevelTableItem.obj
 0001:00005874       __unwindfunclet$?setContentFromEditor@panelsetsTableItem@@UAEXPAVQWidget@@@Z$1 10006874 f   userLevelTableItem.obj
 0001:00005874       __unwindfunclet$?setContentFromEditor@userLevelTableItem@@UAEXPAVQWidget@@@Z$1 10006874 f   userLevelTableItem.obj
 0001:0000587d       __ehhandler$?setContentFromEditor@panelsetsTableItem@@UAEXPAVQWidget@@@Z 1000687d f   userLevelTableItem.obj
 0001:0000587d       __ehhandler$?setContentFromEditor@userLevelTableItem@@UAEXPAVQWidget@@@Z 1000687d f   userLevelTableItem.obj
 0001:00005898       __unwindfunclet$??0config_plugin_base@@QAE@ABVQString@@00@Z$0 10006898 f   usersEditor.obj
 0001:000058a1       __unwindfunclet$??0config_plugin_base@@QAE@ABVQString@@00@Z$1 100068a1 f   usersEditor.obj
 0001:000058ad       __unwindfunclet$??0config_plugin_base@@QAE@ABVQString@@00@Z$2 100068ad f   usersEditor.obj
 0001:000058b9       __unwindfunclet$??0config_plugin_base@@QAE@ABVQString@@00@Z$3 100068b9 f   usersEditor.obj
 0001:000058c5       __ehhandler$??0config_plugin_base@@QAE@ABVQString@@00@Z 100068c5 f   usersEditor.obj
 0001:000058e0       __unwindfunclet$??0usersEditor@@QAE@ABVQString@@00@Z$0 100068e0 f   usersEditor.obj
 0001:000058e8       __unwindfunclet$??0usersEditor@@QAE@ABVQString@@00@Z$1 100068e8 f   usersEditor.obj
 0001:000058f3       __unwindfunclet$??0usersEditor@@QAE@ABVQString@@00@Z$2 100068f3 f   usersEditor.obj
 0001:000058fe       __unwindfunclet$??0usersEditor@@QAE@ABVQString@@00@Z$3 100068fe f   usersEditor.obj
 0001:0000590c       __unwindfunclet$??0usersEditor@@QAE@ABVQString@@00@Z$4 1000690c f   usersEditor.obj
 0001:0000591a       __unwindfunclet$??0usersEditor@@QAE@ABVQString@@00@Z$5 1000691a f   usersEditor.obj
 0001:00005929       __unwindfunclet$??0usersEditor@@QAE@ABVQString@@00@Z$6 10006929 f   usersEditor.obj
 0001:00005933       __unwindfunclet$??0usersEditor@@QAE@ABVQString@@00@Z$7 10006933 f   usersEditor.obj
 0001:0000593d       __unwindfunclet$??0usersEditor@@QAE@ABVQString@@00@Z$8 1000693d f   usersEditor.obj
 0001:00005957       __unwindfunclet$??0usersEditor@@QAE@ABVQString@@00@Z$9 10006957 f   usersEditor.obj
 0001:00005961       __unwindfunclet$??0usersEditor@@QAE@ABVQString@@00@Z$10 10006961 f   usersEditor.obj
 0001:0000596b       __unwindfunclet$??0usersEditor@@QAE@ABVQString@@00@Z$11 1000696b f   usersEditor.obj
 0001:00005985       __unwindfunclet$??0usersEditor@@QAE@ABVQString@@00@Z$12 10006985 f   usersEditor.obj
 0001:0000599f       __unwindfunclet$??0usersEditor@@QAE@ABVQString@@00@Z$13 1000699f f   usersEditor.obj
 0001:000059b9       __unwindfunclet$??0usersEditor@@QAE@ABVQString@@00@Z$14 100069b9 f   usersEditor.obj
 0001:000059d3       __unwindfunclet$??0usersEditor@@QAE@ABVQString@@00@Z$16 100069d3 f   usersEditor.obj
 0001:000059dc       __unwindfunclet$??0usersEditor@@QAE@ABVQString@@00@Z$17 100069dc f   usersEditor.obj
 0001:000059e5       __unwindfunclet$??0usersEditor@@QAE@ABVQString@@00@Z$18 100069e5 f   usersEditor.obj
 0001:000059ee       __unwindfunclet$??0usersEditor@@QAE@ABVQString@@00@Z$19 100069ee f   usersEditor.obj
 0001:000059f8       __unwindfunclet$??0usersEditor@@QAE@ABVQString@@00@Z$20 100069f8 f   usersEditor.obj
 0001:00005a12       __unwindfunclet$??0usersEditor@@QAE@ABVQString@@00@Z$21 10006a12 f   usersEditor.obj
 0001:00005a2c       __unwindfunclet$??0usersEditor@@QAE@ABVQString@@00@Z$22 10006a2c f   usersEditor.obj
 0001:00005a4b       __unwindfunclet$??0usersEditor@@QAE@ABVQString@@00@Z$23 10006a4b f   usersEditor.obj
 0001:00005a6a       __unwindfunclet$??0usersEditor@@QAE@ABVQString@@00@Z$25 10006a6a f   usersEditor.obj
 0001:00005a73       __unwindfunclet$??0usersEditor@@QAE@ABVQString@@00@Z$26 10006a73 f   usersEditor.obj
 0001:00005a7c       __unwindfunclet$??0usersEditor@@QAE@ABVQString@@00@Z$27 10006a7c f   usersEditor.obj
 0001:00005a85       __unwindfunclet$??0usersEditor@@QAE@ABVQString@@00@Z$28 10006a85 f   usersEditor.obj
 0001:00005a8e       __unwindfunclet$??0usersEditor@@QAE@ABVQString@@00@Z$29 10006a8e f   usersEditor.obj
 0001:00005a97       __ehhandler$??0usersEditor@@QAE@ABVQString@@00@Z 10006a97 f   usersEditor.obj
 0001:00005ab2       __unwindfunclet$??1?$QDict@VQAction@@@@UAE@XZ$0 10006ab2 f   usersEditor.obj
 0001:00005abb       __ehhandler$??1?$QDict@VQAction@@@@UAE@XZ 10006abb f   usersEditor.obj
 0001:00005ad6       __unwindfunclet$??1QDockWindowList@@UAE@XZ$0 10006ad6 f   usersEditor.obj
 0001:00005adf       __unwindfunclet$??1QDockWindowList@@UAE@XZ$1 10006adf f   usersEditor.obj
 0001:00005ae8       __ehhandler$??1QDockWindowList@@UAE@XZ 10006ae8 f   usersEditor.obj
 0001:00005b03       __unwindfunclet$??1QPopupMenuList@@UAE@XZ$0 10006b03 f   usersEditor.obj
 0001:00005b0b       __ehhandler$??1QPopupMenuList@@UAE@XZ 10006b0b f   usersEditor.obj
 0001:00005b26       __unwindfunclet$??1config_plugin_base@@UAE@XZ$0 10006b26 f   usersEditor.obj
 0001:00005b2f       __unwindfunclet$??1config_plugin_base@@UAE@XZ$1 10006b2f f   usersEditor.obj
 0001:00005b3b       __unwindfunclet$??1config_plugin_base@@UAE@XZ$2 10006b3b f   usersEditor.obj
 0001:00005b47       __ehhandler$??1config_plugin_base@@UAE@XZ 10006b47 f   usersEditor.obj
 0001:00005b62       __unwindfunclet$??1usersEditor@@UAE@XZ$0 10006b62 f   usersEditor.obj
 0001:00005b6a       __unwindfunclet$??1usersEditor@@UAE@XZ$1 10006b6a f   usersEditor.obj
 0001:00005b75       __unwindfunclet$??1usersEditor@@UAE@XZ$2 10006b75 f   usersEditor.obj
 0001:00005b80       __unwindfunclet$??1usersEditor@@UAE@XZ$3 10006b80 f   usersEditor.obj
 0001:00005b8e       __unwindfunclet$??1usersEditor@@UAE@XZ$4 10006b8e f   usersEditor.obj
 0001:00005b9c       __unwindfunclet$??1usersEditor@@UAE@XZ$5 10006b9c f   usersEditor.obj
 0001:00005bab       __ehhandler$??1usersEditor@@UAE@XZ 10006bab f   usersEditor.obj
 0001:00005bc6       __unwindfunclet$??0?$QGuardedPtr@VQDockWindow@@@@QAE@XZ$0 10006bc6 f   usersEditor.obj
 0001:00005bc6       __unwindfunclet$?create@plugindesc@@UAEPAVconfig_plugin_base@@ABVQString@@00@Z$0 10006bc6 f   usersEditor.obj
 0001:00005bc6       __unwindfunclet$??4?$QGuardedPtr@VQPopupMenu@@@@QAEAAV0@PAVQPopupMenu@@@Z$0 10006bc6 f   usersEditor.obj
 0001:00005bc6       __unwindfunclet$??0?$QGuardedPtr@VQPopupMenu@@@@QAE@XZ$0 10006bc6 f   usersEditor.obj
 0001:00005bc6       __unwindfunclet$??4?$QGuardedPtr@VQDockWindow@@@@QAEAAV0@PAVQDockWindow@@@Z$0 10006bc6 f   usersEditor.obj
 0001:00005bd0       __ehhandler$??0?$QGuardedPtr@VQPopupMenu@@@@QAE@XZ 10006bd0 f   usersEditor.obj
 0001:00005bd0       __ehhandler$?create@plugindesc@@UAEPAVconfig_plugin_base@@ABVQString@@00@Z 10006bd0 f   usersEditor.obj
 0001:00005bd0       __ehhandler$??0?$QGuardedPtr@VQDockWindow@@@@QAE@XZ 10006bd0 f   usersEditor.obj
 0001:00005bd0       __ehhandler$??4?$QGuardedPtr@VQPopupMenu@@@@QAEAAV0@PAVQPopupMenu@@@Z 10006bd0 f   usersEditor.obj
 0001:00005bd0       __ehhandler$??4?$QGuardedPtr@VQDockWindow@@@@QAEAAV0@PAVQDockWindow@@@Z 10006bd0 f   usersEditor.obj
 0001:00005beb       __unwindfunclet$?about@config_plugin_base@@UAE?AVQString@@XZ$0 10006beb f   usersEditor.obj
 0001:00005bf4       __unwindfunclet$?about@config_plugin_base@@UAE?AVQString@@XZ$1 10006bf4 f   usersEditor.obj
 0001:00005c0e       __ehhandler$?about@config_plugin_base@@UAE?AVQString@@XZ 10006c0e f   usersEditor.obj
 0001:00005c29       __unwindfunclet$?about@usersEditor@@UAE?AVQString@@XZ$0 10006c29 f   usersEditor.obj
 0001:00005c32       __unwindfunclet$?about@usersEditor@@UAE?AVQString@@XZ$1 10006c32 f   usersEditor.obj
 0001:00005c3b       __unwindfunclet$?about@usersEditor@@UAE?AVQString@@XZ$2 10006c3b f   usersEditor.obj
 0001:00005c44       __unwindfunclet$?about@usersEditor@@UAE?AVQString@@XZ$3 10006c44 f   usersEditor.obj
 0001:00005c4d       __unwindfunclet$?about@usersEditor@@UAE?AVQString@@XZ$4 10006c4d f   usersEditor.obj
 0001:00005c67       __ehhandler$?about@usersEditor@@UAE?AVQString@@XZ 10006c67 f   usersEditor.obj
 0001:00005c82       __unwindfunclet$?activate@usersEditor@@UAEX_N@Z$0 10006c82 f   usersEditor.obj
 0001:00005c8b       __unwindfunclet$?activate@usersEditor@@UAEX_N@Z$2 10006c8b f   usersEditor.obj
 0001:00005c94       __unwindfunclet$?activate@usersEditor@@UAEX_N@Z$4 10006c94 f   usersEditor.obj
 0001:00005c9d       __unwindfunclet$?activate@usersEditor@@UAEX_N@Z$5 10006c9d f   usersEditor.obj
 0001:00005ca6       __unwindfunclet$?activate@usersEditor@@UAEX_N@Z$6 10006ca6 f   usersEditor.obj
 0001:00005caf       __unwindfunclet$?activate@usersEditor@@UAEX_N@Z$7 10006caf f   usersEditor.obj
 0001:00005cb8       __unwindfunclet$?activate@usersEditor@@UAEX_N@Z$8 10006cb8 f   usersEditor.obj
 0001:00005cc1       __unwindfunclet$?activate@usersEditor@@UAEX_N@Z$9 10006cc1 f   usersEditor.obj
 0001:00005cca       __unwindfunclet$?activate@usersEditor@@UAEX_N@Z$10 10006cca f   usersEditor.obj
 0001:00005cd3       __unwindfunclet$?activate@usersEditor@@UAEX_N@Z$11 10006cd3 f   usersEditor.obj
 0001:00005cdc       __unwindfunclet$?activate@usersEditor@@UAEX_N@Z$12 10006cdc f   usersEditor.obj
 0001:00005ce5       __unwindfunclet$?activate@usersEditor@@UAEX_N@Z$13 10006ce5 f   usersEditor.obj
 0001:00005cee       __unwindfunclet$?activate@usersEditor@@UAEX_N@Z$14 10006cee f   usersEditor.obj
 0001:00005cf7       __unwindfunclet$?activate@usersEditor@@UAEX_N@Z$15 10006cf7 f   usersEditor.obj
 0001:00005d00       __unwindfunclet$?activate@usersEditor@@UAEX_N@Z$16 10006d00 f   usersEditor.obj
 0001:00005d09       __ehhandler$?activate@usersEditor@@UAEX_N@Z 10006d09 f   usersEditor.obj
 0001:00005d24       __unwindfunclet$?apply@usersEditor@@UAEXXZ$0 10006d24 f   usersEditor.obj
 0001:00005d2d       __unwindfunclet$?apply@usersEditor@@UAEXXZ$1 10006d2d f   usersEditor.obj
 0001:00005d36       __unwindfunclet$?apply@usersEditor@@UAEXXZ$2 10006d36 f   usersEditor.obj
 0001:00005d3f       __ehhandler$?apply@usersEditor@@UAEXXZ 10006d3f f   usersEditor.obj
 0001:00005d5a       __unwindfunclet$?db@@YAXABVQString@@@Z$0 10006d5a f   usersEditor.obj
 0001:00005d63       __ehhandler$?db@@YAXABVQString@@@Z 10006d63 f   usersEditor.obj
 0001:00005d7e       __unwindfunclet$?menus@usersEditor@@UAE?AVQPopupMenuList@@XZ$0 10006d7e f   usersEditor.obj
 0001:00005d97       __ehhandler$?menus@usersEditor@@UAE?AVQPopupMenuList@@XZ 10006d97 f   usersEditor.obj
 0001:00005db2       __unwindfunclet$?navigate@usersEditor@@UAEXABVQString@@0@Z$0 10006db2 f   usersEditor.obj
 0001:00005dbb       __unwindfunclet$?navigate@usersEditor@@UAEXABVQString@@0@Z$1 10006dbb f   usersEditor.obj
 0001:00005dc4       __unwindfunclet$?navigate@usersEditor@@UAEXABVQString@@0@Z$2 10006dc4 f   usersEditor.obj
 0001:00005dcd       __ehhandler$?navigate@usersEditor@@UAEXABVQString@@0@Z 10006dcd f   usersEditor.obj
 0001:00005de8       __unwindfunclet$?reply@usersEditor@@UAEXPAVresponse@@@Z$0 10006de8 f   usersEditor.obj
 0001:00005df1       __unwindfunclet$?reply@usersEditor@@UAEXPAVresponse@@@Z$1 10006df1 f   usersEditor.obj
 0001:00005dfa       __unwindfunclet$?reply@usersEditor@@UAEXPAVresponse@@@Z$2 10006dfa f   usersEditor.obj
 0001:00005e03       __unwindfunclet$?reply@usersEditor@@UAEXPAVresponse@@@Z$3 10006e03 f   usersEditor.obj
 0001:00005e0c       __unwindfunclet$?reply@usersEditor@@UAEXPAVresponse@@@Z$4 10006e0c f   usersEditor.obj
 0001:00005e15       __unwindfunclet$?reply@usersEditor@@UAEXPAVresponse@@@Z$5 10006e15 f   usersEditor.obj
 0001:00005e1e       __unwindfunclet$?reply@usersEditor@@UAEXPAVresponse@@@Z$6 10006e1e f   usersEditor.obj
 0001:00005e27       __unwindfunclet$?reply@usersEditor@@UAEXPAVresponse@@@Z$7 10006e27 f   usersEditor.obj
 0001:00005e30       __unwindfunclet$?reply@usersEditor@@UAEXPAVresponse@@@Z$8 10006e30 f   usersEditor.obj
 0001:00005e39       __unwindfunclet$?reply@usersEditor@@UAEXPAVresponse@@@Z$9 10006e39 f   usersEditor.obj
 0001:00005e42       __unwindfunclet$?reply@usersEditor@@UAEXPAVresponse@@@Z$10 10006e42 f   usersEditor.obj
 0001:00005e4b       __unwindfunclet$?reply@usersEditor@@UAEXPAVresponse@@@Z$11 10006e4b f   usersEditor.obj
 0001:00005e54       __unwindfunclet$?reply@usersEditor@@UAEXPAVresponse@@@Z$12 10006e54 f   usersEditor.obj
 0001:00005e5d       __unwindfunclet$?reply@usersEditor@@UAEXPAVresponse@@@Z$13 10006e5d f   usersEditor.obj
 0001:00005e66       __unwindfunclet$?reply@usersEditor@@UAEXPAVresponse@@@Z$14 10006e66 f   usersEditor.obj
 0001:00005e6f       __unwindfunclet$?reply@usersEditor@@UAEXPAVresponse@@@Z$16 10006e6f f   usersEditor.obj
 0001:00005e78       __ehhandler$?reply@usersEditor@@UAEXPAVresponse@@@Z 10006e78 f   usersEditor.obj
 0001:00005e93       __unwindfunclet$?toolbars@usersEditor@@UAE?AVQDockWindowList@@XZ$0 10006e93 f   usersEditor.obj
 0001:00005eac       __ehhandler$?toolbars@usersEditor@@UAE?AVQDockWindowList@@XZ 10006eac f   usersEditor.obj
 0001:00005ec7       __unwindfunclet$??0usersEditorDlg@@QAE@ABVQString@@PAVQWidget@@PBDI@Z$0 10006ec7 f   usersEditordlgimpl.obj
 0001:00005ecf       __unwindfunclet$??0usersEditorDlg@@QAE@ABVQString@@PAVQWidget@@PBDI@Z$1 10006ecf f   usersEditordlgimpl.obj
 0001:00005edb       __unwindfunclet$??0usersEditorDlg@@QAE@ABVQString@@PAVQWidget@@PBDI@Z$2 10006edb f   usersEditordlgimpl.obj
 0001:00005ee7       __unwindfunclet$??0usersEditorDlg@@QAE@ABVQString@@PAVQWidget@@PBDI@Z$3 10006ee7 f   usersEditordlgimpl.obj
 0001:00005ef1       __unwindfunclet$??0usersEditorDlg@@QAE@ABVQString@@PAVQWidget@@PBDI@Z$4 10006ef1 f   usersEditordlgimpl.obj
 0001:00005efa       __unwindfunclet$??0usersEditorDlg@@QAE@ABVQString@@PAVQWidget@@PBDI@Z$5 10006efa f   usersEditordlgimpl.obj
 0001:00005f03       __unwindfunclet$??0usersEditorDlg@@QAE@ABVQString@@PAVQWidget@@PBDI@Z$6 10006f03 f   usersEditordlgimpl.obj
 0001:00005f0c       __unwindfunclet$??0usersEditorDlg@@QAE@ABVQString@@PAVQWidget@@PBDI@Z$7 10006f0c f   usersEditordlgimpl.obj
 0001:00005f15       __unwindfunclet$??0usersEditorDlg@@QAE@ABVQString@@PAVQWidget@@PBDI@Z$8 10006f15 f   usersEditordlgimpl.obj
 0001:00005f1e       __unwindfunclet$??0usersEditorDlg@@QAE@ABVQString@@PAVQWidget@@PBDI@Z$9 10006f1e f   usersEditordlgimpl.obj
 0001:00005f27       __unwindfunclet$??0usersEditorDlg@@QAE@ABVQString@@PAVQWidget@@PBDI@Z$10 10006f27 f   usersEditordlgimpl.obj
 0001:00005f30       __unwindfunclet$??0usersEditorDlg@@QAE@ABVQString@@PAVQWidget@@PBDI@Z$11 10006f30 f   usersEditordlgimpl.obj
 0001:00005f39       __ehhandler$??0usersEditorDlg@@QAE@ABVQString@@PAVQWidget@@PBDI@Z 10006f39 f   usersEditordlgimpl.obj
 0001:00005f54       __unwindfunclet$??1?$QPtrList@VQPopupMenu@@@@UAE@XZ$0 10006f54 f   usersEditordlgimpl.obj
 0001:00005f54       __unwindfunclet$??1?$QPtrList@H@@UAE@XZ$0 10006f54 f   usersEditordlgimpl.obj
 0001:00005f5d       __ehhandler$??1?$QPtrList@H@@UAE@XZ 10006f5d f   usersEditordlgimpl.obj
 0001:00005f5d       __ehhandler$??1?$QPtrList@VQPopupMenu@@@@UAE@XZ 10006f5d f   usersEditordlgimpl.obj
 0001:00005f78       __unwindfunclet$??1usersEditorDlg@@UAE@XZ$0 10006f78 f   usersEditordlgimpl.obj
 0001:00005f80       __unwindfunclet$??1usersEditorDlg@@UAE@XZ$1 10006f80 f   usersEditordlgimpl.obj
 0001:00005f8c       __ehhandler$??1usersEditorDlg@@UAE@XZ 10006f8c f   usersEditordlgimpl.obj
 0001:00005fa7       __unwindfunclet$?addUser@usersEditorDlg@@QAEXXZ$0 10006fa7 f   usersEditordlgimpl.obj
 0001:00005fb1       __unwindfunclet$?addUser@usersEditorDlg@@QAEXXZ$1 10006fb1 f   usersEditordlgimpl.obj
 0001:00005fcb       __unwindfunclet$?addUser@usersEditorDlg@@QAEXXZ$2 10006fcb f   usersEditordlgimpl.obj
 0001:00005fd5       __unwindfunclet$?addUser@usersEditorDlg@@QAEXXZ$3 10006fd5 f   usersEditordlgimpl.obj
 0001:00005fef       __unwindfunclet$?addUser@usersEditorDlg@@QAEXXZ$4 10006fef f   usersEditordlgimpl.obj
 0001:00005ff9       __unwindfunclet$?addUser@usersEditorDlg@@QAEXXZ$5 10006ff9 f   usersEditordlgimpl.obj
 0001:00006013       __unwindfunclet$?addUser@usersEditorDlg@@QAEXXZ$6 10007013 f   usersEditordlgimpl.obj
 0001:0000601d       __unwindfunclet$?addUser@usersEditorDlg@@QAEXXZ$7 1000701d f   usersEditordlgimpl.obj
 0001:00006037       __unwindfunclet$?addUser@usersEditorDlg@@QAEXXZ$8 10007037 f   usersEditordlgimpl.obj
 0001:00006041       __unwindfunclet$?addUser@usersEditorDlg@@QAEXXZ$9 10007041 f   usersEditordlgimpl.obj
 0001:0000605b       __ehhandler$?addUser@usersEditorDlg@@QAEXXZ 1000705b f   usersEditordlgimpl.obj
 0001:00006076       __unwindfunclet$?deleteUser@usersEditorDlg@@QAEXXZ$0 10007076 f   usersEditordlgimpl.obj
 0001:0000607e       __ehhandler$?deleteUser@usersEditorDlg@@QAEXXZ 1000707e f   usersEditordlgimpl.obj
 0001:00006099       __unwindfunclet$?load@usersEditorDlg@@QAE_NABVQString@@@Z$0 10007099 f   usersEditordlgimpl.obj
 0001:000060a2       __unwindfunclet$?load@usersEditorDlg@@QAE_NABVQString@@@Z$1 100070a2 f   usersEditordlgimpl.obj
 0001:000060ae       __unwindfunclet$?load@usersEditorDlg@@QAE_NABVQString@@@Z$2 100070ae f   usersEditordlgimpl.obj
 0001:000060b7       __unwindfunclet$?load@usersEditorDlg@@QAE_NABVQString@@@Z$3 100070b7 f   usersEditordlgimpl.obj
 0001:000060c0       __unwindfunclet$?load@usersEditorDlg@@QAE_NABVQString@@@Z$4 100070c0 f   usersEditordlgimpl.obj
 0001:000060c9       __unwindfunclet$?load@usersEditorDlg@@QAE_NABVQString@@@Z$5 100070c9 f   usersEditordlgimpl.obj
 0001:000060d2       __unwindfunclet$?load@usersEditorDlg@@QAE_NABVQString@@@Z$6 100070d2 f   usersEditordlgimpl.obj
 0001:000060db       __unwindfunclet$?load@usersEditorDlg@@QAE_NABVQString@@@Z$7 100070db f   usersEditordlgimpl.obj
 0001:000060e4       __unwindfunclet$?load@usersEditorDlg@@QAE_NABVQString@@@Z$8 100070e4 f   usersEditordlgimpl.obj
 0001:000060ed       __unwindfunclet$?load@usersEditorDlg@@QAE_NABVQString@@@Z$9 100070ed f   usersEditordlgimpl.obj
 0001:000060f7       __unwindfunclet$?load@usersEditorDlg@@QAE_NABVQString@@@Z$10 100070f7 f   usersEditordlgimpl.obj
 0001:00006111       __unwindfunclet$?load@usersEditorDlg@@QAE_NABVQString@@@Z$11 10007111 f   usersEditordlgimpl.obj
 0001:0000612b       __unwindfunclet$?load@usersEditorDlg@@QAE_NABVQString@@@Z$12 1000712b f   usersEditordlgimpl.obj
 0001:00006135       __unwindfunclet$?load@usersEditorDlg@@QAE_NABVQString@@@Z$13 10007135 f   usersEditordlgimpl.obj
 0001:0000614f       __unwindfunclet$?load@usersEditorDlg@@QAE_NABVQString@@@Z$14 1000714f f   usersEditordlgimpl.obj
 0001:00006169       __unwindfunclet$?load@usersEditorDlg@@QAE_NABVQString@@@Z$15 10007169 f   usersEditordlgimpl.obj
 0001:00006173       __unwindfunclet$?load@usersEditorDlg@@QAE_NABVQString@@@Z$16 10007173 f   usersEditordlgimpl.obj
 0001:0000618d       __unwindfunclet$?load@usersEditorDlg@@QAE_NABVQString@@@Z$17 1000718d f   usersEditordlgimpl.obj
 0001:000061a7       __unwindfunclet$?load@usersEditorDlg@@QAE_NABVQString@@@Z$18 100071a7 f   usersEditordlgimpl.obj
 0001:000061b1       __unwindfunclet$?load@usersEditorDlg@@QAE_NABVQString@@@Z$19 100071b1 f   usersEditordlgimpl.obj
 0001:000061cb       __unwindfunclet$?load@usersEditorDlg@@QAE_NABVQString@@@Z$20 100071cb f   usersEditordlgimpl.obj
 0001:000061d4       __unwindfunclet$?load@usersEditorDlg@@QAE_NABVQString@@@Z$21 100071d4 f   usersEditordlgimpl.obj
 0001:000061dd       __unwindfunclet$?load@usersEditorDlg@@QAE_NABVQString@@@Z$22 100071dd f   usersEditordlgimpl.obj
 0001:000061e7       __unwindfunclet$?load@usersEditorDlg@@QAE_NABVQString@@@Z$23 100071e7 f   usersEditordlgimpl.obj
 0001:00006206       __unwindfunclet$?load@usersEditorDlg@@QAE_NABVQString@@@Z$24 10007206 f   usersEditordlgimpl.obj
 0001:0000620f       __unwindfunclet$?load@usersEditorDlg@@QAE_NABVQString@@@Z$25 1000720f f   usersEditordlgimpl.obj
 0001:00006218       __unwindfunclet$?load@usersEditorDlg@@QAE_NABVQString@@@Z$26 10007218 f   usersEditordlgimpl.obj
 0001:00006221       __ehhandler$?load@usersEditorDlg@@QAE_NABVQString@@@Z 10007221 f   usersEditordlgimpl.obj
 0001:0000623f       __unwindfunclet$?save@usersEditorDlg@@QAEXABVQString@@@Z$0 1000723f f   usersEditordlgimpl.obj
 0001:00006248       __unwindfunclet$?save@usersEditorDlg@@QAEXABVQString@@@Z$1 10007248 f   usersEditordlgimpl.obj
 0001:00006254       __unwindfunclet$?save@usersEditorDlg@@QAEXABVQString@@@Z$2 10007254 f   usersEditordlgimpl.obj
 0001:00006260       __unwindfunclet$?save@usersEditorDlg@@QAEXABVQString@@@Z$3 10007260 f   usersEditordlgimpl.obj
 0001:00006269       __unwindfunclet$?save@usersEditorDlg@@QAEXABVQString@@@Z$4 10007269 f   usersEditordlgimpl.obj
 0001:00006272       __unwindfunclet$?save@usersEditorDlg@@QAEXABVQString@@@Z$5 10007272 f   usersEditordlgimpl.obj
 0001:0000627b       __unwindfunclet$?save@usersEditorDlg@@QAEXABVQString@@@Z$6 1000727b f   usersEditordlgimpl.obj
 0001:00006284       __unwindfunclet$?save@usersEditorDlg@@QAEXABVQString@@@Z$7 10007284 f   usersEditordlgimpl.obj
 0001:0000628d       __unwindfunclet$?save@usersEditorDlg@@QAEXABVQString@@@Z$8 1000728d f   usersEditordlgimpl.obj
 0001:00006296       __unwindfunclet$?save@usersEditorDlg@@QAEXABVQString@@@Z$9 10007296 f   usersEditordlgimpl.obj
 0001:0000629f       __unwindfunclet$?save@usersEditorDlg@@QAEXABVQString@@@Z$10 1000729f f   usersEditordlgimpl.obj
 0001:000062a8       __unwindfunclet$?save@usersEditorDlg@@QAEXABVQString@@@Z$11 100072a8 f   usersEditordlgimpl.obj
 0001:000062b1       __unwindfunclet$?save@usersEditorDlg@@QAEXABVQString@@@Z$12 100072b1 f   usersEditordlgimpl.obj
 0001:000062ba       __unwindfunclet$?save@usersEditorDlg@@QAEXABVQString@@@Z$13 100072ba f   usersEditordlgimpl.obj
 0001:000062c3       __unwindfunclet$?save@usersEditorDlg@@QAEXABVQString@@@Z$14 100072c3 f   usersEditordlgimpl.obj
 0001:000062cc       __unwindfunclet$?save@usersEditorDlg@@QAEXABVQString@@@Z$15 100072cc f   usersEditordlgimpl.obj
 0001:000062d5       __unwindfunclet$?save@usersEditorDlg@@QAEXABVQString@@@Z$16 100072d5 f   usersEditordlgimpl.obj
 0001:000062de       __unwindfunclet$?save@usersEditorDlg@@QAEXABVQString@@@Z$17 100072de f   usersEditordlgimpl.obj
 0001:000062e7       __unwindfunclet$?save@usersEditorDlg@@QAEXABVQString@@@Z$18 100072e7 f   usersEditordlgimpl.obj
 0001:000062f0       __ehhandler$?save@usersEditorDlg@@QAEXABVQString@@@Z 100072f0 f   usersEditordlgimpl.obj
 0001:0000630e       __unwindfunclet$?fileSelected@usersEditor@@AAEXABVQString@@@Z$0 1000730e f   usersEditordlgimpl.obj
 0001:0000630e       __unwindfunclet$?setClean@usersEditorDlg@@QAEXXZ$0 1000730e f   usersEditordlgimpl.obj
 0001:0000630e       __unwindfunclet$?closeEvent@usersEditor@@UAEXPAVQCloseEvent@@@Z$0 1000730e f   usersEditordlgimpl.obj
 0001:0000630e       __unwindfunclet$?setDirty@usersEditorDlg@@QAEXXZ$0 1000730e f   usersEditordlgimpl.obj
 0001:00006317       __ehhandler$?fileSelected@usersEditor@@AAEXABVQString@@@Z 10007317 f   usersEditordlgimpl.obj
 0001:00006317       __ehhandler$?setDirty@usersEditorDlg@@QAEXXZ 10007317 f   usersEditordlgimpl.obj
 0001:00006317       __ehhandler$?setClean@usersEditorDlg@@QAEXXZ 10007317 f   usersEditordlgimpl.obj
 0001:00006317       __ehhandler$?closeEvent@usersEditor@@UAEXPAVQCloseEvent@@@Z 10007317 f   usersEditordlgimpl.obj
 0001:00006332       __unwindfunclet$?textChanged@usersEditorDlg@@QAEXHH@Z$0 10007332 f   usersEditordlgimpl.obj
 0001:0000633b       __ehhandler$?textChanged@usersEditorDlg@@QAEXHH@Z 1000733b f   usersEditordlgimpl.obj
 0001:00006356       __unwindfunclet$?toXML@usersEditorDlg@@AAE?AVQString@@ABV2@@Z$0 10007356 f   usersEditordlgimpl.obj
 0001:00006370       __unwindfunclet$?toXML@usersEditorDlg@@AAE?AVQString@@ABV2@@Z$1 10007370 f   usersEditordlgimpl.obj
 0001:00006379       __unwindfunclet$?toXML@usersEditorDlg@@AAE?AVQString@@ABV2@@Z$2 10007379 f   usersEditordlgimpl.obj
 0001:00006382       __unwindfunclet$?toXML@usersEditorDlg@@AAE?AVQString@@ABV2@@Z$3 10007382 f   usersEditordlgimpl.obj
 0001:0000638b       __unwindfunclet$?toXML@usersEditorDlg@@AAE?AVQString@@ABV2@@Z$4 1000738b f   usersEditordlgimpl.obj
 0001:00006394       __unwindfunclet$?toXML@usersEditorDlg@@AAE?AVQString@@ABV2@@Z$5 10007394 f   usersEditordlgimpl.obj
 0001:0000639d       __unwindfunclet$?toXML@usersEditorDlg@@AAE?AVQString@@ABV2@@Z$6 1000739d f   usersEditordlgimpl.obj
 0001:000063a6       __unwindfunclet$?toXML@usersEditorDlg@@AAE?AVQString@@ABV2@@Z$7 100073a6 f   usersEditordlgimpl.obj
 0001:000063af       __unwindfunclet$?toXML@usersEditorDlg@@AAE?AVQString@@ABV2@@Z$8 100073af f   usersEditordlgimpl.obj
 0001:000063b8       __unwindfunclet$?toXML@usersEditorDlg@@AAE?AVQString@@ABV2@@Z$9 100073b8 f   usersEditordlgimpl.obj
 0001:000063c1       __unwindfunclet$?toXML@usersEditorDlg@@AAE?AVQString@@ABV2@@Z$10 100073c1 f   usersEditordlgimpl.obj
 0001:000063ca       __ehhandler$?toXML@usersEditorDlg@@AAE?AVQString@@ABV2@@Z 100073ca f   usersEditordlgimpl.obj
 0001:000063e5       __unwindfunclet$?command@usersEditor@@IAEXVQString@@0@Z$0 100073e5 f   moc_usersEditordlgimpl.obj
 0001:000063e5       __unwindfunclet$?command@usersEditorDlg@@IAEXVQString@@0@Z$0 100073e5 f   moc_usersEditordlgimpl.obj
 0001:000063ee       __unwindfunclet$?command@usersEditor@@IAEXVQString@@0@Z$1 100073ee f   moc_usersEditordlgimpl.obj
 0001:000063ee       __unwindfunclet$?command@usersEditorDlg@@IAEXVQString@@0@Z$1 100073ee f   moc_usersEditordlgimpl.obj
 0001:000063f7       __unwindfunclet$?command@usersEditor@@IAEXVQString@@0@Z$2 100073f7 f   moc_usersEditordlgimpl.obj
 0001:000063f7       __unwindfunclet$?command@usersEditorDlg@@IAEXVQString@@0@Z$2 100073f7 f   moc_usersEditordlgimpl.obj
 0001:0000640b       __ehhandler$?command@usersEditorDlg@@IAEXVQString@@0@Z 1000740b f   moc_usersEditordlgimpl.obj
 0001:0000640b       __ehhandler$?command@usersEditor@@IAEXVQString@@0@Z 1000740b f   moc_usersEditordlgimpl.obj
 0001:00006430       __unwindfunclet$?qt_emit@usersEditor@@UAE_NHPAUQUObject@@@Z$0 10007430 f   moc_usersEditordlgimpl.obj
 0001:00006430       __unwindfunclet$?qt_emit@usersEditorDlg@@UAE_NHPAUQUObject@@@Z$0 10007430 f   moc_usersEditordlgimpl.obj
 0001:00006439       __ehhandler$?qt_emit@usersEditor@@UAE_NHPAUQUObject@@@Z 10007439 f   moc_usersEditordlgimpl.obj
 0001:00006439       __ehhandler$?qt_emit@usersEditorDlg@@UAE_NHPAUQUObject@@@Z 10007439 f   moc_usersEditordlgimpl.obj
 0001:00006454       __unwindfunclet$??0usersEditorDlgBase@@QAE@PAVQWidget@@PBDI@Z$0 10007454 f   usersEditordlg.obj
 0001:0000645d       __unwindfunclet$??0usersEditorDlgBase@@QAE@PAVQWidget@@PBDI@Z$1 1000745d f   usersEditordlg.obj
 0001:00006467       __unwindfunclet$??0usersEditorDlgBase@@QAE@PAVQWidget@@PBDI@Z$2 10007467 f   usersEditordlg.obj
 0001:00006471       __ehhandler$??0usersEditorDlgBase@@QAE@PAVQWidget@@PBDI@Z 10007471 f   usersEditordlg.obj
 0001:0000648c       __unwindfunclet$?languageChange@usersEditorDlgBase@@MAEXXZ$0 1000748c f   usersEditordlg.obj
 0001:00006495       __unwindfunclet$?languageChange@usersEditorDlgBase@@MAEXXZ$1 10007495 f   usersEditordlg.obj
 0001:0000649e       __unwindfunclet$?languageChange@usersEditorDlgBase@@MAEXXZ$2 1000749e f   usersEditordlg.obj
 0001:000064a7       __ehhandler$?languageChange@usersEditorDlgBase@@MAEXXZ 100074a7 f   usersEditordlg.obj
 0001:000064c2       ??__FcleanUp_bncsTable@@YAXXZ 100074c2 f   moc_bncsTable.obj
 0001:000064cd       ??__FcleanUp_toolWindowBase@@YAXXZ 100074cd f   moc_toolwindow.obj
 0001:000064d8       ??__FcleanUp_toolWindow@@YAXXZ 100074d8 f   moc_toolwindowimpl.obj
 0001:000064e3       ??__FcleanUp_usersEditor@@YAXXZ 100074e3 f   moc_usersEditor.obj
 0001:000064ee       ??__FcleanUp_usersEditorDlgBase@@YAXXZ 100074ee f   moc_usersEditordlg.obj
 0001:000064f9       ??__FcleanUp_usersEditorDlg@@YAXXZ 100074f9 f   moc_usersEditordlgimpl.obj
 0002:00000a2c       _cleanUp_bncsTable$initializer$ 10008a2c     moc_bncsTable.obj
 0002:00000a30       _cleanUp_toolWindowBase$initializer$ 10008a30     moc_toolwindow.obj
 0002:00000a34       _cleanUp_toolWindow$initializer$ 10008a34     moc_toolwindowimpl.obj
 0002:00000a38       _cleanUp_usersEditor$initializer$ 10008a38     moc_usersEditor.obj
 0002:00000a3c       _cleanUp_usersEditorDlgBase$initializer$ 10008a3c     moc_usersEditordlg.obj
 0002:00000a40       _cleanUp_usersEditorDlg$initializer$ 10008a40     moc_usersEditordlgimpl.obj
 0002:00000a4c       _pcinit                    10008a4c     MSVCRT:crtdll.obj
 0002:00000a50       _pinit                     10008a50     MSVCRT:atonexit.obj
 0002:00002694       ?slot_0@?3??staticMetaObject@bncsTable@@SAPAVQMetaObject@@XZ@4UQUMethod@@B 1000a694     moc_bncsTable.obj
 0002:000026a8       ?slot_1@?3??staticMetaObject@bncsTable@@SAPAVQMetaObject@@XZ@4UQUMethod@@B 1000a6a8     moc_bncsTable.obj
 0002:000026bc       ?slot_2@?3??staticMetaObject@bncsTable@@SAPAVQMetaObject@@XZ@4UQUMethod@@B 1000a6bc     moc_bncsTable.obj
 0002:000026d0       ?slot_3@?3??staticMetaObject@bncsTable@@SAPAVQMetaObject@@XZ@4UQUMethod@@B 1000a6d0     moc_bncsTable.obj
 0002:000026e8       ?slot_tbl@?3??staticMetaObject@bncsTable@@SAPAVQMetaObject@@XZ@4QBUQMetaData@@B 1000a6e8     moc_bncsTable.obj
 0002:00002758       ?slot_0@?3??staticMetaObject@toolWindowBase@@SAPAVQMetaObject@@XZ@4UQUMethod@@B 1000a758     moc_toolwindow.obj
 0002:00002774       ?slot_tbl@?3??staticMetaObject@toolWindowBase@@SAPAVQMetaObject@@XZ@4QBUQMetaData@@B 1000a774     moc_toolwindow.obj
 0002:000027b0       ?slot_0@?3??staticMetaObject@toolWindow@@SAPAVQMetaObject@@XZ@4UQUMethod@@B 1000a7b0     moc_toolwindowimpl.obj
 0002:000027d0       ?slot_tbl@?3??staticMetaObject@toolWindow@@SAPAVQMetaObject@@XZ@4QBUQMetaData@@B 1000a7d0     moc_toolwindowimpl.obj
 0002:00002800       ?signal_0@?3??staticMetaObject@toolWindow@@SAPAVQMetaObject@@XZ@4UQUMethod@@B 1000a800     moc_toolwindowimpl.obj
 0002:0000281c       ?signal_tbl@?3??staticMetaObject@toolWindow@@SAPAVQMetaObject@@XZ@4QBUQMetaData@@B 1000a81c     moc_toolwindowimpl.obj
 0002:00002860       ?slot_0@?3??staticMetaObject@usersEditor@@SAPAVQMetaObject@@XZ@4UQUMethod@@B 1000a860     moc_usersEditor.obj
 0002:0000286c       ?slot_tbl@?3??staticMetaObject@usersEditor@@SAPAVQMetaObject@@XZ@4QBUQMetaData@@B 1000a86c     moc_usersEditor.obj
 0002:00002878       ?signal_0@?3??staticMetaObject@usersEditor@@SAPAVQMetaObject@@XZ@4UQUMethod@@B 1000a878     moc_usersEditor.obj
 0002:0000288c       ?signal_tbl@?3??staticMetaObject@usersEditor@@SAPAVQMetaObject@@XZ@4QBUQMetaData@@B 1000a88c     moc_usersEditor.obj
 0002:000028c8       ?slot_0@?3??staticMetaObject@usersEditorDlgBase@@SAPAVQMetaObject@@XZ@4UQUMethod@@B 1000a8c8     moc_usersEditordlg.obj
 0002:000028d4       ?slot_tbl@?3??staticMetaObject@usersEditorDlgBase@@SAPAVQMetaObject@@XZ@4QBUQMetaData@@B 1000a8d4     moc_usersEditordlg.obj
 0002:000028f8       ?slot_0@?3??staticMetaObject@usersEditorDlg@@SAPAVQMetaObject@@XZ@4UQUMethod@@B 1000a8f8     moc_usersEditordlgimpl.obj
 0002:00002910       ?slot_1@?3??staticMetaObject@usersEditorDlg@@SAPAVQMetaObject@@XZ@4UQUMethod@@B 1000a910     moc_usersEditordlgimpl.obj
 0002:00002924       ?slot_2@?3??staticMetaObject@usersEditorDlg@@SAPAVQMetaObject@@XZ@4UQUMethod@@B 1000a924     moc_usersEditordlgimpl.obj
 0002:0000293c       ?slot_tbl@?3??staticMetaObject@usersEditorDlg@@SAPAVQMetaObject@@XZ@4QBUQMetaData@@B 1000a93c     moc_usersEditordlgimpl.obj
 0002:00002994       ?signal_0@?3??staticMetaObject@usersEditorDlg@@SAPAVQMetaObject@@XZ@4UQUMethod@@B 1000a994     moc_usersEditordlgimpl.obj
 0002:000029a0       ?signal_tbl@?3??staticMetaObject@usersEditorDlg@@SAPAVQMetaObject@@XZ@4QBUQMetaData@@B 1000a9a0     moc_usersEditordlgimpl.obj
 0002:00002ec4       _GS_ExceptionPointers      1000aec4     MSVCRT:gs_report.obj
 0002:00003c70       __ehfuncinfo$?doCopy@bncsTable@@QAEXXZ 1000bc70     bncsTable.obj
 0002:00003c94       __unwindtable$?doCopy@bncsTable@@QAEXXZ 1000bc94     bncsTable.obj
 0002:00003cbc       __unwindtable$??1userLevelTableItem@@UAE@XZ 1000bcbc     panelsetsTableItem.obj
 0002:00003cbc       __unwindtable$??1panelsetsTableItem@@UAE@XZ 1000bcbc     panelsetsTableItem.obj
 0002:00003cc4       __ehfuncinfo$??1panelsetsTableItem@@UAE@XZ 1000bcc4     panelsetsTableItem.obj
 0002:00003cc4       __ehfuncinfo$??1userLevelTableItem@@UAE@XZ 1000bcc4     panelsetsTableItem.obj
 0002:00003ce8       __ehfuncinfo$?createEditor@panelsetsTableItem@@UBEPAVQWidget@@XZ 1000bce8     panelsetsTableItem.obj
 0002:00003d0c       __unwindtable$?createEditor@panelsetsTableItem@@UBEPAVQWidget@@XZ 1000bd0c     panelsetsTableItem.obj
 0002:00003d84       __unwindtable$?keys@plugindesc@@UAE?AVQStringList@@ABVQString@@0@Z 1000bd84     plugindesc.obj
 0002:00003d94       __ehfuncinfo$?keys@plugindesc@@UAE?AVQStringList@@ABVQString@@0@Z 1000bd94     plugindesc.obj
 0002:00003db8       __unwindtable$??0userLevelTableItem@@QAE@ABVQString@@PAVQTable@@W4EditType@QTableItem@@0@Z 1000bdb8     userLevelTableItem.obj
 0002:00003db8       __unwindtable$??0panelsetsTableItem@@QAE@ABVQString@@PAVQTable@@W4EditType@QTableItem@@0@Z 1000bdb8     userLevelTableItem.obj
 0002:00003dc8       __ehfuncinfo$??0userLevelTableItem@@QAE@ABVQString@@PAVQTable@@W4EditType@QTableItem@@0@Z 1000bdc8     userLevelTableItem.obj
 0002:00003dc8       __ehfuncinfo$??0panelsetsTableItem@@QAE@ABVQString@@PAVQTable@@W4EditType@QTableItem@@0@Z 1000bdc8     userLevelTableItem.obj
 0002:00003dec       __ehfuncinfo$?createEditor@userLevelTableItem@@UBEPAVQWidget@@XZ 1000bdec     userLevelTableItem.obj
 0002:00003e10       __unwindtable$?createEditor@userLevelTableItem@@UBEPAVQWidget@@XZ 1000be10     userLevelTableItem.obj
 0002:00003e50       __unwindtable$?setContentFromEditor@userLevelTableItem@@UAEXPAVQWidget@@@Z 1000be50     userLevelTableItem.obj
 0002:00003e50       __unwindtable$?setContentFromEditor@panelsetsTableItem@@UAEXPAVQWidget@@@Z 1000be50     userLevelTableItem.obj
 0002:00003e60       __ehfuncinfo$?setContentFromEditor@userLevelTableItem@@UAEXPAVQWidget@@@Z 1000be60     userLevelTableItem.obj
 0002:00003e60       __ehfuncinfo$?setContentFromEditor@panelsetsTableItem@@UAEXPAVQWidget@@@Z 1000be60     userLevelTableItem.obj
 0002:00003e84       __unwindtable$??1QDockWindowList@@UAE@XZ 1000be84     usersEditor.obj
 0002:00003e94       __ehfuncinfo$??1QDockWindowList@@UAE@XZ 1000be94     usersEditor.obj
 0002:00003eb8       __unwindtable$??1QPopupMenuList@@UAE@XZ 1000beb8     usersEditor.obj
 0002:00003ec0       __ehfuncinfo$??1QPopupMenuList@@UAE@XZ 1000bec0     usersEditor.obj
 0002:00003ee4       __unwindtable$??0config_plugin_base@@QAE@ABVQString@@00@Z 1000bee4     usersEditor.obj
 0002:00003f04       __ehfuncinfo$??0config_plugin_base@@QAE@ABVQString@@00@Z 1000bf04     usersEditor.obj
 0002:00003f28       __unwindtable$??1config_plugin_base@@UAE@XZ 1000bf28     usersEditor.obj
 0002:00003f40       __ehfuncinfo$??1config_plugin_base@@UAE@XZ 1000bf40     usersEditor.obj
 0002:00003f64       __unwindtable$?about@config_plugin_base@@UAE?AVQString@@XZ 1000bf64     usersEditor.obj
 0002:00003f74       __ehfuncinfo$?about@config_plugin_base@@UAE?AVQString@@XZ 1000bf74     usersEditor.obj
 0002:00003f98       __ehfuncinfo$??0usersEditor@@QAE@ABVQString@@00@Z 1000bf98     usersEditor.obj
 0002:00003fbc       __unwindtable$??0usersEditor@@QAE@ABVQString@@00@Z 1000bfbc     usersEditor.obj
 0002:000040e4       __ehfuncinfo$??1usersEditor@@UAE@XZ 1000c0e4     usersEditor.obj
 0002:00004108       __unwindtable$??1usersEditor@@UAE@XZ 1000c108     usersEditor.obj
 0002:00004138       __unwindtable$?toolbars@usersEditor@@UAE?AVQDockWindowList@@XZ 1000c138     usersEditor.obj
 0002:00004140       __ehfuncinfo$?toolbars@usersEditor@@UAE?AVQDockWindowList@@XZ 1000c140     usersEditor.obj
 0002:00004164       __unwindtable$?menus@usersEditor@@UAE?AVQPopupMenuList@@XZ 1000c164     usersEditor.obj
 0002:0000416c       __ehfuncinfo$?menus@usersEditor@@UAE?AVQPopupMenuList@@XZ 1000c16c     usersEditor.obj
 0002:00004190       __ehfuncinfo$?reply@usersEditor@@UAEXPAVresponse@@@Z 1000c190     usersEditor.obj
 0002:000041b4       __unwindtable$?reply@usersEditor@@UAEXPAVresponse@@@Z 1000c1b4     usersEditor.obj
 0002:00004234       __unwindtable$?navigate@usersEditor@@UAEXABVQString@@0@Z 1000c234     usersEditor.obj
 0002:0000424c       __ehfuncinfo$?navigate@usersEditor@@UAEXABVQString@@0@Z 1000c24c     usersEditor.obj
 0002:00004270       __ehfuncinfo$?activate@usersEditor@@UAEX_N@Z 1000c270     usersEditor.obj
 0002:00004294       __unwindtable$?activate@usersEditor@@UAEX_N@Z 1000c294     usersEditor.obj
 0002:0000430c       __unwindtable$?apply@usersEditor@@UAEXXZ 1000c30c     usersEditor.obj
 0002:00004324       __ehfuncinfo$?apply@usersEditor@@UAEXXZ 1000c324     usersEditor.obj
 0002:00004348       __ehfuncinfo$?about@usersEditor@@UAE?AVQString@@XZ 1000c348     usersEditor.obj
 0002:0000436c       __unwindtable$?about@usersEditor@@UAE?AVQString@@XZ 1000c36c     usersEditor.obj
 0002:00004394       __unwindtable$??4?$QGuardedPtr@VQDockWindow@@@@QAEAAV0@PAVQDockWindow@@@Z 1000c394     usersEditor.obj
 0002:00004394       __unwindtable$?create@plugindesc@@UAEPAVconfig_plugin_base@@ABVQString@@00@Z 1000c394     usersEditor.obj
 0002:00004394       __unwindtable$??0?$QGuardedPtr@VQDockWindow@@@@QAE@XZ 1000c394     usersEditor.obj
 0002:00004394       __unwindtable$??0?$QGuardedPtr@VQPopupMenu@@@@QAE@XZ 1000c394     usersEditor.obj
 0002:00004394       __unwindtable$??4?$QGuardedPtr@VQPopupMenu@@@@QAEAAV0@PAVQPopupMenu@@@Z 1000c394     usersEditor.obj
 0002:0000439c       __ehfuncinfo$??0?$QGuardedPtr@VQDockWindow@@@@QAE@XZ 1000c39c     usersEditor.obj
 0002:0000439c       __ehfuncinfo$??0?$QGuardedPtr@VQPopupMenu@@@@QAE@XZ 1000c39c     usersEditor.obj
 0002:0000439c       __ehfuncinfo$?create@plugindesc@@UAEPAVconfig_plugin_base@@ABVQString@@00@Z 1000c39c     usersEditor.obj
 0002:0000439c       __ehfuncinfo$??4?$QGuardedPtr@VQPopupMenu@@@@QAEAAV0@PAVQPopupMenu@@@Z 1000c39c     usersEditor.obj
 0002:0000439c       __ehfuncinfo$??4?$QGuardedPtr@VQDockWindow@@@@QAEAAV0@PAVQDockWindow@@@Z 1000c39c     usersEditor.obj
 0002:000043c0       __unwindtable$??1?$QDict@VQAction@@@@UAE@XZ 1000c3c0     usersEditor.obj
 0002:000043c8       __ehfuncinfo$??1?$QDict@VQAction@@@@UAE@XZ 1000c3c8     usersEditor.obj
 0002:000043ec       __unwindtable$?db@@YAXABVQString@@@Z 1000c3ec     usersEditor.obj
 0002:000043f4       __ehfuncinfo$?db@@YAXABVQString@@@Z 1000c3f4     usersEditor.obj
 0002:00004418       __ehfuncinfo$??0usersEditorDlg@@QAE@ABVQString@@PAVQWidget@@PBDI@Z 1000c418     usersEditordlgimpl.obj
 0002:0000443c       __unwindtable$??0usersEditorDlg@@QAE@ABVQString@@PAVQWidget@@PBDI@Z 1000c43c     usersEditordlgimpl.obj
 0002:0000449c       __unwindtable$??1usersEditorDlg@@UAE@XZ 1000c49c     usersEditordlgimpl.obj
 0002:000044ac       __ehfuncinfo$??1usersEditorDlg@@UAE@XZ 1000c4ac     usersEditordlgimpl.obj
 0002:000044d0       __ehfuncinfo$?load@usersEditorDlg@@QAE_NABVQString@@@Z 1000c4d0     usersEditordlgimpl.obj
 0002:000044f4       __unwindtable$?load@usersEditorDlg@@QAE_NABVQString@@@Z 1000c4f4     usersEditordlgimpl.obj
 0002:0000460c       __ehfuncinfo$?save@usersEditorDlg@@QAEXABVQString@@@Z 1000c60c     usersEditordlgimpl.obj
 0002:00004630       __unwindtable$?save@usersEditorDlg@@QAEXABVQString@@@Z 1000c630     usersEditordlgimpl.obj
 0002:000046e0       __unwindtable$?setDirty@usersEditorDlg@@QAEXXZ 1000c6e0     usersEditordlgimpl.obj
 0002:000046e0       __unwindtable$?closeEvent@usersEditor@@UAEXPAVQCloseEvent@@@Z 1000c6e0     usersEditordlgimpl.obj
 0002:000046e0       __unwindtable$?fileSelected@usersEditor@@AAEXABVQString@@@Z 1000c6e0     usersEditordlgimpl.obj
 0002:000046e0       __unwindtable$?setClean@usersEditorDlg@@QAEXXZ 1000c6e0     usersEditordlgimpl.obj
 0002:000046e8       __ehfuncinfo$?closeEvent@usersEditor@@UAEXPAVQCloseEvent@@@Z 1000c6e8     usersEditordlgimpl.obj
 0002:000046e8       __ehfuncinfo$?setClean@usersEditorDlg@@QAEXXZ 1000c6e8     usersEditordlgimpl.obj
 0002:000046e8       __ehfuncinfo$?setDirty@usersEditorDlg@@QAEXXZ 1000c6e8     usersEditordlgimpl.obj
 0002:000046e8       __ehfuncinfo$?fileSelected@usersEditor@@AAEXABVQString@@@Z 1000c6e8     usersEditordlgimpl.obj
 0002:0000470c       __unwindtable$?textChanged@usersEditorDlg@@QAEXHH@Z 1000c70c     usersEditordlgimpl.obj
 0002:00004714       __ehfuncinfo$?textChanged@usersEditorDlg@@QAEXHH@Z 1000c714     usersEditordlgimpl.obj
 0002:00004738       __ehfuncinfo$?addUser@usersEditorDlg@@QAEXXZ 1000c738     usersEditordlgimpl.obj
 0002:0000475c       __unwindtable$?addUser@usersEditorDlg@@QAEXXZ 1000c75c     usersEditordlgimpl.obj
 0002:000047d4       __unwindtable$?deleteUser@usersEditorDlg@@QAEXXZ 1000c7d4     usersEditordlgimpl.obj
 0002:000047dc       __ehfuncinfo$?deleteUser@usersEditorDlg@@QAEXXZ 1000c7dc     usersEditordlgimpl.obj
 0002:00004800       __ehfuncinfo$?toXML@usersEditorDlg@@AAE?AVQString@@ABV2@@Z 1000c800     usersEditordlgimpl.obj
 0002:00004824       __unwindtable$?toXML@usersEditorDlg@@AAE?AVQString@@ABV2@@Z 1000c824     usersEditordlgimpl.obj
 0002:0000487c       __unwindtable$??1?$QPtrList@VQPopupMenu@@@@UAE@XZ 1000c87c     usersEditordlgimpl.obj
 0002:0000487c       __unwindtable$??1?$QPtrList@H@@UAE@XZ 1000c87c     usersEditordlgimpl.obj
 0002:00004884       __ehfuncinfo$??1?$QPtrList@VQPopupMenu@@@@UAE@XZ 1000c884     usersEditordlgimpl.obj
 0002:00004884       __ehfuncinfo$??1?$QPtrList@H@@UAE@XZ 1000c884     usersEditordlgimpl.obj
 0002:000048a8       __unwindtable$?qt_emit@usersEditorDlg@@UAE_NHPAUQUObject@@@Z 1000c8a8     moc_usersEditordlgimpl.obj
 0002:000048a8       __unwindtable$?qt_emit@usersEditor@@UAE_NHPAUQUObject@@@Z 1000c8a8     moc_usersEditordlgimpl.obj
 0002:000048b0       __ehfuncinfo$?qt_emit@usersEditorDlg@@UAE_NHPAUQUObject@@@Z 1000c8b0     moc_usersEditordlgimpl.obj
 0002:000048b0       __ehfuncinfo$?qt_emit@usersEditor@@UAE_NHPAUQUObject@@@Z 1000c8b0     moc_usersEditordlgimpl.obj
 0002:000048d4       __unwindtable$?command@usersEditor@@IAEXVQString@@0@Z 1000c8d4     moc_usersEditordlgimpl.obj
 0002:000048d4       __unwindtable$?command@usersEditorDlg@@IAEXVQString@@0@Z 1000c8d4     moc_usersEditordlgimpl.obj
 0002:000048ec       __ehfuncinfo$?command@usersEditor@@IAEXVQString@@0@Z 1000c8ec     moc_usersEditordlgimpl.obj
 0002:000048ec       __ehfuncinfo$?command@usersEditorDlg@@IAEXVQString@@0@Z 1000c8ec     moc_usersEditordlgimpl.obj
 0002:00004910       __unwindtable$??0usersEditorDlgBase@@QAE@PAVQWidget@@PBDI@Z 1000c910     usersEditordlg.obj
 0002:00004928       __ehfuncinfo$??0usersEditorDlgBase@@QAE@PAVQWidget@@PBDI@Z 1000c928     usersEditordlg.obj
 0002:0000494c       __unwindtable$?languageChange@usersEditorDlgBase@@MAEXXZ 1000c94c     usersEditordlg.obj
 0002:00004964       __ehfuncinfo$?languageChange@usersEditorDlgBase@@MAEXXZ 1000c964     usersEditordlg.obj
 0002:00004988       __sehtable$__onexit        1000c988     MSVCRT:atonexit.obj
 0002:000049a8       __sehtable$??_L@YGXPAXIHP6EX0@Z1@Z 1000c9a8     MSVCRT:ehvecctr.obj
 0002:000049c8       __sehtable$??_M@YGXPAXIHP6EX0@Z@Z 1000c9c8     MSVCRT:ehvecdtr.obj
 0002:000049e8       __sehtable$?__ArrayUnwind@@YGXPAXIHP6EX0@Z@Z 1000c9e8     MSVCRT:ehvecdtr.obj
 0002:00004a08       __sehtable$___DllMainCRTStartup 1000ca08     MSVCRT:crtdll.obj
 0002:00004a30       __sehtable$__IsNonwritableInCurrentImage 1000ca30     MSVCRT:pesect.obj
 0002:00004a50       .edata                     1000ca50     usersEditor.exp
 0002:00004a78       rgpv                       1000ca78     usersEditor.exp
 0002:00004a7c       rgszName                   1000ca7c     usersEditor.exp
 0002:00004a80       rgwOrd                     1000ca80     usersEditor.exp
 0002:00004a82       szName                     1000ca82     usersEditor.exp
 0002:00004a92       $N00001                    1000ca92     usersEditor.exp
 0002:0000555c       .idata$6                   1000d55c     config_icons:config_icons.dll
 0002:0000b8fc       .idata$6                   100138fc     qt-mt323:qt-mt323.dll
 0002:0000b94c       .idata$6                   1001394c     MSVCRT:MSVCR120.dll
 0002:0000bb60       .idata$6                   10013b60     kernel32:KERNEL32.dll
 0003:00000000       _usersEditor_XPM           10014000     plugindesc.obj
 0003:00000044       ?param_slot_0@?3??staticMetaObject@usersEditor@@SAPAVQMetaObject@@XZ@4QBUQUParameter@@B 10014044     moc_usersEditor.obj
 0003:00000054       ?param_slot_0@?3??staticMetaObject@usersEditorDlg@@SAPAVQMetaObject@@XZ@4QBUQUParameter@@B 10014054     moc_usersEditordlgimpl.obj
 0003:0000052c       _cleanUp_bncsTable         1001452c     moc_bncsTable.obj
 0003:00000534       _cleanUp_toolWindowBase    10014534     moc_toolwindow.obj
 0003:0000053c       _cleanUp_toolWindow        1001453c     moc_toolwindowimpl.obj
 0003:00000540       ?param_slot_0@?3??staticMetaObject@toolWindow@@SAPAVQMetaObject@@XZ@4QBUQUParameter@@B 10014540     moc_toolwindowimpl.obj
 0003:00000550       ?$S1@?3??staticMetaObject@toolWindow@@SAPAVQMetaObject@@XZ@4IA 10014550     moc_toolwindowimpl.obj
 0003:00000554       ?param_signal_0@?3??staticMetaObject@toolWindow@@SAPAVQMetaObject@@XZ@4QBUQUParameter@@B 10014554     moc_toolwindowimpl.obj
 0003:00000568       _cleanUp_usersEditor       10014568     moc_usersEditor.obj
 0003:0000056c       ?$S1@?3??staticMetaObject@usersEditor@@SAPAVQMetaObject@@XZ@4IA 1001456c     moc_usersEditor.obj
 0003:00000570       ?param_signal_0@?3??staticMetaObject@usersEditor@@SAPAVQMetaObject@@XZ@4QBUQUParameter@@B 10014570     moc_usersEditor.obj
 0003:00000594       _cleanUp_usersEditorDlgBase 10014594     moc_usersEditordlg.obj
 0003:0000059c       _cleanUp_usersEditorDlg    1001459c     moc_usersEditordlgimpl.obj
 0003:000005a0       ?$S1@?3??staticMetaObject@usersEditorDlg@@SAPAVQMetaObject@@XZ@4IA 100145a0     moc_usersEditordlgimpl.obj
 0003:000005a4       ?param_signal_0@?3??staticMetaObject@usersEditorDlg@@SAPAVQMetaObject@@XZ@4QBUQUParameter@@B 100145a4     moc_usersEditordlgimpl.obj
 0003:000005c4       ___proc_attached           100145c4     MSVCRT:crtdll.obj
 0003:000005c8       _GS_ExceptionRecord        100145c8     MSVCRT:gs_report.obj
 0003:00000618       _GS_ContextRecord          10014618     MSVCRT:gs_report.obj
 0003:000008e4       _DebuggerWasPresent        100148e4     MSVCRT:gs_report.obj
 0004:000000a0       $R000000                   100150a0     Script1.res
 0004:00000528       $R000488                   10015528     Script1.res
